:100000006CC700009BC7000099C7000097C700009D
:1000100095C7000093C7000091C700008FC700007C
:100020008DC700008BC7000089C7000087C700008C
:1000300085C700000C94E16581C700007FC7000000
:100040007DC700007BC7000079C7000077C70000AC
:1000500075C7000073C7000071C700000C94F283DD
:100060006DC700000C94DC870C94128867C70000F1
:1000700065C7000063C7000061C700005FC70000DC
:100080005DC700005BC7000059C7000057C70000EC
:1000900055C7000053C7000051C700000C940577F6
:1000A0004DC700004BC7000049C7000047C700000C
:1000B00045C7000043C7000041C700003FC700001C
:1000C0003DC700003BC7000039C700000C9487887B
:1000D0000C94BD8833C700000C9432890C94688955
:1000E0002DC7000020480048324832483248324884
:1000F0003248324832483248324832481247244760
:100100002B47324739473F4744474D4754476B4792
:100110006E4732487247754777477A479447964704
:100120009D47A447B747BE47C5473F8542853185B0
:1001300035853B85798546854A8550855485588522
:100140005E856285668579856C8570857485084ACB
:10015000D73B3BCE016E84BCBFFDC12F3D6C7431DB
:100160009ABD56833DDA3D00C77F11BED9E4BB4C32
:100170003E916BAAAABE000000803F07634236B7DB
:100180009BD8A71A39685618AEBAAB558C1D3CB728
:10019000CC5763BD6DEDFD753EF6177231BF0000A3
:1001A00000803F08000000BE922449123EABAAAA7C
:1001B0002ABECDCCCC4C3E00000080BEABAAAAAA81
:1001C0003E00000000BF000000803F000000000073
:1001D000084178D3BB4387D1133D190E3CC3BD42C0
:1001E00082AD2B3E68EC8276BED98FE1A93E4C8071
:1001F000EFFFBE01C4FF7F3F0000000000003E4D46
:100200006F74696F6E20627920756C747261736FA0
:100210006E632073656E736F723A0A00696E707553
:10022000742044535463616C6962726174653A006E
:100230004E6F20445320546865726D6F6D65746510
:1002400072210050726573732061206B6579004CD8
:100250004344206F6E00234E6F2073656E736F7280
:1002600020666F7220504D21004E6F2073656E73B3
:100270006F722100504D313A322E353A3130004DF7
:100280006561737572696E672E2E004F3220436F61
:100290006E6300434F3220436F6E630053656E738D
:1002A0006F72206572726F722100234E6F2073652A
:1002B0006E736F722100434F3220436F6E63004DA7
:1002C0006561737572696E670070482076616C7540
:1002D0006500547572626964697479004E6F2073A9
:1002E000656E736F72210049522054656D7065729E
:1002F0006174757265004D6561737572696E672E04
:100300002E004C6967687420496E74656E73697459
:100310007900416E676C65732F0067657453656C77
:10032000665465737442697428293A2000697349D8
:100330006E74657272757074456E61626C65642866
:1003400031293A2000676574496E74657272757060
:10035000744D617070696E672831293A20006765B5
:1003600074496E74657272757074536F75726365DB
:100370002831293A2000676574496E746572727578
:100380007074536F7572636528293A20006765742D
:100390005261746528293A20332E31343135393F82
:1003A00000616363656C2E69734C6F77506F77657E
:1003B0007228293A2000616363656C2E697341736A
:1003C0006C65657028293A2000616363656C2E694D
:1003D00073546170536F757263654F6E5A28293A72
:1003E0002000616363656C2E6973546170536F758F
:1003F0007263654F6E5928293A2000616363656C0A
:100400002E6973546170536F757263654F6E58280F
:10041000293A2000616363656C2E697341637469D6
:1004200076697479536F757263654F6E5A28293AED
:100430002000616363656C2E69734163746976693A
:100440007479536F757263654F6E5928293A20008D
:1004500069734163746976697479536F7572636502
:100460004F6E5828293A20006973546170446574AE
:10047000656374696F6E4F6E5A28293B2066616C04
:1004800073653F20006973546170446574656374DB
:10049000696F6E4F6E5A28293B20747275653F2034
:1004A000006973546170446574656374696F6E4F5D
:1004B0006E5928293B2066616C73653F2000697383
:1004C000546170446574656374696F6E4F6E59282A
:1004D000293B20747275653F200069735461704434
:1004E0006574656374696F6E4F6E5828293B20668A
:1004F000616C73653F200069735461704465746575
:100500006374696F6E4F6E5828293B20747275654D
:100510003F2000676574537570707265737342692C
:100520007428293B2066616C73653F200067657401
:10053000537570707265737342697428293B207417
:100540007275653F200069734163746976697479D7
:10055000416328293A20006973496E6163746976A2
:100560006974795A456E61626C656428293A200085
:100570006973496E616374697669747959456E610E
:10058000626C656428293A20006973496E6163745E
:10059000697669747958456E61626C656428293A98
:1005A0002000697341637469766974795A456E6194
:1005B000626C656428293A20006973416374697626
:1005C00069747959456E61626C656428293A200026
:1005D0006973416374697669747958456E61626CB8
:1005E000656428293A20006765744672656546612E
:1005F0006C6C4475726174696F6E28293A200067CB
:1006000065744672656546616C6C546872657368A2
:100610006F6C6428293A200067657454696D6549D8
:100620006E616374697669747928293A2000676578
:1006300074496E616374697669747954687265731C
:10064000686F6C642829200067657441637469765B
:100650006974795468726573686F6C642829200026
:10066000676574446F75626C6554617057696E6438
:100670006F7728292000676574446F75626C655434
:1006800061704C6174656E637928293A2000676552
:10069000745461704475726174696F6E28293A20D0
:1006A00000676574417869734F66667365742826C0
:1006B000782C2026792C20267A293A200067657428
:1006C0005461705468726573686F6C6428293A20AD
:1006D0000058595A2047733A200058595A20434F1E
:1006E000554E54533A2000736574206761696E73E8
:1006F0005B5D3A006761696E735F6F7269675B5D2E
:100700003A00466C616D65204952004F6666206173
:1007100069722D636F6E6421004974277320746FB2
:100720006F20636F6F6C210054656D7020697320BA
:1007300066696E6521004973206169722D636F6E71
:1007400064206F6E3F00497427732071756974656A
:1007500020686F74210049742773207665727920B0
:10076000686F74210054656D702048756D69646907
:10077000747900234E6F2073656E736F7220666FFD
:10078000722074656D7020262068756D69646974C7
:100790007921004E6F2053656E736F72210054658E
:1007A0006D702048756D6964697479004F666620C4
:1007B0006169722D636F6E64210049742773207420
:1007C0006F6F20636F6F6C210054656D70206973CB
:1007D0002066696E6521004973206169722D636F1F
:1007E0006E64206F6E3F00497427732071756974C1
:1007F0006520686F742100497427732076657279CB
:1008000020686F74212000616E6F746865722049E2
:100810005220696E7075743D006B6579323D006BD6
:100820006579323D00496E76616C6964206B65794B
:1008300021007265706C6965733D00233A53686FDF
:10084000772F48696465204C4344002A3A5468690C
:10085000732048656C700044433A436C65617220B4
:100860004C43440044423A5265736574204C6F67B0
:100870006765720044373A4D6F74696F6E00443695
:100880003A44532054656D700044353A555620491A
:100890006E74656E736974790044343A4F32206324
:1008A0006F6E632E0044333A434F3220636F6E63A2
:1008B0002E0044323A504D28313A322E353A3130FA
:1008C000290044323A504D28313A322E353A3130EF
:1008D000292A0044313A5475726269646974790056
:1008E00044303A566F6C7461676500393A6F722014
:1008F000334420616363656C2E00393A496E636C42
:100900002E20616E672E00383A70482076616C7533
:100910006500373A49522054656D7000373A4952A4
:100920002054656D702A00363A4D61676E657469B2
:1009300063206669656C6400353A476173204C65D5
:1009400076656C00343A495220466C616D6500331F
:100950003A4C6967687420496E742E00323A616EB1
:10096000642048656967687400323A54656D702088
:10097000507265737375726500313A54656D7020FD
:1009800048756D696469747900303A536F756E64A7
:10099000204C6576656C00303A536F756E64204C60
:1009A0006576656C2A002020202020202020202031
:1009B0002020202020002020202020202020202057
:1009C0002020202020002020202020202020202047
:1009D0002020202020200020202020202020202037
:1009E0002020202020202000202020202020202027
:1009F0002020202020202020002020202020202017
:100A0000202020202020202020004C6F6767657266
:100A100020446972656374696F6E002D2D2D2D2D34
:100A20002D2D2D2D2D2D2D2D2D2D2D2D2D2D2D2DF6
:100A30002D2D2D2D2D2D2D2D2D2D2D2D2D2D2D0013
:100A40005265736F6C7574696F6E3A202020004D8B
:100A5000696E2056616C75653A20202020004D613A
:100A6000782056616C75653A2020202000556E690B
:100A70007175652049443A2020202000447269762F
:100A80006572205665723A2020200053656E736FA0
:100A9000723A20202020202020002D2D2D2D204DA9
:100AA00061676E657469632053656E736F72202D84
:100AB0002D2D2D2D2D2D2D2D2D2D2D2D2D2D2D2D66
:100AC0002D2D2D006E6F20484D4335383833206D65
:100AD00061676E657469632073656E736F72202E33
:100AE0002E2E20436865636B20776972696E6721DB
:100AF0000020766F6C746167653D005475726269A1
:100B000064697479205570706572204C696D6974E0
:100B10003A200020766F6C746167653D00547572F1
:100B2000626964697479204C6F776572204C696DD5
:100B300069743A2000547572626964697479204C52
:100B40006F776572204C696D69742056696E663ADC
:100B50002000434F32204D415820766F6C7420287E
:100B600000434F32207A65726F20766F6C742028B4
:100B7000004F322063616C6962726174696F6E3A12
:100B80002000547572626964697479204C6F7765CE
:100B900072204C696D69742056313A2000235061EF
:100BA00072616D6574657273002343616C69627272
:100BB0006174696F6E2050726573737572653D0064
:100BC00023536561206C6576656C20502863616CE9
:100BD00063293D00234572726F723A7072657373B8
:100BE00075726520424D503038352C20636865633E
:100BF0006B20776972696E67210049522054656DD8
:100C0000702073656E736F7220666F756E6400502E
:100C10004D322E352073656E736F72206C696B6573
:100C20006C7920666F756E6400536F756E64204C2E
:100C30006576656C2073656E736F7220666F756E76
:100C4000640053656E736F7220736C6F7420616EF5
:100C50006420747970653A00005EBCE2613FDD8318
:100C6000C29C7E20A3FD1F41009D23BE46DB65F88C
:100C70008C11AF32CA57E97400000A0B02090C0D3F
:100C80000E0807030401000000000000000000003F
:100C90000000000000000000000000000000000054
:100CA0000000000012111000000000000000000011
:100CB0000000000000000000000000000000010231
:100CC000102020080810204010204080020102015E
:100CD0000804020101020408102040808040201016
:100CE000080402018004020180402010080402016F
:100CF00008040201010204081020408001020408D7
:100D000010204080050505050705080808080202AF
:100D100002020A0A08080404040401010101010195
:100D200001010303030303030303040707070C0C78
:100D30000C0C0C0C0C0C020202020606060606063F
:100D400006060B0B0B0B0B0B0B0B000020002300FC
:100D5000260029002C002F003200000100000301B2
:100D60000601090100002200250028002B002E00AA
:100D70003100340002010000050108010B010000F0
:100D80002100240027002A002D003000330001013B
:100D90000000040107010A014E414E494E495459D1
:100DA000494E46CDCCCC3D0AD7233C17B7D1387736
:100DB000CC2B329595E6241FB14F0A00002041004C
:100DC00000C84200401C4620BCBE4CCA1B0E5AAE96
:100DD000C59D7400407A10F35A00A0724E180900A5
:100DE00010A5D4E80000E87648170000E40B540290
:100DF0000000CA9A3B000000E1F5050000809698CB
:100E000000000040420F000000A08601000000101A
:100E10002700000000E8030000000064000000005C
:100E2000000A00000000000100000000002C76D83D
:100E300088DC674F0823DFC1DFAE59E1B1B796E523
:100E4000E3E453C63AE651997696E8E6C28426EB87
:100E5000898C9B62ED407C6FFCEFBC9C9F40F2BA9A
:100E6000A56FA5F490055A2AF75C936B6CF9676D32
:100E7000C11BFCE0E40D47FEF520E6B500D0ED9087
:100E80002E0300943577050080841E080000204E54
:100E90000A000000C80C333333330F986E128311ED
:100EA00041EF8D2114893BE65516CFFEE6DB18D1C4
:100EB000844B381BF77C1D901DA4BBE42420328496
:100EC000725E228100C9F124ECA1E53D2700823643
:100ED0001C764488EF889A89563711241FBECFEFBD
:100EE000D1E2DEBFCDBF00E00CBF1AE0A0E0B2E06F
:100EF000EAEFFBE301E00BBF02C007900D92A63DB5
:100F0000B107D9F720E1A6EDBAE001C01D92A73DD7
:100F1000B207E1F71EE0C8EDDEE000E006C0229770
:100F20000109FE010BBF0E946F96CE3CD10780E005
:100F30000807A9F70E949D910C94EC9D61C8CF927F
:100F4000DF92EF92FF920F931F93E82FF92F05C0C6
:100F5000015011092109310961F1908196239417FB
:100F6000B9F305C0015011092109310911F190812E
:100F700096239413F7CFC12CD12CE12CF12C0AC06D
:100F80008FEFC81AD80AE80AF80A0C151D052E05B5
:100F90003F0579F080818623841791F36C2D7D2D98
:100FA0008E2D9F2D1F910F91FF90EF90DF90CF908E
:100FB000089560E070E080E090E01F910F91FF9055
:100FC000EF90DF90CF9008952DE43AE0FC0131835B
:100FD0002083089508952DE43AE0FC0131832083B5
:100FE0000C94AB912F923F924F925F926F927F92AF
:100FF0008F929F92AF92BF92CF92DF92EF92FF9229
:101000000F931F93CF93DF93CDB7DEB72E970FB615
:10101000F894DEBF0FBECDBF8C017E876D87DC01EB
:101020004D915C91119712962D913C911397421717
:1010300053072CF4942F852FA901292F382FD8017D
:10104000149660E070E0CB01E2E0F0E0ED84FE8415
:10105000EE15FF0544F5CD90DD90C216D3065CF485
:101060004901AA2497FCA094BA2C680D791D8A1D09
:101070009B1D960116C04C155D055CF44A01AA241F
:1010800097FCA094BA2C680D791D8A1D9B1DA601A2
:1010900008C0EE24D7FCE094FE2C6C0D7D1D8E1D47
:1010A0009F1D3196D3CF0E9444936B017C016D85C7
:1010B0007E8562507109882777FD8095982F0E9460
:1010C00044939B01AC01C701B6010E9478926B0169
:1010D0007C012D853E85243131050CF4BFC04801CB
:1010E000412C512C3201A12CB12CD4016D917D9158
:1010F0004D01882777FD8095982F0E944493A70182
:1011000096010E94AD919B01AC010E94D8949B0175
:10111000AC01C301B2010E94AE912B013C01BFEFB3
:10112000AB1ABB0AED85FE85AE16BF06F1F6BF0110
:1011300061507109882777FD8095982F0E9444930C
:101140009B01AC01C301B2010E9478920E948B9571
:101150004B015C0120E030E040E85FE30E9419941D
:1011600018160CF07BC018870F83212C312C1B82A2
:101170001C821D821E821A821982AF81B8858D91D0
:101180009D91B887AF839C01442737FD4095542F2C
:1011900029873A874B875C87CA01B9010E9444932B
:1011A000A70196010E94AD912B013C0120E030E0A7
:1011B000A9010E941994181624F0C301B201905895
:1011C00002C0C301B201A50194010E94749287FF7D
:1011D00013C08B819C81AD81BE8129853A854B8569
:1011E0005C85820F931FA41FB51F8B839C83AD83E7
:1011F000BE833FEF231A330A49815A814F5F5F4F05
:101200005A8349838D859E854817590709F0B5CFC4
:1012100020E030E040EC5FE3C501B4010E94D894C7
:101220004B015C0195E0291631040CF49CCF6B81D5
:101230007C818D819E810E9444936B017C01B10170
:10124000882777FD8095982F0E9444939B01AC01DD
:10125000C701B6010E9478926B017C01C701B601FB
:101260002E960FB6F894DEBF0FBECDBFDF91CF91A3
:101270001F910F91FF90EF90DF90CF90BF90AF90B4
:101280009F908F907F906F905F904F903F902F90A6
:101290000895CF93DF93EC01FB01248135810E94F7
:1012A000E890CE01DF91CF91089526E00C94498714
:1012B000DC01ED91FC910190F081E02D1994EF9209
:1012C000FF920F931F93CF93DF931F92CDB7DEB79B
:1012D0007C01FC0100811181C80169830E94EB99A6
:1012E0006981681719F0C8010E94F399C7010F902E
:1012F000DF91CF911F910F91FF90EF900895EF92A2
:10130000FF920F931F93CF93DF931F921F92CDB73E
:10131000DEB709E11BE089519B407C01C701800FCA
:10132000911FF80161918F019A838983CE01019603
:10133000C6DFFBE00F381F0789F789E19BE00F90BC
:101340000F90DF91CF911F910F91FF90EF90089533
:101350000F931F93CF93DF931F921F92CDB7DEB7EA
:101360000EE51DE0F80160818EED93E09A8389839C
:10137000CE010196A4DFF80161818FED93E09A839D
:101380008983CE0101969BDFC8010F900F90DF91FA
:10139000CF911F910F910895BF92CF92DF92EF925C
:1013A000FF920F931F93CF93DF93CDB7DEB7629772
:1013B0000FB6F894DEBF0FBECDBF6C017B018A0172
:1013C0008091F504882309F480C08091F404882377
:1013D00009F47BC077FF09C0E094F09440E06E2DE3
:1013E00085E49DE00E945E784CC040E060E085E4CA
:1013F0009DE00E945E780E943C8428EE33E040E04D
:1014000050E00E943D96BA01A9012AE0CE01019662
:101410000E94F78EBE016F5F7F4FCE0107960E943C
:10142000808E67E978E0CE0107960E940B90BC01A0
:10143000CE010D960E94808ECE0107960E94968D59
:10144000CE0101960E94968DBE01635F7F4F85E4B9
:101450009DE00E943E8AB98840E06B2D85E49DE0C6
:101460000E945E78E114F10411F4EB2C06C040E018
:101470006E2D85E49DE00E945E78CE010D960E945F
:10148000968DB60185E49DE00E943E8A69EF79E081
:1014900085E49DE00E941B8AF60164816E0D40E0A8
:1014A00085E49DE00E945E780E943C846093410D3B
:1014B0007093420D8093430D9093440DB80188279B
:1014C00077FD8095982F0E946B8462960FB6F894F2
:1014D000DEBF0FBECDBFDF91CF911F910F91FF9067
:1014E000EF90DF90CF90BF9008954F925F926F92F0
:1014F0007F92AF92BF92CF92DF92EF92FF920F93C3
:101500001F93CF93DF93CDB7DEB762970FB6F894F2
:10151000DEBF0FBECDBF6C017B015A018091F50487
:10152000882309F498C08091F404882309F493C0B7
:101530000E943C840091410D1091420D2091430D79
:101540003091440D4090E8045090E9046090EA0422
:101550007090EB04040D151D261D371D0617170787
:101560002807390708F077C0F7FE0AC08701009501
:10157000109540E0602F85E49DE00E945E7847C0B2
:1015800040E060E085E49DE00E945E780E943C843B
:1015900028EE33E040E050E00E943D96BA01A901F8
:1015A0002AE0CE0101960E94F78EBE016F5F7F4F49
:1015B000CE0107960E94808E67E978E0CE010796FB
:1015C0000E940B90BC01CE010D960E94808ECE0130
:1015D00007960E94968DCE0101960E94968DBE01BF
:1015E000635F7F4F85E49DE00E943E8A09891A89E6
:1015F000E114F10441F00E0D1F1D40E0602F85E461
:101600009DE00E945E78CE010D960E94968DB601F7
:1016100085E49DE00E943E8A68EE79E085E49DE0E5
:101620000E941B8AF6016481600F40E085E49DE022
:101630000E945E780E943C846093410D7093420D3D
:101640008093430D9093440DB501882777FD8095D5
:10165000982F0E946B8462960FB6F894DEBF0FBE7F
:10166000CDBFDF91CF911F910F91FF90EF90DF9051
:10167000CF90BF90AF907F906F905F904F90089504
:101680008F929F92AF92BF92CF92DF92EF92FF9292
:101690000F931F93CF93DF937C016B01EA0180913D
:1016A000F504882309F474C08091F404882309F4B4
:1016B0006FC077FF1CC0C094D09441E06C2D85E4CE
:1016C0009DE00E945E78B70185E49DE00E943E8A1D
:1016D00067ED79E085E49DE00E941B8AF701648153
:1016E0006C0D41E085E49DE00E945E783EC00E9462
:1016F0003C840091E8041091E9042091EA043091BF
:10170000EB0480903D0D90903E0DA0903F0DB09069
:10171000400D080D191D2A1D3B1D06171707280728
:101720003907B0F541E06C2D85E49DE00E945E78BC
:10173000B70185E49DE00E943E8A66EC79E085E48D
:101740009DE00E941B8AF70164816C0D41E085E4F5
:101750009DE00E945E780E943C8460933D0D7093F2
:101760003E0D80933F0D9093400DBE01882777FD7D
:101770008095982FDF91CF911F910F91FF90EF905F
:10178000DF90CF90BF90AF909F908F900C946B8420
:10179000DF91CF911F910F91FF90EF90DF90CF904D
:1017A000BF90AF909F908F9008958091F50488230B
:1017B00079F08091F404882359F0E091450DF0917F
:1017C000460D0190F081E02D60E085E49DE01994E4
:1017D00008958091F504882379F08091F40488239A
:1017E00059F06FED85E49DE00E944D8A6DE875E04B
:1017F00085E49DE00C944C8A0895CF93DF93EC012F
:101800008091F5048823A1F08091F404882381F06D
:101810006FED85E49DE00E944D8A8C819D81892B2E
:1018200039F0BE0185E49DE0DF91CF910C943E8AB2
:10183000DF91CF9108958091F504882301F1809183
:10184000F4048823E1F085E49DE00E94587840E0AC
:1018500060E085E49DE00E945E7866EB79E085E4D7
:101860009DE00E941B8A41E060E085E49DE00E94CB
:101870005E7866EA79E085E49DE00C941B8A089521
:10188000CF93DF93CDB7DEB72C970FB6F894DEBFBA
:101890000FBECDBF62E075E0CE0107960E94018EBB
:1018A00067E37DE0CE0107960E94FA8FBC01CE016E
:1018B00001960E94808E48EC50E06FEF7FEFCE01E2
:1018C00001966ADDCE0101960E94968DCE010796A3
:1018D0000E94968D66E075E0CE0107960E94018E0B
:1018E00061E37DE0CE0107960E94FA8FBC01CE0134
:1018F00001960E94808E40ED57E06FEF7FEFCE01A2
:101900000196BEDECE0101960E94968DCE0107960D
:101910000E94968D80915C0D90915D0D019719F458
:1019200067E979E002C069E879E0CE0101960E949A
:101930009F8F48EC50E06FEF7FEFCE010196D5DD31
:10194000CE0101960E94968D69E779E0CE0101965D
:101950000E949F8F40ED57E06FEF7FEFCE01019621
:101960008FDECE0101960E94968D69E679E0CE0168
:1019700001960E949F8F48EC50E06FEF7FEFCE0101
:101980000196B3DDCE0101960E94968D6CE579E05B
:10199000CE0101960E949F8F40ED57E06FEF7FEFE1
:1019A000CE0101966DDECE0101960E94968D6FE408
:1019B00079E0CE0101960E949F8F48EC50E06FEFD6
:1019C0007FEFCE01019691DDCE0101960E94968DAA
:1019D00064E479E0CE0101960E949F8F40ED57E0CC
:1019E0006FEF7FEFCE0101964BDECE0101960E9494
:1019F000968D68E379E0CE0101960E949F8F48ECB6
:101A000050E06FEF7FEFCE0101966FDDCE010196C2
:101A10000E94968D67E279E0CE0101960E949F8F29
:101A200040ED57E06FEF7FEFCE01019629DECE014A
:101A300001960E94968D80915C0D90915D0D0397AB
:101A400019F46CE179E002C062E179E0CE0101961F
:101A50000E949F8F48EC50E06FEF7FEFCE01019620
:101A600044DDCE0101960E94968D67E079E0CE01BB
:101A700001960E949F8F40ED57E06FEF7FEFCE0100
:101A80000196FEDDCE0101960E94968D6AEF78E008
:101A9000CE0101960E949F8F48EC50E06FEF7FEFE0
:101AA000CE01019622DDCE0101960E94968D6BEE4D
:101AB00078E0CE0101960E949F8F40ED57E06FEFD6
:101AC0007FEFCE010196DCDDCE0101960E94968D5E
:101AD00060EE78E0CE0101960E949F8F48EC50E0C6
:101AE0006FEF7FEFCE01019600DDCE0101960E94DF
:101AF000968D63ED78E0CE0101960E949F8F40EDB8
:101B000057E06FEF7FEFCE010196BADDCE0101966F
:101B10000E94968D80915C0D90915D0D029719F455
:101B200062EC78E002C062EB78E0CE0101960E94A0
:101B30009F8F48EC50E06FEF7FEFCE010196D5DC30
:101B4000CE0101960E94968D65EA78E0CE0101965D
:101B50000E949F8F40ED57E06FEF7FEFCE0101961F
:101B60008FDDCE0101960E94968D69E978E0CE0165
:101B700001960E949F8F48EC50E06FEF7FEFCE01FF
:101B80000196B3DCCE0101960E94968D69E878E05B
:101B9000CE0101960E949F8F40ED57E06FEF7FEFDF
:101BA000CE0101966DDDCE0101960E94968D6EE705
:101BB00078E0CE0101960E949F8F48EC50E06FEFD5
:101BC0007FEFCE01019691DCCE0101960E94968DA9
:101BD00064E778E0CE0101960E949F8F40ED57E0C8
:101BE0006FEF7FEFCE0101964BDDCE0101960E9493
:101BF000968D64E678E0CE0101960E949F8F48ECB6
:101C000050E06FEF7FEFCE0101966FDCCE010196C1
:101C10000E94968D67E578E0CE0101960E949F8F25
:101C200040ED57E06FEF7FEFCE01019629DDCE0149
:101C300001960E94968D6BE478E0CE0101960E9499
:101C40009F8F48EC50E06FEF7FEFCE0101964DDCA7
:101C5000CE0101960E94968D6BE378E0CE0101964D
:101C60000E949F8F40ED57E06FEF7FEFCE0101960E
:101C700007DDCE0101960E94968D2C960FB6F89442
:101C8000DEBF0FBECDBFDF91CF9108954F925F921F
:101C90006F927F928F929F92AF92BF92CF92DF927C
:101CA000EF92FF92CF93DF93CDB7DEB72C970FB6AD
:101CB000F894DEBF0FBECDBFBEDD87E59CE00E947D
:101CC0001D7C2B013C0187E59CE00E94AE7B4B0113
:101CD0005C01609138027091390280913A029091D2
:101CE0003B020E944493AB01BC0187E59CE00E944B
:101CF000BA7D6B017C01C301B2010E94449320E0D4
:101D000030E048EC52E40E947892AB01BC0122E042
:101D1000CE0101960E94238FBE016F5F7F4F8FE23D
:101D20009CE00E94888ECE0101960E94968D6BEEFB
:101D300078E08FE29CE00E94D88F6FE27CE085E340
:101D40009CE00E946B8E67EE78E0CE0101960E94C7
:101D5000018E6FE27CE0CE0101960E94FA8FBC01F9
:101D60008FE29CE00E946B8ECE0101960E94968DC0
:101D70006BEA76E08BE39CE00E949E8E21E0B50149
:101D8000A401CE0101960E94238FBE016F5F7F4F99
:101D90008BE39CE00E94D28FCE0101960E94968D2B
:101DA0006BE075E08BE39CE00E94D88F21E0B701E7
:101DB000A601CE0107960E94238FBE01695F7F4F67
:101DC000CE0101960E94808E63E476E0CE010196FA
:101DD0000E940B90BC018BE39CE00E94D28FCE014D
:101DE00001960E94968DCE0107960E94968D6FE215
:101DF0007CE0CE0101960E94808E62E275E0CE0109
:101E000001960E940B906BE37CE00E94FA8FBC016C
:101E10008BE39CE00E946B8ECE0101960E94968D12
:101E200065E37CE0CE0101960E94808E4AE050E09E
:101E300060E070E0CE010196AFDACE0101960E941B
:101E4000968D21E0B501A401CE0101960E94238F59
:101E5000BE016F5F7F4F81E49CE00E94888ECE01BF
:101E600001960E94968D61E47CE0CE0101960E946D
:101E7000808E4AE050E06FEF7FEFCE01019600DCEC
:101E8000CE0101960E94968D61E175E0CE0101962A
:101E90000E94018ECE010196B0DCCE0101960E9417
:101EA000968D21E0B701A601CE0107960E94238FEF
:101EB000BE01695F7F4FCE0101960E94808E63E470
:101EC00076E0CE0101960E940B90BC0181E49CE07B
:101ED0000E946B8ECE0101960E94968DCE010796D0
:101EE0000E94968D61E47CE0CE0101960E94808E76
:101EF0004AE050E068EF7FEFCE010196C1DBCE01F2
:101F000001960E94968D80912C0C882331F068E513
:101F100072E080E090E00E946B842C960FB6F894FB
:101F2000DEBF0FBECDBFDF91CF91FF90EF90DF906E
:101F3000CF90BF90AF909F908F907F906F905F9069
:101F40004F900895CF93DF93EC018C819D81892B75
:101F500061F0BE018AEF9EE00E94678ABE0184E3C1
:101F600090E1DF91CF910C94678ADF91CF91089532
:101F70001F93CF93DF93CDB7DEB7A8970FB6F89432
:101F8000DEBF0FBECDBF182F8EE69CE00E94385FEB
:101F900081110EC064EC7AE0CE0101960E949F8F01
:101FA000CE010196CFDFCE0101960E94968DA9C089
:101FB000BE016F5F7F4F8EE69CE00E94165E11238C
:101FC00009F499C06AE97AE08AEF9EE00E94578A94
:101FD0006BE87AE08AEF9EE00E941B8ABE016F5F89
:101FE0007F4F8AEF9EE00E94778A6CE77AE08AEF63
:101FF0009EE00E941B8A4D855E856F8578892AE068
:1020000030E08AEF9EE00E94538B6DE67AE08AEF23
:102010009EE00E941B8A49895A896B897C892AE043
:1020200030E08AEF9EE00E94538B6EE57AE08AEF03
:102030009EE00E941B8A20E030E040E251E4698D7E
:102040007A8D8B8D9C8D0E94D894AB01BC0122E0CF
:1020500030E08AEF9EE00E946F8C64E275E08AEFC8
:102060009EE00E94778A6FE47AE08AEF9EE00E9409
:102070001B8A20E030E040E251E46D8D7E8D8F8D33
:1020800098A10E94D894AB01BC0122E030E08AEF15
:102090009EE00E946F8C64E275E08AEF9EE00E94F1
:1020A000778A60E47AE08AEF9EE00E941B8A20E053
:1020B00030E040E251E469A17AA18BA19CA10E9489
:1020C000D894AB01BC0122E030E08AEF9EE00E9490
:1020D0006F8C64E275E08AEF9EE00E94778A6BE184
:1020E0007AE08AEF9EE00E94578A69EC7AE08AEFF4
:1020F0009EE00E94778A64EF71E080E090E00E94A9
:102100006B84A8960FB6F894DEBF0FBECDBFDF91EB
:10211000CF911F9108954F925F926F927F928F920D
:102120009F92AF92BF92CF92DF92EF92FF920F9366
:102130001F93CF93DF93CDB7DEB7CA54D1090FB643
:10214000F894DEBF0FBECDBF8C0169EC7AE0CE0102
:10215000CD960E94018E69EC7AE0CE01C7960E946E
:10216000018EBE016F5F7F4F8EE69CE00E94D65FBE
:102170004D885E886F88788CC98CDA8CEB8CFC8CEF
:102180008D8D9E8DAF8DB8A12B968CAF9DAFAEAFD0
:10219000BFAF2B97C8010197039708F0E2C1A701D1
:1021A0009601C301B20190580E9421922BED3FE0AD
:1021B00049EC5FE30E94AE912091340230913502E8
:1021C00040913602509137020E94AE914B015C0162
:1021D00020E030E0A9010E94749287FD09C080923E
:1021E0001B0C90921C0CA0921D0CB0921E0C10C0E7
:1021F0002BED3FE049EC50E4C501B4010E94AE91E3
:1022000060931B0C70931C0C80931D0C90931E0C00
:1022100080901B0C90901C0CA0901D0CB0901E0C7C
:102220002BED3FE049EC50E4C501B4010E94199444
:10223000181684F42BED3FE049EC50E4C501B401DD
:102240000E94AD9160931B0C70931C0C80931D0C2D
:1022500090931E0C20E030E044E353E460911B0CAB
:1022600070911C0C80911D0C90911E0C0E94D894B2
:102270002BED3FE049E450E40E9478926093170C04
:102280007093180C8093190C90931A0C0E94119360
:102290004AE0CE018B960E94CC8E68E275E0CE01BA
:1022A00085960E94018EBE01655D7F4FCE018596A9
:1022B0000E94FA8F62E375E00E940B90BC0181E4FA
:1022C0009CE00E946B8ECE0185960E94968DCE0179
:1022D0008B960E94968D8090170C9090180CA09071
:1022E000190CB0901A0C20E030E044EB52E4C50128
:1022F000B4010E947492181694F020E030E040E09F
:102300005FE3C501B4010E94AE910E9411934AE0BF
:10231000CE018B960E94CC8E69E375E023C020E04D
:1023200030E044E353E4C501B4010E9474921816EE
:10233000A4F1A501940160E070E884E393E40E94B5
:10234000AD916093170C7093180C8093190C9093B7
:102350001A0C0E9411934AE0CE018B960E94CC8EFB
:102360006CE375E0CE0185960E94018EBE01655D2D
:102370007F4FCE0185960E94FA8FBC01CE01CD968B
:102380000E946B8ECE0185960E94968DCE018B9613
:102390000E94968D69E379E063C020E030E047E871
:1023A00053E4C501B4010E947492181604F120E0B0
:1023B00030E044E353E4C501B4010E94AD9120E054
:1023C00030E040E05FE30E94AE916093170C7093A1
:1023D000180C8093190C90931A0C0E9411934AE0E8
:1023E000CE018B960E94CC8E6CE375E01FC0A501D8
:1023F000940160E070E084EB93E40E94AD9120E0F2
:1024000030E040E05FE30E94AE916093170C709360
:10241000180C8093190C90931A0C0E9411934AE0A7
:10242000CE018B960E94CC8E69E375E0CE01859635
:102430000E94018EBE01655D7F4FCE0185960E9490
:10244000FA8FBC01CE01CD960E946B8ECE0185968F
:102450000E94968DCE018B960E94968D6FE375E05B
:10246000CE01C7960E949E8EBE01635C7F4FCE0157
:1024700085960E94808E4AE050E060E070E0CE01D8
:1024800085960E94CC09CE0185960E94968D0E9469
:102490003C842091E8043091E9044091EA04509191
:1024A000EB048090410D9090420DA090430DB090B0
:1024B000440D280D391D4A1D5B1D26173707480797
:1024C000590708F441C20E943C840E9442934B0188
:1024D0005C016091E8047091E9048091EA049091B4
:1024E000EB040E94449320E030E040E85EE30E9469
:1024F000D89427966CAF7DAF8EAF9FAF2797609132
:10250000410D7091420D8091430D9091440D0E94B8
:1025100044939B01AC0127966CAD7DAD8EAD9FAD14
:1025200027970E94AE919B01AC01C501B4010E94A6
:10253000749287FD09C262E275E0CE0185960E9421
:10254000018EBE01695C7F4FCE0185960E94FA8F95
:10255000BC01CE01CD960E94D28FCE0185960E94FD
:10256000968DC8010297029708F0C8C120E030E0BC
:1025700040E251E4C301B2010E94D8944B015C01D6
:1025800020E030E040E251E4C701B6010E94D89457
:102590006B017C0120E030E040E251E42B966CAD11
:1025A0007DAD8EAD9FAD2B970E94D8942B013C0141
:1025B0000E943C8420918F0B3091900B4091910BA5
:1025C0005091920B621B730B840B950B0E944293EC
:1025D00020E030E04AE754E40E947892AB01BC016D
:1025E00023E0CE018B960E94238F65E575E0CE0136
:1025F00085960E94018EBE01655D7F4FCE01859656
:102600000E94FA8F67E978E00E940B90BC018FE28C
:102610009CE00E946B8ECE0185960E94968DCE0125
:102620008B960E94968D6FE27CE0CE0185960E948B
:10263000808E61E47CE0CE0185960E94FA8FBE0117
:10264000635C7F4F0E94FA8FBC01CE01CD960E9441
:102650006B8ECE0185960E94968D61E475E08BE3CA
:102660009CE00E949E8E21E0B501A401CE018596DA
:102670000E94238FBE016B5D7F4F8BE39CE00E9425
:10268000D28FCE0185960E94968D21E0B301A201E2
:10269000CE0185960E94238F21E0B701A601CE01CD
:1026A000C1960E94238F62E275E0CE018B960E9454
:1026B000018EBE016F5C7F4FCE018B960E94FA8F18
:1026C00062E275E00E940B90BE016B5D7F4F0E943D
:1026D000FA8F6CE475E00E940B90BC018BE39CE0E8
:1026E0000E94D28FCE018B960E94968DCE01C1960C
:1026F0000E94968DCE0185960E94968DA50194012B
:10270000C501B4010E94D8944B015C01A701960158
:10271000C701B6010E94D8949B01AC01C501B40168
:102720000E94AE916B017C01A3019201C301B20131
:102730000E94D8949B01AC01C701B6010E94AE91E2
:102740000E948B956093130C7093140C8093150C5E
:102750009093160C60E575E08BE39CE00E94D88FA7
:102760004091130C5091140C6091150C7091160C43
:1027700021E0CE018B960E94238FBE01655D7F4FC5
:10278000CE0185960E94808E65E275E0CE01859629
:102790000E940B90BC0181E49CE00E946B8ECE01F4
:1027A00085960E94968DCE018B960E94968D61E44F
:1027B0007CE08BE39CE00E94D28FC090130CD09001
:1027C000140CE090150CF090160C20E030E04AE775
:1027D00054E4C701B6010E94199487FD29C020E086
:1027E00030E04AE754E4C701B6010E947892AB0199
:1027F000BC0123E0CE018B960E94518FBE01655D26
:102800007F4FCE0185960E94808E66E275E0CE01F4
:1028100085960E940B90BC0181E49CE00E946B8E27
:10282000CE0185960E94968DCE018B960E94968D44
:1028300020E030E64AE656E46091130C7091140CE7
:102840008091150C9091160C0E947492BE01635CED
:102850007F4F87FF4FC0CE0185960E94808E64E532
:1028600075E0CE0185960E940B906BE37CE00E94A0
:10287000FA8FBC018BE39CE00E946B8ECE018596A3
:102880000E94968D0330110599F46BE37CE0CE0134
:1028900085960E94808ECE01859654DBCE0185966A
:1028A0000E94968D69EC7AE08BE39CE00E949E8EFC
:1028B00067E575E0CE018B960E94018E61E47CE0B5
:1028C000CE018B960E94FA8FBC01CE0185960E94A4
:1028D000808E4AE050E06FEF7FEFCE0185960E9438
:1028E000400BCE0185960E94968DCE018B960E945C
:1028F000968D04C08BE39CE00E946B8E6AE070E0D2
:1029000080E090E00E946B84CE01C7960E94968D75
:10291000CE01CD960E94968DC65BDF4F0FB6F89420
:10292000DEBF0FBECDBFDF91CF911F910F91FF9002
:10293000EF90DF90CF90BF90AF909F908F907F905F
:102940006F905F904F90089569EC7AE0CE01859684
:102950000E94018ECE0185960E94FD0BCE018596C8
:102960000E94968DBE01695C7F4F85E49DE00E94C8
:102970003E8AE1CD8F929F92AF92BF92CF92DF922B
:10298000EF92FF920F931F93CF93DF9300D000D06D
:10299000CDB7DEB78C01C0900A02D0900B02E09058
:1029A0000C02F0900D0220E030E040E450E4C7015A
:1029B000B6010E94199418166CF420E030E04AE742
:1029C00054E4C701B6010E94D8940E9411936B0190
:1029D0007C0106C080E3C82E85E7D82EE12CF12CBF
:1029E0000E941B0C40E060E085E49DE00E945E7860
:1029F00060E675E085E49DE00E944C8A41E060E07D
:102A000085E49DE00E945E7861E775E085E49DE0E5
:102A10000E944C8A64E670E080E090E00E946B8443
:102A20000E943C8460938F0B7093900B8093910B6A
:102A30009093920B0E943C8480908F0B9090900B0F
:102A4000A090910BB090920BDC01CB0188199909F1
:102A5000AA09BB098C159D05AE05BF055CF4C8012C
:102A60005ADB0E943C8464E170E080E090E00E94C8
:102A70006B84E0CF0130110509F041C06BE37CE0CD
:102A800085E39CE00E946B8E0E941B0C65E37CE05A
:102A9000CE0101960E94808E4AE050E060E070E036
:102AA000CE0101960E94CC09CE0101960E94968D1E
:102AB0006AE07AE0CE0101960E949F8F4AE050E0E2
:102AC0006FEF7FEFCE0101960E94400BCE01019681
:102AD0000E94968D69E775E0CE0101960E94018EF5
:102AE0006BE37CE0CE0101960E94FA8FBC018BE380
:102AF0009CE00E946B8ECE0101960E94968D2696D8
:102B00000FB6F894DEBF0FBECDBFDF91CF911F91FE
:102B10000F91FF90EF90DF90CF90BF90AF909F907C
:102B20008F900895CF92DF92EF92FF92CF93DF9331
:102B300000D000D0CDB7DEB70E941B0C6EE170E074
:102B400080E090E00E946B8487E59CE00E94AE7B71
:102B50006B017C0164E670E080E090E00E946B8491
:102B60006BEA76E08BE39CE00E949E8E21E0B70149
:102B7000A601CE0101960E94238FBE016F5F7F4F99
:102B80008BE39CE00E94D28FCE0101960E94968D2D
:102B90006BE37CE0CE0101960E94808E4AE050E01B
:102BA00060E070E0CE0101960E94CC09CE01019652
:102BB0000E94968D0E94E90B6CE875E08BE39CE027
:102BC0000E94D88FC092230CD092240CE092250C46
:102BD000F092260C20E030E040EF51E4C701B6014E
:102BE0000E94199487FD03C067EF77E054C020E08E
:102BF00030E040ED51E4C701B6010E94199487FD11
:102C00001FC067EE77E0CE0101960E949F8F4AE0D9
:102C100050E06FEF7FEFCE0101960E94400BCE0196
:102C200001960E94968D8091F804882331F06CED16
:102C300075E080E090E00E946B8467ED77E02BC048
:102C400020E030E040EB51E4C701B6010E94199446
:102C500087FD03C069EC77E01EC06AEB77E0CE0128
:102C600001960E949F8F4AE050E06FEF7FEFCE0108
:102C700001960E94400BCE0101960E94968D809194
:102C8000F804882331F06CED75E080E090E00E945C
:102C90006B846CEA77E0CE0101960E949F8F4AE038
:102CA00050E06FEF7FEFCE0101960E94400BCE0106
:102CB00001960E94968D6CE271E080E090E00E94A7
:102CC0006B848091F804882331F068EE73E080E033
:102CD00090E00E946B8426960FB6F894DEBF0FBE7C
:102CE000CDBFDF91CF91FF90EF90DF90CF9008950F
:102CF000CF92DF92EF92FF92CF93DF93CDB7DEB703
:102D00002C970FB6F894DEBF0FBECDBF6EE977E00B
:102D1000CE0101960E949F8F4AE050E06FEF7FEF57
:102D2000CE0101960E94400BCE0101960E94968D25
:102D30006091C6047091C7048FE99CE00E946E7098
:102D4000E12CF12C64E670E080E090E00E946B845E
:102D50006091C6047091C7048FE99CE00E946E7078
:102D60002FEFE21AF20A23E0E216F1045CF32AE004
:102D7000E216F1041CF4892B29F703C0892B09F012
:102D8000D4C06091A10C7091A20C882777FD80952A
:102D9000982F0E9444936B017C016093230C7093E5
:102DA000240C8093250C9093260C60919F0C7091BD
:102DB000A00C882777FD8095982F0E9444936093FC
:102DC0001F0C7093200C8093210C9093220C21E017
:102DD000B701A601CE0107960E94238F6BEA76E029
:102DE000CE0101960E94018EBE01695F7F4FCE0128
:102DF00001960E94FA8FBC018BE39CE00E946B8ECF
:102E0000CE0101960E94968DCE0107960E94968D66
:102E100040911F0C5091200C6091210C7091220C5C
:102E200021E0CE0107960E94238F6FE875E0CE0166
:102E300001960E94018EBE01695F7F4FCE0101960F
:102E40000E94FA8FBC018BE39CE00E94D28FCE01DE
:102E500001960E94968DCE0107960E94968D65E898
:102E600076E08BE39CE00E94D88F69EC7AE0CE019B
:102E700001960E94018E44E150E060E070E0CE01D6
:102E800001960E94CC09CE0101960E94968D609118
:102E9000230C7091240C8091250C9091260C0E949B
:102EA00011934AE0CE0101960E94CC8EBE016F5F65
:102EB0007F4F85E39CE00E94888ECE0101960E94A0
:102EC000968D40E066E085E49DE00E945E7865E3D3
:102ED0007CE085E49DE00E943E8A6FED85E49DE004
:102EE0000E944D8A61E175E085E49DE00E944C8A74
:102EF00060911F0C7091200C8091210C9091220CFC
:102F00000E9411934AE050E085E49DE00E94368BD8
:102F100065E876E085E49DE00E944C8A64E670E016
:102F200080E090E00E946B8418C063E977E0CE01F6
:102F300001960E949F8F4AE050E060E070E0CE0171
:102F400001960E94CC09CE0101960E94968D63E7FE
:102F500077E08BE39CE00E947F8F2C960FB6F8946D
:102F6000DEBF0FBECDBFDF91CF91FF90EF90DF901E
:102F7000CF900895CF92DF92EF92FF92CF93DF939D
:102F8000CDB7DEB72C970FB6F894DEBF0FBECDBF1E
:102F900065E677E0CE0101960E949F8F4CE251E0FA
:102FA0006FEF7FEFCE0101960E94400BCE0101969C
:102FB0000E94968D6091C6047091C7048FE99CE0D1
:102FC0000E946E70E12CF12C64E670E080E090E0ED
:102FD0000E946B846091C6047091C7048FE99CE0E5
:102FE0000E946E702FEFE21AF20A23E0E216F1045B
:102FF0005CF32AE0E216F1041CF4892B29F703C0E4
:10300000892B09F057C16091A10C7091A20C8827FF
:1030100077FD8095982F0E9444936B017C0160930B
:10302000230C7093240C8093250C9093260C6091B4
:103030009F0C7091A00C882777FD8095982F0E9497
:10304000449360931F0C7093200C8093210C9093F9
:10305000220C21E0B701A601CE0107960E94238F22
:103060006BEA76E0CE0101960E94018EBE01695F97
:103070007F4FCE0101960E94FA8FBC018BE39CE04A
:103080000E946B8ECE0101960E94968DCE0107960E
:103090000E94968D40911F0C5091200C6091210C44
:1030A0007091220C21E0CE0107960E94238F6FE8D9
:1030B00075E0CE0101960E94018EBE01695F7F4FCF
:1030C000CE0101960E94FA8FBC018BE39CE00E9426
:1030D000D28FCE0101960E94968DCE0107960E9456
:1030E000968D65E876E08BE39CE00E94D88F69ECD2
:1030F0007AE0CE0101960E94018E44E150E060E04A
:1031000070E0CE0101960E94CC09CE0101960E948A
:10311000968D6091230C7091240C8091250C9091D8
:10312000260C0E9411934AE0CE0101960E94CC8E9B
:10313000BE016F5F7F4F85E39CE00E94888ECE01C9
:1031400001960E94968D40E066E085E49DE00E9435
:103150005E7865E37CE085E49DE00E943E8A6FED49
:1031600085E49DE00E944D8A61E175E085E49DE083
:103170000E944C8A60911F0C7091200C8091210C50
:103180009091220C0E9411934AE050E085E49DE06A
:103190000E94368B65E876E085E49DE00E944C8ACB
:1031A00064E670E080E090E00E946B8487E49CE03D
:1031B0000E948791C090230CD090240CE090250CA5
:1031C000F090260C20E030E040EF51E4C701B6015A
:1031D0000E94199487FD03C066E577E054C020E0A3
:1031E00030E040ED51E4C701B6010E94199487FD1B
:1031F0001FC066E477E0CE0101960E949F8F4AE0EF
:1032000050E06FEF7FEFCE0101960E94400BCE01A0
:1032100001960E94968D8091F804882331F06CED20
:1032200075E080E090E00E946B8466E377E02BC05D
:1032300020E030E040EB51E4C701B6010E94199450
:1032400087FD03C068E277E01EC069E177E0CE0148
:1032500001960E949F8F4AE050E06FEF7FEFCE0112
:1032600001960E94400BCE0101960E94968D80919E
:10327000F804882331F06CED75E080E090E00E9466
:103280006B846BE077E0CE0101960E949F8F4AE04D
:1032900050E06FEF7FEFCE0101960E94400BCE0110
:1032A00001960E94968D62E370E080E090E00E94BB
:1032B0006B8401C037DC2C960FB6F894DEBF0FBECE
:1032C000CDBFDF91CF91FF90EF90DF90CF90089529
:1032D000CF92DF92EF92FF921F93CF93DF93CDB700
:1032E000DEB7AA970FB6F894DEBF0FBECDBF182F7A
:1032F000882331F069EC7AE08AEF9EE00E94778AB9
:1033000083EA9CE00E94F560BE016F5F7F4F83EA15
:103310009CE00E949160CE010D967C01112321F169
:1033200064EF76E08AEF9EE00E94578AFE013196B4
:103330006F01F60141915191619171916F0126E008
:1033400030E08AEF9EE00E946F8C62E275E08AEFC7
:103350009EE00E944C8ACE14DF0459F769EC7AE0B3
:103360008AEF9EE00E94778A23E938E144E85FE330
:1033700069817A818B819C810E94D8946D877E8738
:103380008F87988B22E430E645E85FE36D817E818C
:103390008F8198850E94D894698B7A8B8B8B9C8BBC
:1033A00025E83BEE41E95FE369857A858B859C855D
:1033B0000E94D8946D8B7E8B8F8B988FB70183EA98
:1033C0009CE00E947160112309F48FC0B70183EA69
:1033D0009CE00E94916067EE76E08AEF9EE00E949A
:1033E000578A6E01F9E1CF0ED11CF701419151913D
:1033F000619171917F0122E030E08AEF9EE00E94AE
:103400006F8C62E275E08AEF9EE00E944C8AEC14B9
:10341000FD0459F769EC7AE08AEF9EE00E94778A12
:103420006E01F5E2CF0ED11C9601AE01495D5F4FF2
:10343000BE01675D7F4F83EA9CE00E94E1616AED17
:1034400076E08AEF9EE00E941B8A69A57AA54AE091
:1034500050E08AEF9EE00E94368B62E275E08AEFD0
:103460009EE00E944C8A6FA178A54AE050E08AEF66
:103470009EE00E94368B62E275E08AEF9EE00E9439
:103480004C8A6DA17EA14AE050E08AEF9EE00E9446
:10349000368B69EC7AE08AEF9EE00E94778AB7016A
:1034A00083EA9CE00E941F6261ED76E08AEF9EE075
:1034B0000E941B8AF70141915191619171917F01A5
:1034C0002AE030E08AEF9EE00E946F8C62E275E0B5
:1034D0008AEF9EE00E944C8AEC14FD0459F769ECD7
:1034E0007AE08AEF9EE00E94778A61E070E083EAEA
:1034F0009CE00E940A61112389F06DEB76E08AEF6F
:103500009EE00E941B8A83EA9CE00E9469624AE076
:1035100050E0BC018AEF9EE00E943D8B24E030E049
:1035200043E050E062E070E083EA9CE00E941761B3
:103530001123E9F161EA76E08AEF9EE00E941B8A9E
:103540009E012B5D3F4FAE01495D5F4FBE01675D40
:103550007F4F83EA9CE00E947B6269A57AA54AE0DE
:1035600050E08AEF9EE00E94368B62E275E08AEFBF
:103570009EE00E944C8A6FA178A54AE050E08AEF55
:103580009EE00E94368B62E275E08AEF9EE00E9428
:103590004C8A6DA17EA14AE050E08AEF9EE00E9435
:1035A000368B69EC7AE08AEF9EE00E94778A65E0CC
:1035B00070E083EA9CE00E943461112389F06EE898
:1035C00076E08AEF9EE00E941B8A83EA9CE00E94DC
:1035D000BE624AE050E0BC018AEF9EE00E943D8B53
:1035E00066E070E083EA9CE00E944161112389F06B
:1035F00066E776E08AEF9EE00E941B8A83EA9CE001
:103600000E94D0624AE050E0BC018AEF9EE00E9436
:103610003D8B67E070E083EA9CE00E9444611123E7
:1036200089F060E676E08AEF9EE00E941B8A83EADA
:103630009CE00E94E2624AE050E0BC018AEF9EE01A
:103640000E943D8B68E070E083EA9CE00E9451613B
:10365000112389F068E476E08AEF9EE00E941B8ADD
:1036600083EA9CE00E94F4624AE050E0BC018AEFE9
:103670009EE00E943D8B69E070E083EA9CE00E943E
:103680005E61112389F06EE276E08AEF9EE00E948F
:103690001B8A83EA9CE00E9406634AE050E0BC017A
:1036A0008AEF9EE00E943D8B6AE070E083EA9CE036
:1036B0000E946B61112389F068E176E08AEF9EE059
:1036C0000E941B8A83EA9CE00E9418634AE050E053
:1036D000BC018AEF9EE00E943D8B6BE070E083EAC4
:1036E0009CE00E947861112389F06FEF75E08AEF0A
:1036F0009EE00E941B8A83EA9CE00E942A634AE0C3
:1037000050E0BC018AEF9EE00E943D8B6CE070E0CF
:1037100083EA9CE00E948561112309F48FC067EE63
:1037200075E08AEF9EE00E941B8A83EA9CE00E947B
:103730003C634AE050E0BC018AEF9EE00E943D8B72
:1037400060ED75E08AEF9EE00E941B8A83EA9CE0B0
:103750000E946164682F70E04AE050E08AEF9EE0CA
:103760000E943D8B69EB75E08AEF9EE00E941B8A08
:1037700083EA9CE00E946564682F70E04AE050E0B4
:103780008AEF9EE00E943D8B62EA75E08AEF9EE040
:103790000E941B8A83EA9CE00E946964682F70E0A3
:1037A0004AE050E08AEF9EE00E943D8B69E875E0B8
:1037B0008AEF9EE00E941B8A83EA9CE00E946D646F
:1037C000682F70E04AE050E08AEF9EE00E943D8B57
:1037D00060E775E08AEF9EE00E941B8A83EA9CE026
:1037E0000E947164682F70E04AE050E08AEF9EE02A
:1037F0000E943D8B67E575E08AEF9EE00E941B8A80
:1038000083EA9CE00E947564682F70E04AE050E013
:103810008AEF9EE00E943D8B66E475E08AEF9EE0B1
:103820000E941B8A83EA9CE00E947964682F70E002
:103830004AE050E08AEF9EE00E943D8B61E083EA1F
:103840009CE00E94166461E083EA9CE00E941B6495
:1038500061E083EA9CE00E942064112391F06DE214
:1038600075E08AEF9EE00E941B8A83EA9CE00E943A
:103870007D64682F70E04AE050E08AEF9EE00E948D
:103880003D8B60E083EA9CE00E942064112391F06C
:1038900063E175E08AEF9EE00E941B8A83EA9CE068
:1038A0000E947D64682F70E04AE050E08AEF9EE05D
:1038B0000E943D8B61E083EA9CE00E942564112315
:1038C00091F067EF74E08AEF9EE00E941B8A83EA22
:1038D0009CE00E948164682F70E04AE050E08AEF2B
:1038E0009EE00E943D8B60E083EA9CE00E9425649C
:1038F000112391F06AED74E08AEF9EE00E941B8A2A
:1039000083EA9CE00E948164682F70E04AE050E006
:103910008AEF9EE00E943D8B61E083EA9CE00E947A
:103920002A64112391F06EEB74E08AEF9EE00E940E
:103930001B8A83EA9CE00E948564682F70E04AE05D
:1039400050E08AEF9EE00E943D8B60E083EA9CE0BD
:103950000E942A64112391F061EA74E08AEF9EE0EC
:103960000E941B8A83EA9CE00E948564682F70E0B5
:103970004AE050E08AEF9EE00E943D8B61E083EADE
:103980009CE00E942F64112391F065E874E08AEFB7
:103990009EE00E941B8A83EA9CE00E948964682F53
:1039A00070E04AE050E08AEF9EE00E943D8B60E0CC
:1039B00083EA9CE00E942F64112391F068E674E092
:1039C0008AEF9EE00E941B8A83EA9CE00E94896441
:1039D000682F70E04AE050E08AEF9EE00E943D8B45
:1039E00061E083EA9CE00E94F86361E083EA9CE086
:1039F0000E94FD6361E083EA9CE00E94026460E053
:103A000083EA9CE00E94076460E083EA9CE00E94F5
:103A10000C6460E083EA9CE00E941164112309F4C5
:103A200090C060E574E08AEF9EE00E941B8A83EA02
:103A30009CE00E948D64682F70E04AE050E08AEFBD
:103A40009EE00E943D8B62E374E08AEF9EE00E945C
:103A50001B8A83EA9CE00E949164682F70E04AE030
:103A600050E08AEF9EE00E943D8B64E174E08AEFB3
:103A70009EE00E941B8A83EA9CE00E949564682F66
:103A800070E04AE050E08AEF9EE00E943D8B6BEFD1
:103A900073E08AEF9EE00E941B8A83EA9CE00E940A
:103AA0009964682F70E04AE050E08AEF9EE00E943F
:103AB0003D8B62EE73E08AEF9EE00E941B8A83EAF0
:103AC0009CE00E949D64682F70E04AE050E08AEF1D
:103AD0009EE00E943D8B69EC73E08AEF9EE00E94BD
:103AE0001B8A83EA9CE00E94A164682F70E04AE090
:103AF00050E08AEF9EE00E943D8B66EB73E08AEF18
:103B00009EE00E941B8A83EA9CE00E94A564682FC5
:103B100070E04AE050E08AEF9EE00E943D8B61EA4F
:103B200073E08AEF9EE00E941B8A83EA9CE00E9479
:103B3000A964682F70E04AE050E08AEF9EE00E949E
:103B40003D8B60E083EA9CE00E94346440ED5FE0DE
:103B500069E470E483EA9CE00E947763112309F42E
:103B600049C06DE873E08AEF9EE00E941B8A83EAF9
:103B70009CE00E944E63AB01BC0122E030E08AEF82
:103B80009EE00E94708C66E773E08AEF9EE00E94E0
:103B90001B8A83EA9CE00E94B2634AE050E0682FEF
:103BA0008AEF9EE00E946F8B6EE573E08AEF9EE0E5
:103BB0000E941B8A61E083EA9CE00E94AD64682F4A
:103BC00070E04AE050E08AEF9EE00E943D8B65E4A1
:103BD00073E08AEF9EE00E941B8A61E083EA9CE02A
:103BE0000E94B164682F70E04AE050E08AEF9EE0E6
:103BF0000E943D8B41E061E083EA9CE00E943964D1
:103C0000112399F06DE273E08AEF9EE00E941B8A17
:103C100061E083EA9CE00E94B564682F70E04AE0AE
:103C200050E08AEF9EE00E943D8B41E061E083EA34
:103C30009CE00E943E6460E083EA9CE00E94F363A3
:103C40001123B1F06AE173E08AEF9EE00E941B8AC3
:103C500083EA9CE00E945D64682F70E04AE050E0D7
:103C60008AEF9EE00E943D8B83EA9CE00E94B9644B
:103C7000AA960FB6F894DEBF0FBECDBFDF91CF91ED
:103C80001F91FF90EF90DF90CF9008952F923F9279
:103C90004F925F926F927F928F929F92AF92BF925C
:103CA000CF92DF92EF92FF920F931F93CF93DF9308
:103CB000CDB7DEB7C554D1090FB6F894DEBF0FBE3D
:103CC000CDBF2B013C012DA33EA34FA358A70E94BB
:103CD0003C8422966CAF7DAF8EAF9FAF229720E9D8
:103CE000421621E052066104710434F020E9422EAC
:103CF00055245394612C712C8DA19EA1AFA1B8A520
:103D000080319742A105B1052CF030E127E290E027
:103D100080E004C03DA12EA19FA188A540912C0C5C
:103D2000411104C03DA32EA39FA388A722966CAD8A
:103D30007DAD8EAD9FAD229728EE33E040E050E0A0
:103D40000E943D9626962CAF3DAF4EAF5FAF2697B3
:103D5000F1E0FDAB19A61AA61BA61CA68E01035FF7
:103D60001F4F22273327A90124193509460957096E
:103D700029AB3AAB4BAB5CAB29A53AA54BA55CA5EF
:103D80008DA19EA1AFA1B8A5281739074A075B07E7
:103D90000CF035C369A57AA58BA59CA50E94449318
:103DA00020E030E04AE754E40E947892AB01BC0185
:103DB00023E0C8010E94238FB80185E39CE00E94A4
:103DC000888EC8010E94968D8DA19EA1AFA1B8A535
:103DD0000A97A105B10594F42AE026964CAD5DAD95
:103DE0006EAD7FAD2697C8010E94F78EB80185E3BE
:103DF0009CE00E94888EC8010E94968DBE016F5F74
:103E00007F4F83EA9CE00E941F6265E975E08BE3C7
:103E10009CE00E949E8EDE0111961D01C12CD12CCA
:103E20007601F10181909190A190B1901F01A501BF
:103E30009401C501B4010E94D8949B01AC01C70153
:103E4000B6010E94AE916B017C0123E0B501A40193
:103E5000CE0143960E94518FBE016D5E7F4FC80117
:103E60000E94808E62E275E0C8010E940B90BC0146
:103E70008BE39CE00E94D28FC8010E94968DCE01F8
:103E800043960E94968D2016310659F6C701B60159
:103E90000E948B956B017C01FDE24F16F1E05F06FD
:103EA0006104710444F00E941B0C40E060E085E472
:103EB0009DE00E945E7823E0B701A601C8010E9440
:103EC000238F64E575E0CE0143960E94018E65E381
:103ED0007CE0CE0143960E94FA8F62EA75E00E9470
:103EE0000B90B8010E94FA8F67EA75E00E940B9070
:103EF000BC018BE39CE00E94D28FCE0143960E94CE
:103F0000968DC8010E94968D2DEC3CEC4CE45FE34D
:103F1000C701B6010E94199429813A814B815C81C5
:103F20002DA73EA74FA758AB18160CF0ACC12AE935
:103F300039E949E95FE3C701B6010E94749287FF3E
:103F4000A2C13DA9332309F49EC189849A84AB841C
:103F5000BC8420E030E0A901C501B4010E94749244
:103F6000CD80DE80EF80F884882309F12DA53EA561
:103F70004FA558A9CA01B9010E94D8946EAB7FAB76
:103F800088AF99AFA7019601C701B6010E94D894E6
:103F90009B01AC016EA97FA988AD99AD0E94AE913D
:103FA0000E948B95A50194010E94219204C06BEDA3
:103FB0007FE089EC9FE320EE3EE245E652E40E947A
:103FC000D8946EAB7FAB88AF99AF20E030E0A90109
:103FD000C701B6010E947492882309F12DA53EA560
:103FE0004FA558A9CA01B9010E94D8946AAF7BAF06
:103FF0008CAF9DAFA5019401C501B4010E94D89476
:104000009B01AC016AAD7BAD8CAD9DAD0E94AE91C4
:104010000E948B95A70196010E94219204C06BED2E
:104020007FE089EC9FE320EE3EE245E652E40E9409
:10403000D8946AAF7BAF8CAF9DAF20E030E0A90190
:104040006DA57EA58FA598A90E9474928823F9F08A
:10405000A5019401C501B4010E94D8944B015C01F3
:10406000A7019601C701B6010E94D8949B01AC013B
:10407000C501B4010E94AE910E948B952DA53EA56D
:104080004FA558A90E9421926B017C0108C09BEDAD
:10409000C92E9FE0D92E99ECE92E9FE3F92E65E514
:1040A00075E0C8010E94018E65E37CE0C8010E94B2
:1040B000FA8F6AEA75E00E940B90BC018BE39CE0EA
:1040C0000E946B8EC8010E94968D65E575E0C8015F
:1040D0000E94018E65E37CE0C8010E94FA8F64ECC7
:1040E00075E00E940B90BC0185E39CE00E946B8E02
:1040F000C8010E94968D21E04EA95FA968AD79ADF7
:10410000C8010E94238F21E04AAD5BAD6CAD7DAD4F
:10411000CE0143960E94238F20EE3EE245E652E414
:10412000C701B6010E94D894AB01BC0121E0CE01C9
:104130004F960E94238FBE01615E7F4FCE0149964C
:104140000E94808E62E275E0CE0149960E940B903B
:10415000BE016D5E7F4F0E94FA8F62E275E00E94A1
:104160000B90B8010E94FA8FBC018FE29CE00E9484
:104170006B8ECE0149960E94968DCE014F960E947D
:10418000968DCE0143960E94968DC8010E94968D11
:104190004DE2441641E054066104710474F469A5CB
:1041A0007AA58BA59CA525E030E040E050E00E9478
:1041B0003D96672B682B692BC1F565E37CE0C80150
:1041C0000E94808E45E050E06FEF7FEFC8010E94B3
:1041D000750AC8010E94968D6DEC75E0C8010E94B9
:1041E000018E45E050E061EF7FEFC8010E94CC09ED
:1041F000C8010E94968D69EC7AE0C8010E94018E88
:10420000C8010E94FD0BC8010E94968D6FE27CE000
:10421000C8010E94808E45E050E060E070E0C80177
:104220000E94400BC8010E94968D6FE27CE08BE3F8
:104230009CE00E94D28F5FE1451651046104710435
:1042400034F489A59AA5ABA5BCA5B7FD11C06BE355
:104250007CE0C8010E94808EC8010E94A20FC801A4
:104260000E94968D69EC7AE08BE39CE00E949E8E22
:10427000B201C30177FE04C069A97AA98BA99CA9E0
:104280000E946B84A9C023E04DA55EA56FA578A907
:10429000C8010E94238F65E575E0CE0143960E9418
:1042A000018E65E37CE0CE0143960E94FA8F6FECAD
:1042B00075E00E940B90B8010E94FA8F68EA75E0E1
:1042C0000E940B90BC0185E39CE00E946B8ECE01A6
:1042D00043960E94968DC8010E94968D49855A8505
:1042E0006B857C8523E0C8010E94518F4D815E81E2
:1042F0006F81788523E0CE0149960E94518FBE01DF
:10430000675E7F4FCE0143960E94808E64ED75E01C
:10431000CE0143960E940B90B8010E94FA8F68EA82
:1043200075E00E940B90BC018FE29CE00E946B8EB6
:10433000CE0143960E94968DCE0149960E94968D9D
:10434000C8010E94968D9DE2491691E059066104CC
:10435000710474F469A57AA58BA59CA525E030E0CD
:1043600040E050E00E943D96672B682B692BF1F4EA
:1043700065E37CE0C8010E94808E4AE050E06FEF68
:104380007FEFC8010E94750AC8010E94968D6FE2F6
:104390007CE0C8010E94808E4AE050E060E070E05E
:1043A000C8010E94400BC8010E94968D6BE37CE01F
:1043B000C8010E94808EC8010E94A20FC8010E94FD
:1043C000968D69EC7AE08BE39CE00E949E8EC3019F
:1043D000B2010E946B841DAA0E943C849B01AC0127
:1043E00022968CAD9DADAEADBFAD2297281B390B8B
:1043F0004A0B5B0B29A73AA74BA75CA7BDCC65E38B
:104400007CE0CE010D960E94808E4AE050E06FEF76
:104410007FEFCE010D960E94CC09CE010D960E9431
:10442000968D9DA99923B1F16DEC75E0CE010D96A5
:104430000E94018E45E050E061EF7FEFCE010D96C6
:104440000E94CC09CE010D960E94968D80912C0C75
:10445000882391F062E173E0CE010D960E949F8F58
:1044600045E050E060E070E0CE010D960E94CC097E
:10447000CE010D960E94968D69EC7AE0CE010D96E4
:104480000E94018ECE010D960E94FD0BCE010D966D
:104490000E94968D6FE27CE0CE010D960E94808E88
:1044A0004AE050E06FEF7FEFCE010D960E94400B87
:1044B000CE010D960E94968DCB5BDF4F0FB6F89420
:1044C000DEBF0FBECDBFDF91CF911F910F91FF9047
:1044D000EF90DF90CF90BF90AF909F908F907F90A4
:1044E0006F905F904F903F902F900895CF92DF9202
:1044F000EF92FF920F931F93CF93DF93CDB7DEB769
:104500002C970FB6F894DEBF0FBECDBF80912C0C58
:10451000811102C00E941B0C87E99FE00E94AB87BB
:1045200064E670E080E090E00E946B8466EF72E0E9
:1045300085E39CE00E947F8F65E37CE0CE010196DD
:104540000E94808E44E150E060E070E0CE01019670
:104550000E94CC09CE0101960E94968D67EE72E012
:1045600085E39CE00E947F8F65E37CE0CE010196AD
:104570000E94808E44E150E06FEF7FEFCE01019604
:104580000E94400BCE0101960E94968D60E070E083
:1045900086E29DE00E94F47E6B017C0104E010E065
:1045A000A7019601C701B6010E94CC95882309F4A2
:1045B0003DC00150110909F011C16CED72E085E3B5
:1045C0009CE00E947F8F65E37CE0CE0101960E9413
:1045D000808E4AE050E060E070E0CE0101960E94DB
:1045E000CC09CE0101960E94968D67ED75E0CE0153
:1045F00001960E94018E65E37CE0CE0101960E9447
:10460000FA8FBC018BE39CE00E946B8ECE01019679
:104610000E94968D80915C0D90915D0D039709F03D
:10462000CCC010925D0D10925C0DC7C021E0B701A7
:10463000A601CE0107960E94238F69EE75E0CE0198
:1046400001960E94018EBE01695F7F4FCE010196E7
:104650000E94FA8FBC018BE39CE00E946B8ECE011E
:1046600001960E94968DCE0107960E94968D6BE36F
:104670007CE0CE0101960E94808E42E350E06FEF15
:104680007FEFCE0101960E94400BCE0101960E9461
:10469000968D0E94E90B6CE875E08BE39CE00E942C
:1046A000D88F60E070E086E29DE00E94F27E6B01B0
:1046B0007C0104E010E0A7019601C701B6010E9449
:1046C000CC95882359F00150110909F096C069EC86
:1046D0007AE081E49CE00E949E8E50C021E0B70108
:1046E000A601CE0107960E94238F6BEA76E0CE01E9
:1046F00001960E94018EBE01695F7F4FCE01019637
:104700000E94FA8FBC0181E49CE00E946B8ECE0176
:1047100001960E94968DCE0107960E94968D62E2C8
:1047200075E0CE0101960E94018E61E47CE0CE012D
:1047300001960E94FA8FBC0185E39CE00E946B8E7B
:10474000CE0101960E94968D65E37CE0CE01019634
:104750000E94808E4AE050E060E070E0CE01019659
:104760000E94750ACE0101960E94968D0E94E90B67
:104770006CE875E081E49CE00E94D88F61E47CE005
:10478000CE0101960E94808E62E275E0CE01019614
:104790000E940B906BE37CE00E94FA8FBC018BE3DC
:1047A0009CE00E946B8ECE0101960E94968D83E064
:1047B00090E090935D0D80935C0D64E670E080E086
:1047C00090E00E946B8480912C0C882329F160E298
:1047D00073E080E090E00E946B841EC064E670E0AD
:1047E00080E090E00E946B8460E070E086E29DE0F3
:1047F0000E94F47E6B017C01D3CE68EC70E080E017
:1048000090E00E946B8460E070E086E29DE00E9490
:10481000F27E6B017C014FCF2C960FB6F894DEBF71
:104820000FBECDBFDF91CF911F910F91FF90EF9001
:10483000DF90CF9008951F93CF93DF93182FC3EC91
:10484000DBE0812F0E940185899399936CE370E0EE
:1048500080E090E00E946B848CE0C331D80789F738
:1048600068E270E083EC9BE00E94F20720E030E019
:1048700040EA50E40E94D89420E030E040E85AE357
:104880000E94D894DF91CF911F9108954F925F922B
:104890006F927F928F929F92AF92BF92CF92DF9250
:1048A000EF92FF920F931F93CF93DF93CDB7DEB7B5
:1048B00064970FB6F894DEBF0FBECDBF7C018B01AD
:1048C00062ED72E085E39CE00E947F8F0E941B0CEA
:1048D00065E37CE0CE0101960E94808E4AE050E0C4
:1048E0006FEF7FEFCE0101960E94CC09CE010196B9
:1048F0000E94968DC7019FDF698B7A8B8B8B9C8B77
:1049000040901A0250901B0260901C0270901D0291
:10491000A301920160911602709117028091180212
:10492000909119020E94AD914B015C0120E030E0B2
:10493000A9010E947492882309F451C0C0902202F8
:10494000D0902302E0902402F090250220E030E095
:10495000A901C701B6010E94749218160CF03FC05D
:1049600080911E0290911F02A0912002B09121021D
:104970008D879E87AF87B88B9C01AD01C701B601BB
:104980000E947492882359F1A70196016D857E8556
:104990008F8598890E9478920E9465946D877E87A2
:1049A0008F87988BA301920169897A898B899C8969
:1049B0000E94AD91A50194010E9478922D853E85BB
:1049C0004F8558890E94D8940E94E5929B01AC01C2
:1049D000C701B6010E94D8946B017C0103C0C12CB1
:1049E000D12C760165E37CE0CE0101960E94808E99
:1049F0004AE050E060E070E0CE0101960E94CC09F0
:104A0000CE0101960E94968D20E030E64AEE56E4F3
:104A1000C701B6010E94199418163CF462EF75E0C4
:104A20008BE39CE00E949E8E44C001151105B9F4F1
:104A300021E0B701A601CE0107960E94238F61E015
:104A400076E0CE0101960E94018EBE01695F7F4F24
:104A5000CE0101960E94FA8F65E076E01BC002301D
:104A6000110539F522E049895A896B897C89CE0183
:104A700007960E94238F61E076E0CE0101960E94A6
:104A8000018EBE01695F7F4FCE0101960E94FA8FB1
:104A900069E076E00E940B90BC018BE39CE00E94F1
:104AA0006B8ECE0101960E94968DCE0107960E94D4
:104AB000968D6BE37CE0CE0101960E94808E4AE0E9
:104AC00050E06FEF7FEFCE0101960E94400BCE01C8
:104AD00001960E94968D64E670E080E090E00E946E
:104AE0006B8480912C0C882331F060E273E080E0CD
:104AF00090E00E946B8464960FB6F894DEBF0FBE00
:104B0000CDBFDF91CF911F910F91FF90EF90DF907C
:104B1000CF90BF90AF909F908F907F906F905F905D
:104B20004F9008954F925F926F927F928F929F92D3
:104B3000AF92BF92CF92DF92EF92FF92CF93C82FA6
:104B40008091EE0A81110DC00E943C846093E20ABC
:104B50007093E30A8093E40A9093E50A81E08093DE
:104B6000EE0A8091E60A81110DC00E943C84609398
:104B7000DE0A7093DF0A8093E00A9093E10A81E0F5
:104B80008093E60A1092C20B1092C10BE090C10B09
:104B9000F090C20B88E2E816F1040CF08AC08C2F6A
:104BA0000E940185F701EE0FFF1FED53F44F918333
:104BB000808368E270E083EC9BE00E94F20720E0D3
:104BC00030E040EA50E40E94D89420E030E040E831
:104BD0005AE30E94D8946B017C016093DA0A7093C7
:104BE000DB0A8093DC0A9093DD0A40902A02509001
:104BF0002B0260902C0270902D02A3019201609113
:104C000026027091270280912802909129020E9429
:104C1000AD919B01AC0160E070E080EC90E40E94FB
:104C2000AD914B015C0120E030E0A9010E9474923B
:104C300020E030E040E650E4811105C0C701B60134
:104C40000E94D8941EC0C701B6010E94D894A30147
:104C500092010E94AE9120E030E040E850E40E94D2
:104C6000AD91A50194010E94789220E030E040ECE3
:104C700050E40E94D89420E030E040E850E40E94E4
:104C8000AE916093D60A7093D70A8093D80A909316
:104C9000D90A64E170E080E090E00E946B8480912A
:104CA000C10B9091C20B01969093C20B8093C10BE4
:104CB0006DCF6091D60A7091D70A8091D80A9091F1
:104CC000D90ACF91FF90EF90DF90CF90BF90AF9037
:104CD0009F908F907F906F905F904F900895CF92AC
:104CE000DF92EF92FF92CF93DF93CDB7DEB72C9791
:104CF0000FB6F894DEBF0FBECDBF69EC72E085E35E
:104D00009CE00E947F8F65E37CE0CE0101960E94CB
:104D1000808E4AE050E060E070E0CE0101960E9493
:104D2000CC09CE0101960E94968D809181029091CE
:104D30008202F8DE6B017C0120E030E0A9010E94D4
:104D4000199487FD22C022E0B701A601CE01079683
:104D50000E94238F6BE076E0CE0101960E94018EC7
:104D6000BE01695F7F4FCE0101960E94FA8FBC01A0
:104D70008BE39CE00E946B8ECE0101960E94968D83
:104D8000CE0107960E94968D06C06FE076E08BE319
:104D90009CE00E949E8E6BE37CE0CE0101960E9417
:104DA000808E4AE050E06FEF7FEFCE0101960E94C7
:104DB000400BCE0101960E94968D2C960FB6F8946A
:104DC000DEBF0FBECDBFDF91CF91FF90EF90DF90A0
:104DD000CF9008952F923F924F925F926F927F9261
:104DE0008F929F92AF92BF92CF92DF92EF92FF92FB
:104DF0000F931F93CF93DF9300D01F92CDB7DEB7F1
:104E00006B017C015A8349835901FA012081318168
:104E1000428153810E947492181614F0F50183C0E8
:104E200010E00150104C000F111F000F111FE981FD
:104E3000FA81E00FF11F2081318142815381C70146
:104E4000B6010E94199487FF6BC011E0612E712C8E
:104E50004301880C991C880C991CE981FA81E80DA2
:104E6000F91D2080318042805380A2019101C70149
:104E7000B6010E941994181614F41F5FE7CFA2011F
:104E80009101C701B6010E9474928501080D191D98
:104E9000811102C0F80147C0C3018150904C880FB6
:104EA000991F880F991FA981BA81A80FB91F2D9149
:104EB0003D914D915C9129833A834B835C83F5014D
:104EC000E80FF91F80809180A280B380C701B601EE
:104ED0000E94AD916B017C01A5019401F8016081F4
:104EE0007181828193810E94AD919B01AC01C701C8
:104EF000B6010E94D8946B017C0129813A814B81D3
:104F00005C81C201B1010E94AD919B01AC01C7015E
:104F1000B6010E947892A50194010E94AE9107C04B
:104F2000F501E00FF11F60817181828193810F9003
:104F30000F900F900F90DF91CF911F910F91FF90E5
:104F4000EF90DF90CF90BF90AF909F908F907F9029
:104F50006F905F904F903F902F900895CF92DF9287
:104F6000EF92FF921F93CF93DF93182FCAE0D0E008
:104F7000C12CD12C7601812F0E940185BC0188278C
:104F800077FD8095982F0E9444939B01AC01C70147
:104F9000B6010E94AE916B017C0162E370E080E09B
:104FA00090E00E946B84219731F720E030E040E2EE
:104FB00051E4C701B6010E94789220E030E040EA57
:104FC00050E40E94D89420E030E040E85AE30E9488
:104FD000D894DF91CF911F91FF90EF90DF90CF9009
:104FE0000895FC0120E030E0772767FD7095AB0164
:104FF00042505109DF01A81BB90BA417B50724F4CF
:10500000A1912A0F311DF6CFA9014E5B5F4F860F8C
:10501000971FFC013297208130E0322F22273196F2
:105020008081280F311D81E04217530709F080E08D
:1050300008952F923F924F925F926F927F928F923C
:105040009F92AF92BF92CF92DF92EF92FF920F9317
:105050001F93CF93DF93CDB7DEB763970FB6F89466
:10506000DEBF0FBECDBF8B8B60E00E947A85809142
:105070002C0C811105C08FE090E0A0E0B0E004C0EE
:1050800082E090E0A0E0B0E08F87988BA98BBA8B8C
:1050900063E376E08BE39CE00E949E8E6BE37CE012
:1050A000CE0101960E94808E4AE050E06FEF7FEFC4
:1050B000CE0101960E94CC09CE0101960E94968DE8
:1050C000C12CD12C7601312C1D861E86212C02E3A9
:1050D00010E0412C512C32018B890E940185AA27B6
:1050E00097FDA095BA2F480E591E6A1E7B1E65E0DB
:1050F00070E080E090E00E946B840150110961F73C
:105100008090120290901302A0901402B0901502A9
:10511000C301B2010E94449320E030E040EA50E431
:105120000E94D89420E030E040E85AE30E94D894EE
:1051300020E030E048E452E40E947892A501940116
:105140000E94AD9120E030E040E751E40E94D89405
:105150002B013C01A50194016AE979E989E390E416
:105160000E94AD919B01AC01C301B2010E947892F3
:1051700020E030E0A9010E94AE9120E030E040E262
:1051800051E40E94D8945B018C01232D3D854E850E
:10519000522D0E941994181624F43A2CBD860E87BD
:1051A000212E20E030E0A901B501C8010E947492CF
:1051B00087FF04C0A12CB12C00E010E022E0A50183
:1051C000B801CE0107960E94238FBE01695F7F4F11
:1051D000CE0101960E94808E60E476E0CE010196B9
:1051E0000E940B90BC0185E39CE00E946B8ECE0177
:1051F00001960E94968DCE0107960E94968D65E3DA
:105200007CE0CE0101960E94808E4AE050E060E092
:1052100070E0CE0101960E94400BCE0101960E94E3
:10522000968D0E943C848090E8049090E904A090C0
:10523000EA04B090EB0400913D0D10913E0D2091D9
:105240003F0D3091400D800E911EA21EB31E86169A
:105250009706A806B90608F4DEC00E943C840E94A6
:1052600042934B015C016091E8047091E9048091E4
:10527000EA049091EB040E94449320E030E040E87F
:105280005EE30E94D8942B013C0160913D0D70912A
:105290003E0D80913F0D9091400D0E9444939B01E3
:1052A000AC01C301B2010E94AE919B01AC01C501EA
:1052B000B4010E94749287FDAEC06CE370E080E0A0
:1052C00090E00E946B849FEFC91AD90AE90AF90A93
:1052D0008F859889A989BA898C159D05AE05BF056A
:1052E0000CF0F5CE64E670E080E090E00E946B8404
:1052F0000E941B0C64E670E080E090E00E946B84EA
:1053000065E476E085E39CE00E949E8E65E37CE0A8
:10531000CE0101960E94808E44E150E060E070E092
:10532000CE0101960E94CC09CE0101960E94968D75
:1053300022E0432D5D856E85722DCE0107960E9479
:10534000238FBE01695F7F4FCE0101960E94808E40
:1053500060E476E0CE0101960E940B90BC0185E3EB
:105360009CE00E946B8ECE0101960E94968DCE012C
:1053700007960E94968D65E37CE0CE0101960E941F
:10538000808E42E350E06FEF7FEFCE0101960E94E6
:10539000400BCE0101960E94968D0E94D50B62E3D0
:1053A00070E080E090E00E946B846DE476E0CE01D6
:1053B00001960E94018E65E37CE0CE0101960E9479
:1053C000FA8F61E576E00E940B906BE37CE00E942F
:1053D000FA8FBC018BE39CE00E946B8ECE0101969C
:1053E0000E94968D63960FB6F894DEBF0FBECDBFB8
:1053F000DF91CF911F910F91FF90EF90DF90CF90B1
:10540000BF90AF909F908F907F906F905F904F90E4
:105410003F902F9008950E94D50B4FCFFF920F938E
:105420001F93CF93DF93F82E0AE010E0C0E0D0E0A6
:105430008F2D0E940185C80FD91F65E070E080E0C4
:1054400090E00E946B840150110991F7CE016AE04F
:1054500070E00E94F495CB01DF91CF911F910F91E5
:10546000FF9008950F931F93CF93DF93CDB7DEB7CF
:105470002E970FB6F894DEBF0FBECDBF8D879E87E7
:105480000E941B0C8D859E85C9DF8C0162E370E054
:1054900080E090E00E946B84B801882777FD8095BA
:1054A000982F0E94449320E030E040EA50E40E94AC
:1054B000D89420E030EC4FE754E40E947892AB019E
:1054C000BC0123E0CE0107960E94238F6EE476E0B4
:1054D000CE0101960E94018EBE01695F7F4FCE0111
:1054E00001960E94FA8F67E576E00E940B90BC015E
:1054F0008BE39CE00E946B8ECE0101960E94968DFC
:10550000CE0107960E94968D6AE576E085E39CE0E1
:105510000E949E8E65E37CE0CE0101960E94808E03
:105520004AE050E068E070E0CE0101960E94CC09AC
:10553000CE0101960E94968D6BE37CE0CE01019630
:105540000E94808E4AE050E06FEF7FEFCE0101961F
:105550000E94400BCE0101960E94968D65E37CE08F
:105560008BE39CE00E94D28F80912C0C882331F039
:1055700060E273E080E090E00E946B842E960FB6AC
:10558000F894DEBF0FBECDBFDF91CF911F910F9179
:105590000895CF93DF93CDB7DEB72C970FB6F8946D
:1055A000DEBF0FBECDBF3ADF9093280C8093270C4F
:1055B00062E370E080E090E00E946B846091270CD1
:1055C0007091280C4AE0CE0101960E94CC8EBE015B
:1055D0006F5F7F4F8BE39CE00E94888ECE01019627
:1055E0000E94968D80919D0C90919E0C892B09F4C0
:1055F0005FC069E97CE0CE0107960E94808EBE0103
:10560000695F7F4FCE0101960E94808E44E150E099
:1056100060E070E0CE0101960E94CC09CE010196B7
:105620000E94968D62E676E0CE0101960E94018E80
:105630006BE37CE0CE0101960E94FA8FBC0185E30A
:105640009CE00E946B8ECE0101960E94968D65E3D0
:105650007CE0CE0101960E94808E44E150E06FEF25
:105660007FEFCE0101960E94400BCE0101960E9471
:10567000968DBE01695F7F4FCE0101960E94808E9C
:1056800062E275E0CE0101960E940B9065E37CE03A
:105690000E94FA8FBC018BE39CE00E946B8ECE01CE
:1056A00001960E94968DCE0107960E94968D54C059
:1056B0006DE676E085E39CE00E949E8E65E37CE0EB
:1056C000CE0101960E94808E44E150E060E070E0DF
:1056D000CE0101960E94CC09CE0101960E94968DC2
:1056E00061E776E0CE0101960E94018E6BE37CE0DB
:1056F000CE0101960E94FA8FBC0185E39CE00E94D6
:105700006B8ECE0101960E94968D65E37CE0CE0102
:1057100001960E94808E44E150E06FEF7FEFCE0152
:1057200001960E94400BCE0101960E94968D62E682
:1057300076E0CE0101960E94018E6BE37CE0CE0103
:1057400001960E94FA8FBC018BE39CE00E946B8E55
:10575000CE0101960E94968D80912C0C882331F009
:1057600060E273E080E090E00E946B842C960FB6BC
:10577000F894DEBF0FBECDBFDF91CF9108950F9398
:105780001F93CF93DF93CDB7DEB72C970FB6F89466
:10579000DEBF0FBECDBF8C0181E00E94FE8464E6B7
:1057A00070E080E090E00E946B840E941B0CC801B6
:1057B00035DE60E074E0681B790B4AE0CE010796A5
:1057C0000E94CC8E61E776E0CE0101960E94018EA8
:1057D000BE01695F7F4FCE0101960E94FA8FBC0126
:1057E0008BE39CE00E946B8ECE0101960E94968D09
:1057F000CE0107960E94968D40E066E085E49DE02C
:105800000E945E7862E077E0CE0101960E949F8F51
:1058100042E350E068E070E0CE0101960E94CC09BE
:10582000CE0101960E94968D6BE37CE0CE0101963D
:105830000E94808E42E350E06FEF7FEFCE01019631
:105840000E94400BCE0101960E94968D68E776E09B
:10585000CE0101960E94018E6BE37CE0CE010196A1
:105860000E94FA8FBC018BE39CE00E946B8ECE01FC
:1058700001960E94968D80912C0C882331F060E275
:1058800073E080E090E00E946B842C960FB6F89451
:10589000DEBF0FBECDBFDF91CF911F910F91089555
:1058A0000F9390E0BBDDBC01882777FD8095982F92
:1058B0000E9444932DE038E643E55BE30E94D894D0
:1058C00006E021E532E049E652E084DA20E030E00B
:1058D00048EC52E40E94D89420E030E048EA51E4D9
:1058E0000E94D89420914D0230914E0240914F0277
:1058F000509150020E9478920F910895CF92DF92BA
:10590000EF92FF92CF93DF93CDB7DEB72C970FB610
:10591000F894DEBF0FBECDBFC3DF6B017C016BE827
:1059200072E085E39CE00E947F8F65E37CE0CE011E
:1059300001960E94808E42E350E060E070E0CE016C
:1059400001960E94CC09CE0101960E94968D22E01C
:10595000B701A601CE0107960E94238F6FE176E082
:10596000CE0101960E94018EBE01695F7F4FCE017C
:1059700001960E94FA8F62E876E00E940B90BC01CB
:105980008BE39CE00E946B8ECE0101960E94968D67
:10599000CE0107960E94968D6BE37CE0CE010196C6
:1059A0000E94808E42E350E06FEF7FEFCE010196C0
:1059B0000E94400BCE0101960E94968D80912C0C86
:1059C000882331F060E273E080E090E00E946B8415
:1059D0002C960FB6F894DEBF0FBECDBFDF91CF91EE
:1059E000FF90EF90DF90CF900895CF92DF92EF92EB
:1059F000FF920F9390E012DDBC01882777FD809520
:105A0000982F0E9444932DE038E643E55BE30E9423
:105A1000D89406E021E532E049E652E0DBD920E007
:105A200030E048EC52E40E94D8946B017C0120E005
:105A300030E0A9010E947492181634F0C12CD12CC8
:105A400048EAE42E41E4F42EC0924D02D0924E0278
:105A5000E0924F02F09250020F91FF90EF90DF9092
:105A6000CF9008952F923F924F925F927F928F92A4
:105A70009F92AF92BF92CF92DF92EF92FF920F93DD
:105A80001F93CF93DF9300D01F92CDB7DEB76C0189
:105A900088EA94E09C838B83E6E9F4E0FA83E98367
:105AA00003E51BE0EE24E394F12C6DE3262E312C6C
:105AB0007EE3472E512CE0E1AE2EB12CF1E18F2E8A
:105AC000912CA7E17A2E80919404909195048E15E3
:105AD0009F050CF4ECC0F1E0CF16D10431F4F801CD
:105AE00080819181E981FA8109C0F2E0CF16D10469
:105AF00039F4E981FA8180819181F8019183808371
:105B0000E981FA8180819181009749F4EB81FC81E0
:105B1000808191819093B9048093B80428C081302A
:105B2000910549F4EB81FC81808191819093C704B8
:105B30008093C6041CC08230910549F4EB81FC813E
:105B4000808191819093C5048093C40410C0039711
:105B500071F4EB81FC81808191819093BB048093EF
:105B6000BA0469EC7AE089E99CE00E949E8EE981A2
:105B7000FA8181919191FA83E9838430910549F406
:105B8000EB81FC812081318130938202209381025C
:105B900030C08530910549F4EB81FC812081318151
:105BA0003093C3042093C20424C08630910549F485
:105BB000EB81FC81208131813093BF042093BE04AE
:105BC00024C08730910549F4EB81FC81208131812B
:105BD0003093BD042093BC0446C08A30910549F43B
:105BE000EB81FC81208131813093C1042093C0047A
:105BF0003AC08531910549F4EB81FC8120813181E6
:105C00003093C9042093C8042EC08631910549F40D
:105C1000EB81FC81208131813093E3042093E20405
:105C200022C087319105F9F4EB81FC81208131811B
:105C3000A901475051094230510540F4B092E704A0
:105C4000A092E6049092E5048092E4042550310984
:105C50002230310540F43092E7042092E60450925D
:105C6000E5044092E4049C012B5031092A303105AF
:105C700098F4EB81FC81208131813093BB04209327
:105C8000BA04789EB001799E700D11246D577D4F36
:105C900089E99CE00E949E8EFFEFEF1AFF0A8B813C
:105CA0009C8102969C838B830E5F1F4F0CCF0F90BD
:105CB0000F900F900F90DF91CF911F910F91FF9058
:105CC000EF90DF90CF90BF90AF909F908F907F909C
:105CD0005F904F903F902F90089581E08093F4045F
:105CE00085E49DE00C949A7885E49DE00E94947888
:105CF0001092F4040895CF93DF9300D000D0CDB775
:105D0000DEB78091F504811143C061E08091F60413
:105D10000E94B385E091450DF091460D0480F58118
:105D2000E02D20E042E060E185E49DE019954CEE35
:105D300054E060E085E49DE00E941A7981E0809360
:105D4000F5048093F4046FE472E0CE0101960E94A2
:105D50009F8F4AE050E060E070E0CE0101960E9423
:105D6000CC09CE0101960E94968D63E472E0CE01CB
:105D700001960E949F8F4AE050E060E070E0CE0103
:105D800001960E94400BCE0101960E94968D0DC097
:105D90008091F404882349F0A7DF60E08091F60445
:105DA0000E94B3851092F50401C097DF26960FB6C6
:105DB000F894DEBF0FBECDBFDF91CF9108954F9213
:105DC0005F926F927F92AF92BF92CF92DF92EF92EB
:105DD000FF920F931F93CF93DF93CDB7DEB7EA9770
:105DE0000FB6F894DEBF0FBECDBF182F69EC7AE076
:105DF000CE01C5960E94018E612FCE0145960E946C
:105E00002080BE016B5E7F4FCE0101960E945571CE
:105E1000CE0101960E94B472CE0101960E94487490
:105E20006CE0CE0101960E94A473CE0101960E94FF
:105E30005E71082F10E00330110509F46FC167E8A7
:105E400076E0CE01C5960E949E8E69EC7AE08BE3E7
:105E50009CE00E949E8EBE016B5C7F4FCE018396BC
:105E60000E94808E4AE050E060E070E0CE018396B0
:105E70000E94CC09CE0183960E94968D41E060E09D
:105E800085E49DE00E945E786BEA76E0CE01C596DF
:105E90000E949E8EB7E9AB2EBBE0BB2ECC24C394F0
:105EA000D12CE12CF12CE016F1060CF0EDC06E2D9A
:105EB000CE0101960E94D574F50121913191419155
:105EC00051915F010E94AE912B013C0120E030E036
:105ED0004CEF52EC0E94749287FF25C04AE0B60155
:105EE000CE0189960E94CC8E68EC77E0CE01839635
:105EF0000E94018EBE01675D7F4FCE0183960E9496
:105F0000FA8F61E976E00E940B90BC018BE39CE084
:105F10000E94D28FCE0183960E94968DCE018996E3
:105F20000E94968D49C022E0B301A201CE01839662
:105F30000E94238F4AE0B601CE018F960E94CC8E3C
:105F400068EC77E0CE0189960E94018EBE01615D0A
:105F50007F4FCE0189960E94FA8F60E778E00E9419
:105F60000B90BE016D5D7F4F0E94FA8FBC018FE2E6
:105F70009CE00E946B8ECE0189960E94968DCE0188
:105F80008F960E94968DCE0183960E94968D6FE229
:105F90007CE0CE0183960E94808E62E275E0CE01A5
:105FA00083960E940B90BC018BE39CE00E94D28FF1
:105FB000CE0183960E94968D0130110559F4E114AB
:105FC000F10409F05AC06BE37CE0CE01C5960E9453
:105FD0006B8E53C00230110511F522E0B301A2010E
:105FE000CE0189960E94238FBE01675D7F4FCE014F
:105FF00083960E94808E62E275E0CE0183960E94B5
:106000000B90BC01CE01C5960E94D28FCE01839623
:106010000E94968DCE0189960E94968D2EC06FE2C9
:106020007CE0CE0183960E94808E44E150E06FEFC9
:106030007FEFCE0183960E94400BCE0183960E9493
:10604000968D6DE875E0CE0183960E94018ECE019B
:1060500083960E94FD0BCE0183960E94968D8091BF
:10606000F504882351F08091F404882331F060ED29
:1060700077E080E090E00E946B84FFEFEF1AFF0A68
:106080008FEFC81AD80A0FCFCE01C5960E942B9168
:106090008BE39CE00E942B9101151105C9F460E38C
:1060A00072E08BE39CE00E947F8F6DE976E0CE0189
:1060B00083960E94018E4AE050E06FEF7FEFCE01A1
:1060C00083960E94400BCE0183960E94968DE2C07B
:1060D000043011050CF0F7C0BE016B5C7F4FCE01A0
:1060E00083960E94808E4AE050E06FEF7FEFCE01F2
:1060F00083960E94400BCE0183960E94968D6DE898
:1061000075E0CE0183960E94018ECE0183960E9497
:10611000FD0BCE0183960E94968DD5C068EA76E08D
:10612000CE01C5960E949E8EBE016B5C7F4FCE0154
:1061300083960E94808E4AE050E060E070E0CE01DD
:1061400083960E94CC09CE0183960E94968D69ECBD
:106150007AE08BE39CE00E949E8E6BE37CE0CE01B4
:10616000C5960E946B8E00E010E0602FCE01019674
:106170000E94D5746B017C0122E0AB01BC01CE0111
:106180000115110569F483960E94238FBE016D5D90
:106190007F4F85E49DE00E943E8ACE0183961BC01E
:1061A00089960E94238FBE01675D7F4FCE01839643
:1061B0000E94808E62E275E0CE0183960E940B9071
:1061C000BC01CE01C5960E94D28FCE0183960E945B
:1061D000968DCE0189960E94968D22E0B701A60188
:1061E000CE0189960E94238FBE01675D7F4FCE014D
:1061F00083960E94808E62E275E0CE0183960E94B3
:106200000B90BC018BE39CE00E94D28FCE01839661
:106210000E94968DCE0189960E94968D0F5F1F4F2A
:106220000330110509F0A1CFCE01C5960E942B9134
:10623000BE016B5C7F4FCE0183960E94808E4AE048
:1062400050E06FEF7FEFCE0183960E94400BCE01AE
:1062500083960E94968D0E94E90B8BE39CE00E943E
:106260002B916EEA76E0CE0183960E94018E6BE35D
:106270007CE0CE0183960E94FA8F68EB76E00E9464
:106280000B90BC018BE39CE00E946B8ECE01839649
:106290000E94968DCE01C5960E94968DEA960FB605
:1062A000F894DEBF0FBECDBFDF91CF911F910F914C
:1062B000FF90EF90DF90CF90BF90AF907F906F9066
:1062C0005F904F90089568EB76E08BE39CE00E942E
:1062D000D88FE0CF8F929F92AF92BF92CF92DF92F2
:1062E000EF92FF920F931F93CF93DF93CDB7DEB75B
:1062F000A2970FB6F894DEBF0FBECDBF5C016A0156
:106300007B01122F6CE172E08AEF9EE00E941B8AF3
:106310004AE050E0B5018AEF9EE00E94368B62E2CF
:1063200075E08AEF9EE00E944C8A22E030E0B701DF
:10633000A6018AEF9EE00E94708C612FCE014596E7
:106340000E942080BE016B5E7F4FCE0101960E94AD
:106350005571CE0101960E94B472CE0101960E9441
:1063600048746CE0CE0101960E94A473CE010196A0
:106370000E945E71082F10E00B30110514F00AE046
:1063800010E08BE5A816B10408F44FC047E9842E4D
:106390004BE0942EC12CD12C7601A12CB12CA0164F
:1063A000B106BCF46A2DCE0101960E94D5749B0102
:1063B000AC01F40161937193819391934F01C701F3
:1063C000B6010E94AE916B017C01FFEFAF1ABF0ACC
:1063D000E6CFB801882777FD8095982F0E944493D7
:1063E0009B01AC01C701B6010E9478926B017C0150
:1063F00037E9832E3BE0932EA12CB12CA016B106D9
:106400000CF052C0F4012081318142815381C701D7
:10641000B6010E94AD91F4016193719381939193C0
:106420004F01FFEFAF1ABF0AE9CFA114B10439F44D
:1064300027E9822E2BE0922EA12CB12C1DC00A152B
:106440001B050CF0850101501109602FCE0101964A
:106450000E94D5749B01AC01000F111F000F111F8A
:106460000956144FC701B6010E94AD91F80160832F
:1064700071838283938318C0A016B106ACF46A2D91
:10648000CE0101960E94D5749B01AC01C701B601F3
:106490000E94AD91F40161937193819391934F01A7
:1064A000FFEFAF1ABF0AE8CFA2960FB6F894DEBF8F
:1064B0000FBECDBFDF91CF911F910F91FF90EF9055
:1064C000DF90CF90BF90AF909F908F900895CF9323
:1064D000DF93C6EED4E060E088810E94B38582E05D
:1064E00090E00E94918461E088810E94B3858AE0F7
:1064F00090E00E94918460E088810E94B38520E44E
:1065000032E44FE050E061E08091E4040E941086A4
:106510000E94429320E030E048EC52E40E947892DE
:1065200020912D0D30912E0D40912F0D5091300D59
:106530000E94D89420E030E44CE156E40E94789226
:1065400020E030E040E05FE30E94D894DF91CF91FB
:106550000895CF92DF92EF92FF92B9DF6B017C0139
:1065600020E030E040E050E40E94199418161CF43A
:10657000AEDF6B017C0120E030E040E050E4C70179
:10658000B6010E94199418161CF4A1DF6B017C015E
:1065900020E030E040E050E4C701B6010E941994C9
:1065A00018161CF494DF6B017C0120E030E040E021
:1065B00050E4C701B6010E94199418162CF4FF90FC
:1065C000EF90DF90CF9083CFC701B601FF90EF909F
:1065D000DF90CF9008954F925F926F927F928F924B
:1065E0009F92AF92BF92CF92DF92EF92FF92CF93A2
:1065F000DF9300D01F92CDB7DEB7ABDF9B01AC01BC
:1066000069833A834B835C830E9448842B013C015D
:106610006EE170E080E090E00E946B849ADF6B0195
:106620007C010E9448844B015C0184189508A608EF
:10663000B70829813A814B815C8181ED881687E01A
:106640009806A104B1040CF43DC0C701B6010E9434
:10665000AD916B017C0120E030E0A9010E9419940A
:1066600018165CF426EA3BE944EC5BE3C701B6018B
:106670000E94749287FF0BC025C026EA3BE944ECD8
:106680005BEBC701B6010E9419941816DCF0C50136
:10669000B40128EE33E040E050E00E943D96CA018C
:1066A000B9010E9444934B015C0120E030E04AE7CD
:1066B00054E4C701B6010E94D894A50194010E9438
:1066C000789203C060E070E0CB010F900F900F90C4
:1066D0000F90DF91CF91FF90EF90DF90CF90BF9020
:1066E000AF909F908F907F906F905F904F900895A4
:1066F00023E333E948E853E40E94789220E030E055
:1067000040E85FE30E94AE910E948B9526E636EA50
:1067100045EA53E40E94D89460932D0D70932E0D9A
:1067200080932F0D9093300D08954F925F926F924A
:106730007F928F929F92AF92BF92CF92DF92EF9211
:10674000FF92CF93DF93CDB7DEB76C970FB6F89477
:10675000DEBF0FBECDBF6B017C010E943C846D8B00
:106760007E8B8F8B988F61E08091E6040E947A8502
:1067700060E08091E4040E947A8587E59CE00E94B5
:10678000AE7B6093290D70932A0D80932B0D90930F
:106790002C0DAEDFDEDE6D877E878F87988B0E94A3
:1067A0004884698B7A8B8B8B9C8B6AE070E080E0ED
:1067B00090E00E946B846EEF71E08BE39CE00E949E
:1067C0007F8F20E030E04AE754E4C701B6010E9421
:1067D000D894698F7A8F8B8F9C8F412C512C3201EA
:1067E000C12CD12C7601C701B6010E944493298D9A
:1067F0003A8D4B8D5C8D0E94749287FF87C10E94F9
:106800003C842D893E894F89588D621B730B840B04
:10681000950B0E94429320E030E04AE754E40E9446
:106820007892AB01BC0123E0CE0101960E94238F38
:10683000BE016F5F7F4F85E39CE00E94888ECE0192
:1068400001960E94968D85DE6B017C010E94488432
:106850004B015C0189899A89AB89BC89881A990A9C
:10686000AA0ABB0A91ED891697E09906A104B10422
:106870000CF441C020E030E0A901C701B6010E943C
:10688000199418165CF426EA3BE944EC5BE3C70173
:10689000B6010E94749287FF0BC02DC026EA3BE927
:1068A00044EC5BEBC701B6010E94199418161CF169
:1068B000C501B40128EE33E040E050E00E943D966F
:1068C000CA01B9010E9444934B015C012D853E85AC
:1068D0004F855889C701B6010E94AD9120E030E094
:1068E0004AE754E40E94D894A50194010E9478924A
:1068F0004B015C0103C0812C912C540165E37CE0C9
:10690000CE0101960E94808E64ED76E0CE01019664
:106910000E940B90BC0185E39CE00E946B8ECE012F
:1069200001960E94968D23E0B701A601CE0107963D
:106930000E94238FBE01695F7F4FCE0101960E94A6
:10694000808E6BEC76E0CE0101960E940B90BC012C
:106950008FE29CE00E946B8ECE0101960E94968D84
:10696000CE0107960E94968D22E0B501A401CE01CA
:1069700001960E94238F65E575E0CE0107960E947F
:10698000018E65E37CE0CE0107960E94FA8F6EECE3
:1069900076E00E940B906FE27CE00E94FA8F6EED31
:1069A00076E00E940B90BE016F5F7F4F0E94FA8FCE
:1069B00062ED76E00E940B90BC018BE39CE00E94AC
:1069C000D28FCE0107960E94968DCE0101960E942D
:1069D000968D20E030E0A901C501B4010E94199410
:1069E00087FD06C062E275E08FE29CE00E94D88FCE
:1069F00022E0B501A401CE0107960E94238FBE01BB
:106A0000695F7F4FCE0101960E94808E62ED76E035
:106A1000CE0101960E940B90BC018FE29CE00E9487
:106A2000D28FCE0101960E94968DCE0107960E94CC
:106A3000968D6BE37CE0CE0101960E94808ECE01A4
:106A400001960E94A20FCE0101960E94968DC3016D
:106A5000B20125E030E040E050E00E943D96672B17
:106A6000682B692B21F566ED76E0CE0101960E9438
:106A7000018E45E050E060E070E0CE0101960E949A
:106A8000CC09CE0101960E94968D6FE27CE0CE018A
:106A900001960E94808E45E050E06FEF7FEFCE01BF
:106AA00001960E94400BCE0101960E94968D69ECE2
:106AB0007AE08BE39CE00E949E8E65E070E080E0CF
:106AC00090E00E946B840E943C846B017C012D89C4
:106AD0003E894F89588DC21AD30AE40AF50A39DD76
:106AE0006D877E878F87988B0E944884698B7A8B0D
:106AF0008B8B9C8B6AE070E080E090E00E946B845E
:106B00003FEF431A530A630A730A6DCE60E0809127
:106B1000E6040E947A856C960FB6F894DEBF0FBE2D
:106B2000CDBFDF91CF91FF90EF90DF90CF90BF90DE
:106B3000AF909F908F907F906F905F904F9008954F
:106B40000F931F93CF93DF93CDB7DEB72C970FB67C
:106B5000F894DEBF0FBECDBF06EE14E061E0F80191
:106B600080810E947A8560E08091E4040E947A85A9
:106B700087E59CE00E94AE7B6093290D70932A0DFF
:106B800080932B0D90932C0DB3DDE3DCAB01BC01A6
:106B900023E0CE0107960E94238FBE01695F7F4FDD
:106BA000CE0101960E94808E63E476E0CE010196CC
:106BB0000E940B90BC0185E39CE00E946B8ECE018D
:106BC00001960E94968DCE0107960E94968D6FECDD
:106BD00076E0CE0101960E94018E65E37CE0CE0155
:106BE00001960E94FA8FBC018BE39CE00E946B8EA1
:106BF000CE0101960E94968DEEDCAB01BC0122E035
:106C0000CE0107960E94238FBE01695F7F4FCE01A0
:106C100001960E94808E62ED76E0CE0101960E9480
:106C20000B90BC018FE29CE00E946B8ECE0101961E
:106C30000E94968DCE0107960E94968D6DED76E0AE
:106C4000CE0101960E94018E6FE27CE0CE0101969A
:106C50000E94FA8FBC018BE39CE00E94D28FCE0190
:106C600001960E94968D62E275E0CE0101960E9427
:106C7000018E6FE27CE0CE0101960E94FA8FBC018A
:106C800085E39CE00E94D28FCE0101960E94968DF2
:106C900066ED76E0CE0101960E94018E4AE050E05A
:106CA00060E070E0CE0101960E94CC09CE01019611
:106CB0000E94968D65E37CE0CE0101960E94808E55
:106CC00045E050E06FEF7FEFCE0101960E94400B50
:106CD000CE0101960E94968D61EE76E08BE39CE0FA
:106CE0000E94D88F60E0F80180810E947A852C96FE
:106CF0000FB6F894DEBF0FBECDBFDF91CF911F91CD
:106D00000F9108958F929F92AF92BF92CF92DF9290
:106D1000EF92FF920F9352E0C52E63E0E62E04E05F
:106D200025E04BE06CE085E49DE00E94007A64EF92
:106D300076E087E39DE00E94018E6AEF76E081E3D2
:106D40009DE00E94018E20E141E168E186E29DE044
:106D50000E940A7E74E0E72E2AEC34E04EEC54E008
:106D600062ED74E087EB9CE00E94FD8083EA9CE08A
:106D70000E94546069EC7AE089E99CE00E94018EEF
:106D80008091BE049091BF049093980C8093970CCF
:106D90008090450290904602A0904702B090480231
:106DA00020914102309142024091430250914402AD
:106DB000C501B4010E94AD916B017C016093930CFD
:106DC0007093940C8093950C9093960C609149026B
:106DD00070914A0280914B0290914C026093870C13
:106DE0007093880C8093890C90938A0C80928B0C02
:106DF00090928C0CA0928D0CB0928E0C20913D0242
:106E000030913E0240913F02509140020E94AD916C
:106E10009B01AC01C701B6010E94789260938F0C70
:106E20007093900C8093910C9093920C4FEF5FEFC6
:106E3000BA018EE69CE00E94635E87E59CE00E94BA
:106E4000A37A69EC7AE08DE49CE00E94018E69EC03
:106E50007AE087E49CE00E94018E69EC7AE081E4AC
:106E60009CE00E94018E69EC7AE08BE39CE00E943A
:106E7000018E69EC7AE085E39CE00E94018E69EC6A
:106E80007AE08FE29CE00E94018E60913202709164
:106E9000330288E19BE00F91FF90EF90DF90CF905D
:106EA000BF90AF909F908F900C948D668FE29CE086
:106EB0000E94968D85E39CE00E94968D8BE39CE07A
:106EC0000E94968D81E49CE00E94968D87E49CE070
:106ED0000E94968D8DE49CE00E94968D8DE49AE050
:106EE00090936F0C80936E0C89E99CE00E94968DC4
:106EF00081E39DE00E94968D87E39DE00C94968D42
:106F00006F927F928F929F92AF92BF92CF92DF92B9
:106F1000EF92FF920F931F93CF93DF93CDB7DEB71E
:106F2000E8970FB6F894DEBF0FBECDBF4B015C01F2
:106F300087E99FE00E94AB8764E670E080E090E024
:106F40000E946B8440E855E260E070E087E99FE0D2
:106F50000E94550964E670E080E090E00E946B8436
:106F60006FE772E085E39CE00E947F8F65E37CE041
:106F7000CE0101960E94808E42E350E06FEF7FEFDA
:106F8000CE0101960E94CC09CE0101960E94968DF9
:106F900064E772E085E39CE00E947F8F65E37CE01C
:106FA000CE0101960E94808E42E350E06FEF7FEFAA
:106FB000CE0101960E94400BCE0101960E94968D53
:106FC00080915C0D90915D0D8D7F712CC12CD12C29
:106FD000E12CF12C00E010E0019709F459C0B2E473
:106FE0006B2E0E943C84681979098A099B09683BC9
:106FF0007B408105910508F04BC087E99FE00E9426
:107000003C86892BF1F14CED55E060E070E087E9BA
:107010009FE00E94AE8C68AE41E050E0BE01685C2B
:107020007F4F87E99FE00E94958D882351F14FE1C2
:1070300050E0BE016F5F7F4F87E99FE00E94B48CF4
:1070400089818D34F1F46FE1CE0101960E94F12720
:107050008823B9F00C8110E0102F00278D81080FD4
:10706000111DEE80F12CFE2CEE248F81E80EF11C18
:10707000C884D12CDC2CCC248985C80ED11C772463
:10708000739462E370E080E090E00E946B84A9CF8B
:107090000E943C84681979098A099B09683B7B40F6
:1070A0008105910510F47110C3C00E941B0C65E3AB
:1070B0007CE0CE0180960E94808E42E350E066E044
:1070C00070E0CE0180960E94CC09CE0180960E948D
:1070D000968D772009F4D1C082E090E090935D0D09
:1070E00080935C0D4AE0B601CE0180960E94CC8E62
:1070F0004AE0B701CE0186960E94CC8E4AE0B801E4
:10710000CE01C2960E94CC8EBE016E5C7F4FCE0136
:107110008C960E94808E64E879E0CE018C960E9465
:107120000B90BE016A5D7F4F0E94FA8F64E879E0A0
:107130000E940B90BE01605E7F4F0E94FA8FBC01DF
:107140008BE39CE00E946B8ECE018C960E94968D04
:10715000CE01C2960E94968DCE0186960E94968D93
:10716000CE0180960E94968D6BE37CE0CE018096E6
:107170000E94808E4AE050E06FEF7FEFCE01809654
:107180000E94400BCE0180960E94968D62E077E0CF
:1071900085E49DE00E944C8A68E077E08BE39CE008
:1071A0000E949E8E4AE0B601CE0180960E94CC8E4F
:1071B0004AE0B701CE0186960E94CC8E4AE0B80123
:1071C000CE01C2960E94CC8EBE016E5C7F4FCE0176
:1071D0008C960E94808E62E275E0CE018C960E94B1
:1071E0000B90BE016A5D7F4F0E94FA8F62E275E0EC
:1071F0000E940B90BE01605E7F4F0E94FA8F62E09A
:1072000077E00E940B90BC018BE39CE00E94D28F40
:10721000CE018C960E94968DCE01C2960E94968DCC
:10722000CE0186960E94968DCE0180960E94968D04
:1072300062E370E080E090E00E946B8487E99FE069
:107240000E94AB8762E370E080E090E00E946B8474
:10725000E8960FB6F894DEBF0FBECDBFDF91CF9199
:107260001F910F91FF90EF90DF90CF90BF90AF9064
:107270009F908F907F906F90089569E672E08BE306
:107280009CE00E947F8F6BE37CE0CE0180960E94A1
:10729000808E4AE050E060E070E0CE0180960E946F
:1072A000400BCE0180960E94968D66E572E08BE3DE
:1072B0009CE00E947F8F80915C0D90915D0D029704
:1072C00009F0B6CF10925D0D10925C0DB1CF7F9298
:1072D0008F929F92AF92BF92CF92DF92EF92FF92E6
:1072E0000F931F93CF93DF9300D000D0CDB7DEB7BD
:1072F0004C0187E99FE00E94AB8740E052EC61E0DF
:1073000070E087E99FE00E9455094CED55E060E090
:1073100070E087E99FE00E94AE8C64E670E080E058
:1073200090E00E946B84A12CB12C712CA814B9049C
:107330000CF051C065E070E080E090E00E946B844A
:1073400000E010E0C12CD12C760171100FC087E94C
:107350009FE00E943C86892B31F485E1C816D10458
:10736000E104F1041CF40330110554F08FEFA81A66
:10737000B80A64E670E080E090E00E946B84D6CFAB
:1073800087E99FE00E943C86892B69F087E99FE0AE
:107390000E945586E1E0F0E0EC0FFD1FE00FF11FC9
:1073A00080830F5F1F4F65E070E080E090E00E94F7
:1073B0006B84023011054CF089818B3B31F47724CA
:1073C00073948A818A3A09F0712C8FEFC81AD80A0F
:1073D000E80AF80ABACF872D26960FB6F894DEBFD2
:1073E0000FBECDBFDF91CF911F910F91FF90EF9016
:1073F000DF90CF90BF90AF909F908F907F90089537
:107400008F929F92AF92BF92CF92DF92EF92FF92B4
:107410000F931F93CF93DF93CDB7DEB72C970FB6A3
:10742000F894DEBF0FBECDBF61E08091F6040E94EC
:107430007A8561E08091F6040E94B385E091450D64
:10744000F091460D0480F581E02D20E042E060E1FE
:1074500085E49DE019954CEE54E060E085E49DE004
:107460000E941A790E946D2E8EED93E09093C00BCE
:107470008093BF0B0E94EB9980935E0D8FED93E09C
:107480000E94EB9980935F0D80915E0D90915F0D4E
:107490001816190654F41092F804019731F410925A
:1074A0005F0D10925E0D0E94A80968E177E085E407
:1074B0009DE00E944C8A40E855E260E070E08AEF6F
:1074C0009EE00E94550940E855E260E070E084E3E8
:1074D00090E10E94550964E670E080E090E00E942F
:1074E0006B848091F804882331F068EE73E080E0CB
:1074F00090E00E946B848AEF9EE00E945586182FD0
:10750000823709F42DC11092C00B1092BF0B49E1D4
:10751000C42E4BE0D42EE12CF12CC7010E94EB9934
:10752000D6018D936D01BFEFEB1AFB0AE6E7EE166D
:10753000F10499F78091190B90911A0BA0911B0BF4
:10754000B0911C0B85369105A105B1050CF408C15D
:107550008093380290933902A0933A02B0933B0291
:1075600080911D0B90911E0BA0911F0BB091200BD1
:107570008093340290933502A0933602B093370281
:107580008091210B9091220BA091230BB091240BA1
:1075900080932E0290932F02A0933002B093310279
:1075A00065E37BE0CE0101960E94018EBE016F5F14
:1075B0007F4F87E39DE00E94888ECE0101960E9456
:1075C000968D8091250B9091260BA091270BB09161
:1075D000280B8093220290932302A0932402B0935D
:1075E00025028091290B90912A0BA0912B0BB09131
:1075F0002C0B80931E0290931F02A0932002B09345
:10760000210280912D0B90912E0BA0912F0BB09108
:10761000300B80931A0290931B02A0931C02B0932C
:107620001D028091310B9091320BA091330BB091E0
:10763000340B8093160290931702A0931802B09314
:10764000190280913D0B90913E0BA0913F0BB091A0
:10765000400B8093450290934602A0934702B0935B
:1076600048028091410B9091420BA091430BB09145
:10767000440B8093410290934202A0934302B09343
:1076800044028091450B9091460BA091470BB0911D
:10769000480B8093490290934A02A0934B02B09307
:1076A0004C028091490B90914A0BA0914B0BB091E9
:1076B0004C0B80933D0290933E02A0933F02B09307
:1076C000400280914D0B90914E0BA0914F0BB091C9
:1076D000500B80934D0290934E02A0934F02B093B3
:1076E0005002C090630BD090640BE090650BF0905B
:1076F000660BA7019601C701B6010E94CC958111C6
:1077000008C0C0921202D0921302E0921402F092CA
:10771000150227E6A22E2BE0B22E37E9832E3BE09E
:10772000932ED501CD90DD90ED90FD905D01A701E8
:107730009601C701B6010E94CC95811105C0F401E4
:10774000C082D182E282F382F4E08F0E911C8FE836
:10775000A8168BE0B80629F781E090E00E94322D50
:107760000EE8010F023070F08091190B90911A0B06
:10777000A0911B0BB0911C0B85369105A105B1059D
:107780000CF032C18091380290913902A0913A02F6
:10779000B0913B028093190B90931A0BA0931B0B93
:1077A000B0931C0B8091340290913502A091360267
:1077B000B091370280931D0B90931E0BA0931F0B6B
:1077C000B093200B80912E0290912F02A091300255
:1077D000B09131028093210B9093220BA093230B45
:1077E000B093240B123751F420E030E048E050E031
:1077F00065E37BE087E39DE00E9467908091220231
:1078000090912302A0912402B09125028093250B30
:107810009093260BA093270BB093280B80911E0208
:1078200090911F02A0912002B09121028093290B18
:1078300090932A0BA0932B0BB0932C0B80911A02E0
:1078400090911B02A0911C02B0911D0280932D0B00
:1078500090932E0BA0932F0BB093300B80911602B8
:1078600090911702A0911802B09119028093310BE8
:107870009093320BA093330BB093340B809145025D
:1078800090914602A0914702B091480280933D0B2F
:1078900090933E0BA0933F0BB093400B809141021D
:1078A00090914202A0914302B09144028093410B17
:1078B0009093420BA093430BB093440B80914902E9
:1078C00090914A02A0914B02B0914C028093450BDB
:1078D0009093460BA093470BB093480B80913D02C9
:1078E00090913E02A0913F02B09140028093490BDB
:1078F00090934A0BA0934B0BB0934C0B80914D028D
:1079000090914E02A0914F02B091500280934D0B86
:1079100090934E0BA0934F0BB093500B809112029B
:1079200090911302A0911402B09115028093630B01
:107930009093640BA093650BB093660BE7E9FBE0B3
:1079400027E63BE04191519161917191D9014D93AD
:107950005D936D937D939D01BBE0EF3BFB0791F73A
:1079600062E47CE08AEF9EE00E94578A81E5A82EBF
:107970008BE0B82E94E9C92E94E0D92EE12CF12C9D
:1079800080919404909195048E159F051CF14601F9
:10799000F601819191916F01D5018D939D935D01C8
:1079A0004AE050E0B7018AEF9EE00E94368B69E220
:1079B00077E08AEF9EE00E944C8AF4016081718139
:1079C0004AE050E08AEF9EE00E943D8BFFEFEF1A05
:1079D000FF0AD6CF023040F41092C00B1092BF0BBA
:1079E00080E090E00E947F0964E670E080E090E033
:1079F0000E946B8488E19BE00E9492666EE277E0D1
:107A0000CE0101960E94018E4AE050E06FEF7FEFB9
:107A1000CE0101960E94CC09CE0101960E94968D5E
:107A200062E075E0CE0107960E94018E67E37DE07B
:107A3000CE0107960E94FA8FBC01CE0101960E94EA
:107A4000808E4AE050E06FEF7FEFCE0101960E94FA
:107A5000400BCE0101960E94968DCE0107960E94A2
:107A6000968D6CE277E0CE0107960E94018E67E367
:107A70007DE0CE0107960E94FA8F6EE377E00E94C8
:107A80000B90BC01CE0101960E94808ECE01019622
:107A90000E94A20FCE0101960E94968DCE010796FC
:107AA0000E94968D64E670E080E090E00E946B8416
:107AB00081E39EE00E94937564E670E080E090E0D0
:107AC0000E946B8463E270E081E39EE00E94A675F1
:107AD00061E070E081E39EE00E94580981E39EE04E
:107AE0000E941A7683E090E090935D0D80935C0D88
:107AF00060E070E086E29DE00E94F47E6B017C0114
:107B000062E370E080E090E00E946B84A701960140
:107B1000C701B6010E94CC95882309F465C060E0D6
:107B200070E086E29DE00E94F27E6B017C0162E3E0
:107B300070E080E090E00E946B84A7019601C7018D
:107B4000B6010E94CC95882309F44EC081E090E0F4
:107B500090935D0D80935C0D40E052EC61E070E02D
:107B600087E99FE00E94550964E670E080E090E0BC
:107B70000E946B8482E090E0AADB882339F069E2FE
:107B80007CE08AEF9EE00E94578A2EC010925D0D25
:107B900010925C0D87E99FE00E94AB8764E670E07D
:107BA00080E090E00E946B8440E855E260E070E085
:107BB00087E99FE00E94550987E99FE00E943C8683
:107BC000892B91F06FE07CE08AEF9EE00E94578A5B
:107BD00082E090E090935D0D80935C0D64E670E030
:107BE00080E090E00E946B8480915C0D90915D0D2F
:107BF000039731F46AEF7BE08AEF9EE00E94578A98
:107C000063E087E59CE00E94507B811111C064ED28
:107C10007BE0CE0101960E949F8FCE0101960E94CB
:107C2000A20FCE0101960E94968D10923C0293C045
:107C300060EC7BE08BE39CE00E947F8F40E050E0B3
:107C4000BA0187E59CE00E94707D0E94449320E089
:107C500030E048EC52E40E947892AB01BC0122E093
:107C6000CE0107960E94238FBE01695F7F4FCE0130
:107C700001960E94808E6BEE78E0CE0101960E9404
:107C80000B90BC018BE39CE00E94D28FCE01019649
:107C90000E94968DCE0107960E94968D6BE37CE044
:107CA0008AEF9EE00E94678A69EA7BE08BE39CE0B2
:107CB0000E947F8F609138027091390280913A0260
:107CC00090913B020E94449320E030E048EC52E463
:107CD0000E947892AB01BC0122E0CE0107960E947F
:107CE000238FBE01695F7F4FCE0101960E94808E77
:107CF0006BEE78E0CE0101960E940B90BC018BE305
:107D00009CE00E94D28FCE0101960E94968DCE01FA
:107D100007960E94968D6BE37CE08AEF9EE00E94BE
:107D2000678A113629F481E00E94681981E011C048
:107D30008AEF9EE00E945586182F64E670E080E08E
:107D400090E00E946B84113671F380E00E94681904
:107D500080E00E94B80F64E670E080E090E00E944E
:107D60006B848091F804882331F068EE73E080E042
:107D700090E00E946B846AEA77E087E49CE00E94CE
:107D80009E8E82E090E090932A0C8093290C809143
:107D9000F80481110E94BA172C960FB6F894DEBF32
:107DA0000FBECDBFDF91CF911F910F91FF90EF904C
:107DB000DF90CF90BF90AF909F908F9008952F92BB
:107DC0003F924F925F926F927F928F929F92AF926B
:107DD000BF92CF92DF92EF92FF920F931F93CF93B8
:107DE000DF93CDB7DEB72B970FB6F894DEBF0FBE8B
:107DF000CDBF1C018BEB8F838AEA888781E089875E
:107E000084E6829D9001839D300D11243B872A8753
:107E1000E12CF12CC12CD12C812C912C5401C214B9
:107E2000D30494F1C501B4010E94449320E030E0F2
:107E300040E251E40E9478926B017C01B1018827F5
:107E400077FD8095982F0E9444939B01AC01C70158
:107E5000B6010E9478922B960FB6F894DEBF0FBE43
:107E6000CDBFDF91CF911F910F91FF90EF90DF90E9
:107E7000CF90BF90AF909F908F907F906F905F90CA
:107E80004F903F902F9008952A853B85E216F30688
:107E90004CF6C7016AE070E00E940896892B79F4DD
:107EA000E091970FF091980F0280F381E02D43E06D
:107EB00050E0BE01695F7F4F87E99FE0199565E05B
:107EC00070E080E090E00E946B843FEFE31AF30AD9
:107ED00000E010E0412C512C320187E99FE00E9424
:107EE0003C86892B39F424E0421651046104710464
:107EF0000CF095CF063011050CF091CF87E99FE08B
:107F00000E943C86892B69F087E99FE00E94558694
:107F1000E1E0F0E0EC0FFD1FE00FF11F80830F5F49
:107F20001F4F65E070E080E090E00E946B840630B7
:107F3000110501F599818F8198131CC09A8188855C
:107F4000981318C09B818985981314C02C818D814A
:107F500090E0A0E0B0E0BA2FA92F982F8827820FD9
:107F6000911DA11DB11D880E991EAA1EBB1E8FEF6B
:107F7000C81AD80A9FEF491A590A690A790AADCF77
:107F8000CF92DF92EF92FF92CF93DF93CDB7DEB720
:107F90002C970FB6F894DEBF0FBECDBF87E99FE0E8
:107FA0000E94AB8740E052EC61E070E087E99FE01F
:107FB0000E9455094CED55E060E070E087E99FE0D4
:107FC0000E94AE8C64E670E080E090E00E946B84DA
:107FD00060E677E08BE39CE00E949E8E6BE37CE0A2
:107FE0008AEF9EE00E94678A62E370E080E090E0A2
:107FF0000E946B846BE37CE0CE0101960E94808E30
:1080000042E350E06FEF7FEFCE0101960E94CC0972
:10801000CE0101960E94968D6CE677E085E39CE0A8
:108020000E949E8E65E37CE0CE0101960E94808EC8
:1080300044E150E06FEF7FEFCE0101960E94400BCC
:10804000CE0101960E94968D80915C0D90915D0D00
:10805000019731F484E090E0B2DE6B017C0103C053
:10806000C12CD12C760180915C0D90915D0D892BF6
:1080700029F481E090E0A3DE6B017C0120E030E098
:1080800040EA51E4C701B6010E941994181664F53C
:1080900021E0B701A601CE0107960E94238F6BE273
:1080A00076E0CE0101960E94018EBE01695F7F4F8E
:1080B000CE0101960E94FA8F68E276E00E940B9052
:1080C000BC018BE39CE00E946B8ECE0101960E9466
:1080D000968DCE0107960E94968D81E090E0909358
:1080E0005D0D80935C0D10C068E777E08BE39CE04A
:1080F0000E949E8E80915C0D90915D0D019721F400
:1081000010925D0D10925C0D6BE37CE0CE01019648
:108110000E94808E4AE050E060E070E0CE0101965F
:108120000E94CC09CE0101960E94968D6BE37CE003
:10813000CE0101960E94808E62E275E0CE0101962A
:108140000E940B9065E37CE00E94FA8FBC018BE3F8
:108150009CE00E946B8ECE0101960E94968D87E96D
:108160009FE00E94AB8780912C0C882331F060E265
:1081700073E080E090E00E946B842C960FB6F89438
:10818000DEBF0FBECDBFDF91CF91FF90EF90DF90AC
:10819000CF9008952F923F924F925F926F927F926D
:1081A0008F929F92AF92BF92CF92DF92EF92FF9207
:1081B0000F931F93CF93DF93CDB7DEB766970FB6BC
:1081C000F894DEBF0FBECDBF6C0187E99FE00E942F
:1081D000AB8740E855E260E070E087E99FE00E94ED
:1081E000550964E670E080E090E00E946B844CEDFD
:1081F00055E060E070E087E99FE00E94AE8C64E6A5
:1082000070E080E090E00E946B848FEF898381E0D2
:108210008A8386E88B831C821D821E821F821886B9
:1082200089E78987C601880F991F9E8B8D8B212C2A
:10823000312CE12CF12C812C912C5401EC14FD04F7
:108240004CF087E99FE00E94AB87E114F104B9F19B
:10825000670135C08D899E892816390694F787E90C
:108260009FE00E94CD8708977CF0E091970FF091F6
:10827000980F0280F381E02D49E050E0BE016F5F6E
:108280007F4F87E99FE0199565E070E080E090E01E
:108290000E946B8400E010E0412C512C320187E9F0
:1082A0009FE00E943C86892B31F4E4E04E16510495
:1082B0006104710484F5023011056CF530C0C5010C
:1082C000B4010E9444934B015C01B601882777FDFD
:1082D0008095982F0E9444939B01AC01C501B40185
:1082E0000E94789266960FB6F894DEBF0FBECDBF9F
:1082F000DF91CF911F910F91FF90EF90DF90CF9082
:10830000BF90AF909F908F907F906F905F904F90B5
:108310003F902F900895FFEF2F1A3F0A8FCF87E9E4
:108320009FE00E943C86892B69F087E99FE00E94CC
:108330005586EAE0F0E0EC0FFD1FE00FF11F8083AF
:108340000F5F1F4F65E070E080E090E00E946B845B
:108350000230110569F59A858981981329C09B859A
:108360008B81981325C0FE013C96FC8BEB8B87E933
:108370009FE00E943C86892B31F4F4E04F165104B3
:1083800061047104DCF409301105E1F42D858C855C
:1083900090E0982F8827820F911DAA2797FDA0951E
:1083A000BA2F880E991EAA1EBB1E8FEFE81AF80A74
:1083B0009FEF491A590A690A790A71CF04301105E9
:1083C000A4F3E4CF87E99FE00E945586EB89FC89FE
:1083D0008193FC8BEB8B0F5F1F4FC9CFFF920F93E5
:1083E0001F93CF93DF93CDB7DEB72C970FB6F894DA
:1083F000DEBF0FBECDBF10922D0C69EC7AE08DE48C
:108400009CE00E949E8E11E08AEF9EE00E943C86D6
:1084100020912D0C1816190684F521112EC08AEF13
:108420009EE00E94558680932E0C8A3041F08D305C
:1084300031F0682F8DE49CE00E94E78F17C0109305
:108440002D0C64E877E0CE0101960E94018E6DE468
:108450007CE0CE0101960E94FA8FBC018AEF9EE07B
:108460000E94678ACE0101960E94968D6AE070E0B4
:1084700080E090E00E946B84C7CF222361F02091BE
:108480002D0C8091510C9091520C21116CC00097D1
:1084900009F069C0B0C000E010E0FF24F39484E369
:1084A00090E10E943C8618161906A4F584E390E139
:1084B0000E94558680932E0C8A3071F08D3061F0C9
:1084C00090912D0C911108C0682F8DE49CE00E94C2
:1084D000E78F0F5F1F4F17C08091510C9091520C86
:1084E000892B89F0F0922D0C84E390E10E943C8668
:1084F0001816190644F469EC7AE08DE49CE00E94B9
:108500009E8E10922D0C6FE070E080E090E00E9453
:108510006B84C5CF62E370E080E090E00E946B84E2
:10852000012B09F4ACCF6DE877E0CE0101960E94F3
:10853000018E6DE47CE0CE0101960E94FA8FBC01B1
:108540008AEF9EE00E94678ACE0101960E94968D76
:1085500084E390E10E94C48664E670E080E090E0ED
:108560000E946B848CCF019709F069C064ED76E0BE
:10857000CE0107960E94018EBE01695F7F4F8DE498
:108580009CE00E944790811115C062E977E0CE011E
:1085900001960E94018EBE016F5F7F4F8DE49CE0CB
:1085A0000E94479011E0811110E0CE0101960E94D7
:1085B000968D01C010E0CE0107960E94968D112382
:1085C00099F040E050E06DE47CE0CE0101960E941D
:1085D0004909BE016F5F7F4F87E49CE00E94888E4F
:1085E000CE0101960E94968D64E170E080E090E0FB
:1085F0000E946B8424C064E670E080E090E00E94FA
:108600006B840E943C84CB0168EE73E00E94089664
:10861000CB0164E670E00E940896823691057CF0FA
:1086200080912C0C81110BC087E49CE00E94879103
:10863000613071058105910511F40E94BA172C96DD
:108640000FB6F894DEBF0FBECDBFDF91CF911F9163
:108650000F91FF900895BF92CF92DF92EF92FF9219
:108660000F931F93CF93DF93CDB7DEB72B970FB642
:10867000F894DEBF0FBECDBF6C0187E99FE00E947A
:10868000AB8740E855E260E070E087E99FE00E9438
:10869000550964E670E080E090E00E946B844CED48
:1086A00055E060E070E087E99FE00E94AE8C64E6F0
:1086B00070E080E090E00E946B848FEF898381E01E
:1086C0008A8386E88B831C821D821E821F82188605
:1086D00089E7898787E99FE00E94C48662E370E0AA
:1086E00080E090E00E946B8487E99FE00E94CD8744
:1086F00008977CF0E091970FF091980F0280F3813A
:10870000E02D49E050E0BE016F5F7F4F87E99FE0B9
:10871000199562E370E080E090E00E946B84E12CA8
:10872000F12CB12CEC14FD040CF05BC087E99FE048
:108730000E943C86892B21F187E99FE00E94CD872A
:1087400008977CF0E091970FF091980F0280F381E9
:10875000E02D49E050E0BE016F5F7F4F87E99FE069
:10876000199565E070E080E090E00E946B8400E085
:1087700010E087E99FE00E943C860230110554F02A
:1087800062E370E080E090E00E946B848FEFE81A73
:10879000F80AC8CF87E99FE00E943C86892B69F0E0
:1087A00087E99FE00E945586EAE0F0E0EC0FFD1FAC
:1087B000E00FF11F80830F5F1F4F65E070E080E0E6
:1087C00090E00E946B840230110599F69A858981A8
:1087D0009813CFCF9B858B819813CBCFBB24B394B9
:1087E000C8CF87E99FE00E94AB878B2D2B960FB6F1
:1087F000F894DEBF0FBECDBFDF91CF911F910F91D7
:10880000FF90EF90DF90CF90BF900895CF92DF92CE
:10881000EF92FF92CF93DF93CDB7DEB72C970FB6D1
:10882000F894DEBF0FBECDBF0E941B0C6FEB72E051
:108830008BE39CE00E947F8F6BE37CE0CE0101968E
:108840000E94808E4AE050E060E070E0CE01019628
:108850000E94CC09CE0101960E94968D66EB72E0D3
:1088600085E39CE00E947F8F65E37CE0CE0101966A
:108870000E94808E44E150E06FEF7FEFCE010196C1
:108880000E94400BCE0101960E94968D80915C0D56
:1088900090915D0D8430910551F481E090E0DBDE34
:1088A00081111CC010925D0D10925C0D17C0892BB8
:1088B000A9F481E090E0CFDE81110AC081E090E070
:1088C000CADE811105C081E090E0C5DE882331F069
:1088D00084E090E090935D0D80935C0D80915C0D41
:1088E00090915D0D049791F16AEA72E08BE39CE050
:1088F0000E947F8F6BE37CE0CE0101960E94808E08
:108900004AE050E060E070E0CE0101960E94CC09A0
:10891000CE0101960E94968D6BE37CE0CE0101961C
:108920000E94808E62E275E0CE0101960E940B905B
:1089300065E37CE00E94FA8FBC018BE39CE00E941F
:108940006B8ECE0101960E94968D8FC08AE090E0DA
:1089500021DC6B017C0120E030E0A9010E947492CF
:1089600018162CF08AE090E015DC6B017C0120E009
:1089700030E041EE53E4C701B6010E94749218162C
:108980004CF068EC70E080E090E00E946B8483E043
:1089900090E0EACF20E030E0A901C701B6010E94D3
:1089A000749218163CF06CE972E08BE39CE00E9434
:1089B0007F8F31C020E030E048EC52E4C701B601BF
:1089C0000E94749287FF02C021E001C020E0B7013D
:1089D000A601CE0107960E94238F6EE176E0CE01BC
:1089E00001960E94018EBE01695F7F4FCE01019604
:1089F0000E94FA8F63E276E00E940B90BC018BE349
:108A00009CE00E946B8ECE0101960E94968DCE0155
:108A100007960E94968D6BE37CE0CE0101960E9442
:108A2000808E42E350E06FEF7FEFCE0101960E940F
:108A3000400BCE0101960E94968D63E972E085E3BA
:108A40009CE00E947F8F65E37CE0CE0101960E944E
:108A5000808E42E350E060E070E0CE0101960E941B
:108A6000CC09CE0101960E94968D80912C0C882312
:108A700031F060E273E080E090E00E946B842C961D
:108A80000FB6F894DEBF0FBECDBFDF91CF91FF9040
:108A9000EF90DF90CF9008954F925F926F927F9208
:108AA0008F929F92AF92BF92CF92DF92EF92FF92FE
:108AB000CF93DF93CDB7DEB760970FB6F894DEBFE4
:108AC0000FBECDBF80912C0C811105C08EE190E0CE
:108AD000A0E0B0E004C082E090E0A0E0B0E08D87CC
:108AE0009E87AF87B88B62E073E08BE39CE00E94C7
:108AF0007F8F6BE37CE0CE0101960E94808E4AE07E
:108B000050E06FEF7FEFCE0101960E94400BCE0147
:108B100001960E94968D812C912C5401C12CD12C50
:108B2000760163E270E081E39EE00E94A67567E053
:108B300070E081E39EE00E94580981E39EE00E947C
:108B40001A7666E970E080E090E00E946B8463E250
:108B500070E081E39EE00E94A67560E270E081E330
:108B60009EE00E94580981E39EE00E941A7666E921
:108B700070E080E090E00E946B8442E050E063E2AD
:108B800070E081E39EE00E941876412C512C320166
:108B900081E39EE00E94FE74181619066CF481E3CE
:108BA0009EE00E940675762C652C542C4424480EB9
:108BB000511C611C711CECCFC301B2010E94449393
:108BC0002AE939E949E95FE30E9478920E9411930A
:108BD000AB01BC01C416D506E606F70614F46A011B
:108BE0007B012AE0CE0107960E94F78EBE01695FE5
:108BF0007F4FCE0101960E94808E64E977E0CE011E
:108C000001960E940B90BC0185E39CE00E946B8E54
:108C1000CE0101960E94968DCE0107960E94968DF8
:108C200065E37CE0CE0101960E94808E4EE150E02B
:108C300060E070E0CE0101960E94750ACE010196B7
:108C40000E94968D9FEF891A990AA90AB90A8D8503
:108C50009E85AF85B88988159905AA05BB050CF0D6
:108C600060CF2AE0B701A601CE0107960E94F78ED9
:108C7000BE01695F7F4FCE0101960E94808E64E93C
:108C800077E0CE0101960E940B90BC0185E39CE049
:108C90000E946B8ECE0101960E94968DCE010796A2
:108CA0000E94968D65E37CE0CE0101960E94808E45
:108CB0004AE050E060E070E0CE0101960E94CC09ED
:108CC000CE0101960E94968D2AE0B701A601CE0141
:108CD00007960E94F78E68E977E0CE0101960E9420
:108CE000018EBE01695F7F4FCE0101960E94FA8F0F
:108CF0006BE977E00E940B906BE37CE00E94FA8FB7
:108D0000BC018BE39CE00E946B8ECE0101960E9419
:108D1000968DCE0107960E94968D62E370E080E00A
:108D200090E00E946B8460960FB6F894DEBF0FBE91
:108D3000CDBFDF91CF91FF90EF90DF90CF90BF90AC
:108D4000AF909F908F907F906F905F904F9008951D
:108D50008F929F92AF92BF92CF92DF92EF92FF924B
:108D60000F931F93CF93DF9300D000D0CDB7DEB722
:108D70008C01E090290CF0902A0C62E378E08AEFF5
:108D80009EE00E941B8A4AE050E0B8018AEF9EE014
:108D90000E943D8BC8010596059708F18091290C2A
:108DA00090912A0C8017910709F10E941B0C1093D7
:108DB0002A0C0093290C0E946D2E4AE0B801CE01C6
:108DC00001960E94CC8EBE016F5F7F4F87E49CE0CE
:108DD0000E94888ECE0101960E94968D07C00E3F9C
:108DE0008FEF1807A9F40E947B2E9DC162E275E007
:108DF000CE0101960E94018E4AE050E06FEF7FEFB6
:108E0000CE0101960E94750ACE0101960E94968DB0
:108E1000F8017996E332F10508F024C1EE58FF4FCE
:108E20000C94599680912C0C882319F00E94A0353F
:108E300047C160910A0270910B0280910C029091DF
:108E40000D020E9495333CC18091E2049091E304AD
:108E50000E94DF2E35C18091C8049091C9040E9400
:108E600019282EC18091BC049091BD040E947E2CD3
:108E700027C18091BE049091BF04C8DC21C10E942B
:108E80003C840E9480371CC160E070E08091C20485
:108E90009091C3040E94462413C18091B80490911C
:108EA000B9040E94322A0CC180912B0C91E08927D1
:108EB00080932B0C80912C0C882331F06BE37CE0A9
:108EC00084E390E10E94678A68EC70E080E090E0C3
:108ED0000E946B84F5C010922C0CF2C081E080934C
:108EE0002C0CEEC00E94400CEBC04AD8E9C00E9496
:108EF0007816E6C080913C02882309F4E1C069EC51
:108F00007AE0CE0101960E94018E4AE050E061E0D5
:108F100070E0CE0101960E94CC09CE0101960E941C
:108F2000968D0E94460ECCC0B7DDCAC08091C404A5
:108F30009091C5040E94BF2BC3C08091BA04909148
:108F4000BB040E94C92ABCC080913C02882309F45A
:108F5000B7C080912C0C882329F082E090E00E9419
:108F60008B10AEC083E090E00E94BA14A9C00E94AA
:108F7000762284E390E10E94C486A2C0809181029F
:108F8000909182020E946F269BC080913C028823B0
:108F900009F496C080912C0C811127C0C0900A0260
:108FA000D0900B02E0900C02F0900D0220E030E037
:108FB0004AE754E4C701B6010E94D8940E94119375
:108FC0004B015C0120E030E040EA50E4C701B6010B
:108FD0000E94D89420E030E040EA50E40E94AE9134
:108FE0000E941193A501940108C021E030E040E007
:108FF00050E06AE070E080E090E00E94461E60C0B1
:1090000080915E0D90915F0D892BA1F481E090E03D
:1090100090935F0D80935E0D8EED93E09093C00B67
:109020008093BF0B0E94A80968EC70E080E090E09C
:109030000E946B84E091F60AF091F70A199540C0FE
:10904000E091450DF091460D0480F581E02D20E082
:1090500042E060E185E49DE019950E946D2E0E943A
:109060001B0C2EC0F0922A0CE092290C65E278E0ED
:109070008BE39CE00E947F8F69EC7AE0CE01019641
:109080000E94018E4AE050E060E070E0CE0101965F
:109090000E94CC09CE0101960E94968D6BE37CE084
:1090A000CE0101960E94808E4AE050E06FEF7FEF84
:1090B000CE0101960E94400BCE0101960E94968D32
:1090C00080913F0C9091400C009799F0419718F4D3
:1090D00002301105ACF46BE37CE0CE0101960E94F6
:1090E000808ECE0101960E94A20FCE0101960E94B1
:1090F000968D64E670E080E090E00E946B8413C07F
:109100006BE37CE0CE0101960E94808E4AE050E045
:109110006FEF7FEFCE0101960E94400BCE010196CA
:109120000E94968DD8CF26960FB6F894DEBF0FBE5C
:10913000CDBFDF91CF911F910F91FF90EF90DF9006
:10914000CF90BF90AF909F908F900895FF920F9314
:109150001F93CF93DF9300D000D0CDB7DEB782341A
:1091600009F472C0D4F4803309F48EC07CF48332E5
:1091700009F481C08A3209F0A5C06CEA77E08DE479
:109180009CE00E949E8E8FEF9FEFF8C0813309F420
:109190008AC0813409F44DC095C0813609F449C0B4
:1091A00034F4833409F45BC0843449F08BC08336D3
:1091B00009F455C00CF448C0843609F083C080918E
:1091C0004B0C90914C0C892B09F4DAC087E49CE09D
:1091D0000E94879197FDD4C06FE178E08AEF9EE00E
:1091E0000E941B8A67E47CE08AEF9EE00E94678A07
:1091F00087E49CE00E948791DC01CB014AEF5FEF9E
:109200006FEF7FEF481B590B6A0B7B0B2AE0CE01F7
:1092100001960E94F78EBE016F5F7F4F87E49CE04E
:109220000E94888ECE0101960E94968D87E49CE074
:10923000A2C060EA77E08DE49CE00E949E8E80915F
:10924000290C90912A0C9AC063EA77E08DE49CE0A7
:109250000E949E8E10922C0C8CEF9FEF8FC066EABE
:1092600077E08DE49CE00E949E8E81E080932C0C40
:109270008DEF9FEF83C069EA77E08DE49CE00E9468
:109280009E8E8EEF9FEF7AC06AEB77E087E49CE0DA
:109290000E949E8E6AEB77E08DE49CE00E949E8E99
:1092A00080E090E06BC06DEA77E087E49CE00E948C
:1092B0009E8E6DEA77E08DE49CE00E949E8E81E0B8
:1092C00090E05CC0682FCE0101960E94B48EBE0172
:1092D0006F5F7F4F87E49CE00E94888ECE010196ED
:1092E0000E94968D87E49CE00E948791CB0130DD3F
:1092F00064E670E080E090E00E946B8449C00F5FFC
:109300001F4F093E83E0180769F06EE170E080E0CE
:1093100090E00E946B8487EB9CE00E94D283F82E41
:10932000FF2069F36AE270E06F197109F7FC739529
:109330004AE0CE0101960E94CC8EBE016F5F7F4F46
:109340008DE49CE00E94888ECE0101960E94968D4D
:109350006DE47CE087E49CE00E946B8E69E178E03C
:109360008AEF9EE00E941B8A6F2D8AEF9EE00E948A
:10937000878A8DE49CE00E948791CB01E9DC08C0DC
:1093800087EB9CE00E94D283F82E00E010E0C8CF6B
:1093900026960FB6F894DEBF0FBECDBFDF91CF91FA
:1093A0001F910F91FF9008950F931F93CF93DF9319
:1093B00000D000D0CDB7DEB740910C0B50910D0B13
:1093C00060910E0B70910F0B20E130E08AEF9EE070
:1093D0000E94848B80910C0B90910D0BA0910E0B31
:1093E000B0910F0B883025E09207A105B10509F473
:1093F000F8C108F08DC0893421E09207A105B105BC
:1094000009F4F2C1E0F5843421E09207A105B10529
:1094100009F4DBC1E8F4813421E09207A105B1052C
:1094200009F4C4C138F480349140A105B10509F4B0
:10943000AEC1DDC1823421E09207A105B10509F476
:10944000BEC183349140A105B10509F4BBC1CFC1B0
:10945000863421E09207A105B10509F4BCC108F4E6
:10946000B7C1873421E09207A105B10509F4B6C15F
:1094700088349140A105B10509F4B3C1B8C1823067
:1094800025E09207A105B10509F499C1E8F48437F4
:1094900021E09207A105B10509F444C138F48237EF
:1094A0009140A105B10509F448C1A1C1811525E08C
:1094B0009207A105B10509F46AC181309540A10563
:1094C000B10509F473C193C1853025E09207A10568
:1094D000B10509F47DC170F4833025E09207A10540
:1094E000B10509F46FC184309540A105B10509F4B7
:1094F0006CC17DC1863025E09207A105B10509F454
:109500006AC187309540A105B10509F467C16FC1F3
:109510008D3B22E492072FEFA207B10509F428C181
:1095200008F04BC08F3E20E192072FEFA207B10554
:1095300009F454C118F5823325E09207A105B1055D
:1095400009F4FBC038F489309540A105B10509F450
:109550004BC14DC1843325E09207A105B10509F443
:10956000E1C08D3F9240AF4FB10509F040C160EAC4
:1095700077E08DE49CE00E949E8EDCC08D3D22E26F
:1095800092072FEFA207B10509F4CCC038F4873E4B
:109590009841AF4FB10509F41BC129C18F3C20E3AD
:1095A00092072FEFA207B10509F40FC1873C98433A
:1095B000AF4FB10509F415C11AC1873928E69207E2
:1095C0002FEFA207B10509F4F1C048F58D3A22E565
:1095D00092072FEFA207B10509F4BBC038F4853B11
:1095E0009A44AF4FB10509F4D2C001C1853A2AE5CA
:1095F00092072FEFA207B10509F4F6C08D39924604
:10960000AF4FB10509F0F3C063EA77E08DE49CE069
:109610000E949E8E10922C0C8CEF9FEF81C087359C
:1096200028EA92072FEFA207B105F9F078F4853800
:109630002AE792072FEFA207B10509F4CCC08736BD
:109640009849AF4FB10509F4BAC0D1C08F3420EBAF
:1096500092072FEFA207B10509F4B4C08D33924CE5
:10966000AF4FB10509F469C0C2C088E19BE00E9418
:10967000A96600E010E068EF7AE088E19BE00E94D4
:109680005E67892B39F40F5F1F4F093E83E018078F
:1096900009F09CC167E078E08AEF9EE00E941B8A97
:1096A0004091FC0A5091FD0A6091FE0A7091FF0AF8
:1096B0002AE030E08AEF9EE00E94848B8091FC0AD1
:1096C0009091FD0AA091FE0AB091FF0A853025E035
:1096D0009207A105B10509F4B9C008F0C0C08734EC
:1096E00021E09207A105B10509F4D9C008F0DAC05C
:1096F000833421E09207A105B10509F4E3C008F025
:109700009EC0813421E09207A105B10509F0E3C0B4
:109710006FEA77E087E49CE00E949E8E89EF9FEFDE
:1097200017DB7EC060EA77E08DE49CE00E949E8EAD
:1097300010922C0C8BEF9FEFF3CF66EA77E08DE46D
:109740009CE00E949E8E81E080932C0C8DEF9FEF19
:10975000E7CF69EA77E087E49CE00E949E8E69EAA1
:1097600077E08DE49CE00E949E8E8EEF9FEFD8CF35
:109770006CEA77E087E49CE00E949E8E6CEA77E0DA
:109780008DE49CE00E949E8E8FEF9FEFC9CF6AEB25
:1097900077E087E49CE00E949E8E6AEB77E08DE4A0
:1097A0009CE00E949E8E80E090E0BACF6DEA77E068
:1097B00087E49CE00E949E8E81E090E0B1CF82E041
:1097C00090E0AECF83E090E0ABCF84E090E0A8CF14
:1097D00085E090E0A5CF86E090E0A2CF87E090E022
:1097E0009FCF88E090E09CCF89E090E099CF40E067
:1097F00050E06DE47CE0CE0101960E944909BE0173
:109800006F5F7F4F87E49CE00E94888ECE010196B7
:109810000E94968D64E670E080E090E00E946B8488
:1098200088E19BE00E94A96626960FB6F894DEBFF9
:109830000FBECDBFDF91CF911F910F910895853459
:1098400021E09207A105B10509F054C06CEB77E067
:1098500087E49CE00E949E8E85EF9FEF61CF8F3C56
:1098600020E392072FEFA207B10509F448C008F0E2
:109870004FC0883025E09207A105B10509F46FC0FB
:1098800008F080C0863025E09207A105B10509F4F3
:109890005DC087309540A105B10509F0BBCF83EFCE
:1098A0009FEF3ECF813025E09207A105B10509F475
:1098B0002FCF08F44EC0833025E09207A105B105F3
:1098C00009F059C065EB77E087E49CE00E949E8E2A
:1098D00087EF9FEF25CF82349140A105B10509F0B4
:1098E00099CF62EB77E087E49CE00E949E8E88EF40
:1098F0009FEF16CF86349140A105B10538F568EB8E
:1099000077E087E49CE00E949E8E86EF9FEF08CF71
:10991000873928E692072FEFA207B10509F4F8CEA0
:1099200008F447C0873628E992072FEFA207B10550
:10993000C1F28F3420EB92072FEFA207B10511F28D
:1099400085389A47AF4FB10509F064CF84EF9FEF98
:10995000E7CE883421E09207A105B10519F482EF22
:109960009FEFDECE89349140A105B10509F052CFB9
:1099700081EF9FEFD5CE84309540A105B10508F465
:10998000B0CFBDCF8F3E20E192072FEFA207B105E8
:1099900009F485CF873E28E192072FEFA207B10592
:1099A00009F454CF89309540A105B10509F032CFB3
:1099B000DFCF873C28E392072FEFA207B10579F2AA
:1099C000853A9A45AF4FB10599F224CF6EE170E028
:1099D00080E090E00E946B844ECE8F929F92AF9277
:1099E000BF92CF92DF92EF92FF920F931F93CF938C
:1099F000DF93CDB7DEB7A6970FB6F894DEBF0FBEE4
:109A0000CDBF68E07BE088E19BE00E945E67892B28
:109A1000C9F00E946D2E0E941B0C62E275E0CE011F
:109A200001960E94018E4AE050E060E070E0CE01B5
:109A300001960E94CC09CE0101960E94968DB4DC5D
:109A40000C94815D69EC7AE08DE49CE00E949E8E2E
:109A50000E94EE416AE070E080E090E00E946B843A
:109A60008091510C9091520C009711F40C94665D0A
:109A7000019709F046C065E576E0CE010F960E9499
:109A8000018EBE01615F7F4F8DE49CE00E94479094
:109A900081112AC069E276E0CE0109960E94018E0A
:109AA000BE01675F7F4F8DE49CE00E94479081116B
:109AB00015C06DE875E0CE0101960E94018EBE01D1
:109AC0006F5F7F4F8DE49CE00E94479011E0811111
:109AD00010E0CE0101960E94968D01C010E0CE01EB
:109AE00009960E94968D01C010E0CE010F960E944B
:109AF000968D112331F06DE47CE087E49CE00E94B8
:109B00006B8E8091510C9091520C0497F0F560ECA3
:109B100077E0CE0101960E94018EBE016F5F7F4FFC
:109B20008DE49CE00E944790182FCE0101960E9480
:109B3000968D112351F141E050E06DE47CE0CE01BF
:109B400009960E944909CE0109960E948791DC017D
:109B5000CB014AEF5FEF6FEF7FEF481B590B6A0BAA
:109B60007B0B2AE0CE0101960E94F78EBE016F5F4B
:109B70007F4F87E49CE00E94888ECE0101960E9470
:109B8000968DCE0109960E94968D62EC77E0CE010B
:109B900009960E94018EBE01675F7F4F8DE49CE0B5
:109BA0000E944790811116C066EC77E0CE010196C5
:109BB0000E94018EBE016F5F7F4F8DE49CE00E948A
:109BC000479011E0811101C010E0CE0101960E9482
:109BD000968D01C011E0CE0109960E94968D112349
:109BE00009F4EFC26DE97BE0CE0101960E949F8FE0
:109BF000CE0101960E94A20FCE0101960E94968D81
:109C0000609138027091390280913A0290913B0242
:109C10000E94449320E030E048EC52E40E947892A5
:109C2000AB01BC0122E0CE010F960E94238F6AECAB
:109C300077E0CE0109960E94018EBE01615F7F4FE1
:109C4000CE0109960E94FA8F6BEE78E00E940B908D
:109C5000BC01CE0101960E94808ECE0101960E9429
:109C6000A20FCE0101960E94968DCE0109960E9408
:109C7000968DCE010F960E94968D409134025091A0
:109C80003502609136027091370224E0CE010F96C2
:109C90000E94238F6FED77E0CE0109960E94018E1E
:109CA000BE01615F7F4FCE0109960E94FA8FBC0111
:109CB000CE0101960E94808ECE0101960E94A20FD5
:109CC000CE0101960E94968DCE0109960E94968D36
:109CD000CE010F960E94968D40911E0250911F0258
:109CE000609120027091210222E0CE0109960E942B
:109CF000238F4091160250911702609118027091C3
:109D0000190223E0CE010F960E94238F4091220278
:109D100050912302609124027091250222E0CE012D
:109D200045960E94238F40911A0250911B02609128
:109D30001C0270911D0223E0CE0181960E94238FA8
:109D40006CEF77E0CE014B960E94018EBE016F5DF5
:109D50007F4FCE014B960E94FA8F61E178E00E941E
:109D60000B90BE016B5E7F4F0E94FA8F64E178E03A
:109D70000E940B90BE01615F7F4F0E94FA8F61E1EC
:109D800078E00E940B90BE01675F7F4F0E94FA8FC0
:109D90006AE178E00E940B90BC01CE0101960E941E
:109DA000808ECE0101960E94A20FCE0101960E94E4
:109DB000968DCE014B960E94968DCE0181960E9483
:109DC000968DCE0145960E94968DCE010F960E94EB
:109DD000968DCE0109960E94968D6FE178E0CE01B6
:109DE00009960E94018E67E37DE0CE0109960E94EC
:109DF000FA8FBC01CE0101960E94808ECE010196A1
:109E00000E94A20FCE0101960E94968DCE01099666
:109E10000E94968D40914502509146026091470202
:109E20007091480223E0CE0109960E94238F209171
:109E3000490230914A0240914B0250914C0260E03D
:109E400070E080E291E40E943B95AB01BC0121E00F
:109E5000CE0145960E94518F60E378E0CE010F96C7
:109E60000E94018EBE016B5E7F4FCE010F960E9455
:109E7000FA8F63E478E00E940B90BE01675F7F4F2A
:109E80000E94FA8F67E576E00E940B90BC01CE013C
:109E900001960E94808ECE0101960E94A20FCE01F3
:109EA00001960E94968DCE010F960E94968DCE014E
:109EB00045960E94968DCE0109960E94968D4091FE
:109EC000410250914202609143027091440223E0AA
:109ED000CE0109960E94238F20913D0230913E02CF
:109EE00040913F025091400260E070E080E291E4D6
:109EF0000E943B95AB01BC0121E0CE0145960E943A
:109F0000518F69E478E0CE010F960E94018EBE0168
:109F10006B5E7F4FCE010F960E94FA8F63E478E06C
:109F20000E940B90BE01675F7F4F0E94FA8F67E52A
:109F300076E00E940B90BC01CE0101960E94808EBB
:109F4000CE0101960E94A20FCE0101960E94968D2D
:109F5000CE010F960E94968DCE0145960E94968D59
:109F6000CE0109960E94968D40914D0250914E026D
:109F700060914F027091500222E0CE010F960E9434
:109F8000238F6CE578E0CE0109960E94018EBE0118
:109F9000615F7F4FCE0109960E94FA8F62E778E0F9
:109FA0000E940B90BC01CE0101960E94808ECE01D2
:109FB00001960E94A20FCE0101960E94968DCE01BD
:109FC00009960E94968DCE010F960E94968D409123
:109FD000120250911302609114027091150222E056
:109FE000CE010F960E94238F69E778E0CE01099693
:109FF0000E94018EBE01615F7F4FCE0109960E94D3
:10A00000FA8F67E576E00E940B90BC01CE010196C5
:10A010000E94808ECE0101960E94A20FCE01019671
:10A020000E94968DCE0109960E94968DCE010F96C4
:10A030000E94968D06E9C02E04E0D02E01E010E0CB
:10A0400087E1E82E80919404909195048017910700
:10A050000CF44FC0D601AD90BD906D014AE0B50142
:10A06000CE0109960E94CC8E4AE0B801CE014596F9
:10A070000E94CC8E6CE878E0CE010F960E94018E93
:10A08000BE016B5E7F4FCE010F960E94FA8F69E48E
:10A0900075E00E940B90BE01675F7F4F0E94FA8FB0
:10A0A00064E978E00E940B90EA9CB001EB9C700D93
:10A0B00011246D577D4F0E940B90BC01CE0101967B
:10A0C0000E94808ECE0101960E94A20FCE010196C1
:10A0D0000E94968DCE010F960E94968DCE014596D8
:10A0E0000E94968DCE0109960E94968D0F5F1F4F9C
:10A0F000A9CF40910E0250910F0260911002709111
:10A10000110222E0CE010F960E94238F6AE978E0C7
:10A11000CE0109960E94018EBE01615F7F4FCE0184
:10A1200009960E94FA8F64ED76E00E940B90BC01C4
:10A13000CE0101960E94808ECE0101960E94A20F50
:10A14000CE0101960E94968DCE0109960E94968DB1
:10A15000CE010F960E94968D40910A0250910B02FB
:10A1600060910C0270910D0222E0CE010F960E94C8
:10A17000238F6AEA78E0CE0109960E94018EBE0123
:10A18000615F7F4FCE0109960E94FA8F64ED76E001
:10A190000E940B90BC01CE0101960E94808ECE01E0
:10A1A00001960E94A20FCE0101960E94968DCE01CB
:10A1B00009960E94968DCE010F960E94968D10E012
:10A1C00001C011E00E946D2E0E941B0C62E275E03E
:10A1D000CE0101960E94018E4AE050E060E070E0FE
:10A1E000CE0101960E94750ACE0101960E94968DBD
:10A1F0008091510C9091520C8330910508F06FC002
:10A20000019739F460E070E08DE49CE00E94669074
:10A21000F82E8091510C9091520C029709F050C089
:10A2200060EC77E0CE0101960E94018EBE016F5F67
:10A230007F4F8DE49CE00E944790182FCE0101963D
:10A240000E94968D1123E1F161E070E08DE49CE0C5
:10A250000E946690682FCE0101960E94B48EBE01C6
:10A260006F5F7F4F87E49CE00E94938ECE01019642
:10A270000E94968D60E070E08DE49CE00E94669004
:10A28000F82E65EA78E0CE0101960E94018E6DE419
:10A290007CE0CE0101960E94FA8F62E275E00E9496
:10A2A0000B90BC018AEF9EE00E943E8ACE0101968F
:10A2B0000E94968D67E47CE08AEF9EE00E94678AA8
:10A2C0008F2D0E94A6480E943C846093530C70938B
:10A2D000540C8093550C9093560C0C94815D21E0A6
:10A2E00030E040E050E06DE47CE0CE0101960E9459
:10A2F000E890BE016F5F7F4F85E39CE00E94888EEF
:10A30000CE0101960E94968D67EE78E0CE01099607
:10A310000E94018EBE01675F7F4F8DE49CE00E942A
:10A320004790811116C06FEE75E0CE0101960E9434
:10A33000018EBE016F5F7F4F8DE49CE00E944790CD
:10A3400001E0811101C000E0CE0101960E94968DCE
:10A3500001C001E0CE0109960E94968D002309F408
:10A36000A7C042E050E06DE47CE0CE0101960E947F
:10A370004909BE016F5F7F4F85E39CE00E94888E94
:10A38000CE0101960E94968D65E37CE08AEF9EE007
:10A390000E94678A85E39CE00E94919120E030E072
:10A3A00048EC52E40E94D8940E941193AB01BC0186
:10A3B000409338025093390260933A0270933B0203
:10A3C0002AE030E08AEF9EE00E94538B60913802D1
:10A3D0007091390280913A0290913B028B019C016D
:10A3E00000591F452140310901341C49210531051F
:10A3F00088F06AEB78E0CE0101960E94018E65E359
:10A400007CE0CE0101960E94FA8F6DEC78E00E940C
:10A410000B9073C119821A821B821C821D821E82BC
:10A420001F8218860E94449320E030E048EC52E4FA
:10A430000E9478928E010F5F1F4F22E047E00E943A
:10A44000B996BC018BE39CE00E949E8E6DED78E096
:10A45000CE0109960E94018E6BE37CE0CE01099645
:10A460000E94FA8F6AEE78E00E940B90BC018BE3A9
:10A470009CE00E946B8ECE0109960E94968D1092F0
:10A48000C00B1092BF0B8091380290913902A091BD
:10A490003A02B0913B028093190B90931A0BA09350
:10A4A0001B0BB0931C0B80E090E00E947F092EC133
:10A4B0006FEE78E0CE0109960E94018EBE01675FC3
:10A4C0007F4F8DE49CE00E944790811116C065EF9C
:10A4D00078E0CE0101960E94018EBE016F5F7F4F32
:10A4E0008DE49CE00E94479001E0811101C000E0F2
:10A4F000CE0101960E94968D01C001E0CE01099621
:10A500000E94968D002309F46DC026E030E045E0FE
:10A5100050E06DE47CE0CE0101960E94E890BE011F
:10A520006F5F7F4F85E39CE00E94888ECE0101968D
:10A530000E94968D85E39CE00E9487916B017C01CF
:10A5400060E778E0CE0109960E94018EBE01675F48
:10A550007F4F8DE49CE00E94DF90AC014F5F5F4F26
:10A560006DE47CE0CE0101960E944909BE016F5F57
:10A570007F4F85E39CE00E94888ECE0101960E9469
:10A58000968DCE0109960E94968D85E39CE00E94EF
:10A590008791DB01E6E9F4E021E030E040919404AA
:10A5A00050919504421753075CF0408151814A173E
:10A5B0005B0711F4118210822F5F3F4F3296EECF6E
:10A5C000F601EE0FFF1FEC56FB4F7183608382E0B4
:10A5D00090E00E94322D6DE47CE08AEF9EE00E94C4
:10A5E000678A49C06BEF78E0CE0109960E94018E20
:10A5F000BE01675F7F4F8DE49CE00E944790811110
:10A6000016C061E079E0CE0101960E94018EBE0184
:10A610006F5F7F4F8DE49CE00E94479001E08111C5
:10A6200001C000E0CE0101960E94968D01C001E0BC
:10A63000CE0109960E94968D002339F1E6E9F4E0F7
:10A6400081E090E020919404309195042817390717
:10A6500074F0863091051CF49183808305C09C01C1
:10A660002E5F3F4F3183208301963296EBCF82E0FD
:10A6700090E00E94322D1092C00B1092BF0B80E030
:10A6800090E00E947F090C94815D67E079E0CE0143
:10A6900009960E94018EBE01675F7F4F8DE49CE0AA
:10A6A0000E944790811116C06FE079E0CE010196BB
:10A6B0000E94018EBE016F5F7F4F8DE49CE00E947F
:10A6C000479001E0811101C000E0CE0101960E9497
:10A6D000968D01C001E0CE0109960E94968D00235F
:10A6E00091F167E179E0CE0101960E94018E61E36C
:10A6F0007DE0CE0101960E94FA8FBC018BE39CE0C5
:10A700000E946B8ECE0101960E94968D6CE277E0DE
:10A71000CE0109960E94018E6BE37CE0CE01099682
:10A720000E94FA8FBC01CE0101960E94808ECE015C
:10A7300001960E94A20FCE0101960E94968DCE0135
:10A7400009960C94635D61E279E0CE0109960E945E
:10A75000018EBE01675F7F4F8DE49CE00E944790B1
:10A76000811116C066E279E0CE0101960E94018E49
:10A77000BE016F5F7F4F8DE49CE00E94479001E037
:10A78000811101C000E0CE0101960E94968D01C0AA
:10A7900001E0CE0109960E94968D002309F444C081
:10A7A00060E778E0CE0109960E94018EBE01675FE6
:10A7B0007F4F8DE49CE00E94DF90AC014F5F5F4FC4
:10A7C0006DE47CE0CE0101960E944909BE016F5FF5
:10A7D0007F4F85E39CE00E94888ECE0101960E9407
:10A7E000968DCE0109960E94968D85E39CE00E948D
:10A7F00087916115710521F481E08093F50410C003
:10A800006130710519F41092F5040AC062307105C7
:10A8100011F00C94815D81E08093F5041092F404B2
:10A820000E947B2E0C94815D6BE279E0CE0109964B
:10A830000E94018EBE01675F7F4F8DE49CE00E9405
:10A840004790811116C06FE279E0CE0101960E9417
:10A85000018EBE016F5F7F4F8DE49CE00E944790A8
:10A8600001E0811101C000E0CE0101960E94968DA9
:10A8700001C001E0CE0109960E94968D002309F4E3
:10A880005CC043E050E06DE47CE0CE0101960E94A4
:10A890004909BE016F5F7F4F85E39CE00E94888E6F
:10A8A000CE0101960E94968D65E37CE08AEF9EE0E2
:10A8B0000E94678A1092C00B1092BF0B65E37CE088
:10A8C00087E39DE00E946B8E20E030E048E050E09E
:10A8D00065E37BE087E39DE00E9467908091BF0B7A
:10A8E0009091C00B0E947F0963E379E0CE0101964D
:10A8F0000E94018E67E37DE0CE0101960E94FA8FEF
:10A90000BC01CE0109960E94808ECE0101960E9464
:10A91000968DBE01675F7F4F84E390E10E943E8A7F
:10A9200068EB7BE080E090E00E946B8465E37BE075
:10A930008AEF9EE00E94778A69C06BE379E0CE01DE
:10A9400009960E94018EBE01675F7F4F8DE49CE0F7
:10A950000E944790811116C060E479E0CE01019613
:10A960000E94018EBE016F5F7F4F8DE49CE00E94CC
:10A97000479001E0811101C000E0CE0101960E94E4
:10A98000968D01C001E0CE0109960E94968D0023AC
:10A9900009F43FC044E050E06DE47CE0CE01019654
:10A9A0000E944909BE016F5F7F4F85E39CE00E94D2
:10A9B000888ECE0101960E94968D65E479E0CE01E5
:10A9C00001960E94018E65E37CE0CE0101960E9413
:10A9D000FA8FBC01CE0109960E94808ECE010196AD
:10A9E0000E94968DBE01675F7F4F84E390E10E94D5
:10A9F0003E8A68EB7BE080E090E00E946B84BE01C1
:10AA0000675F7F4F8AEF9EE00E94678ACE010996BA
:10AA100091C76CE479E0CE010F960E94018EBE01D1
:10AA2000615F7F4F8DE49CE00E94479081112BC0B5
:10AA30006FE479E0CE0109960E94018EBE01675F46
:10AA40007F4F8DE49CE00E944790811116C062E523
:10AA500079E0CE0101960E94018EBE016F5F7F4FAB
:10AA60008DE49CE00E94479001E0811101C000E06C
:10AA7000CE0101960E94968D01C001E0CE0109969B
:10AA80000E94968D01C001E0CE010F960E94968D26
:10AA9000002309F42DC1AAE0AA2EB12CC12CD12C7F
:10AAA000760188248A94B3E09B2E6EE170E080E00A
:10AAB00090E00E946B84809181020E940185B40124
:10AAC0000E940896882777FD8095982F0E944493CE
:10AAD00020E030E040EA50E40E94D8949B01AC01B1
:10AAE000C701B6010E94AE916B017C01E1E0AE1A94
:10AAF000B108D9F620E030E040E251E40E947892BB
:10AB00006B017C0165E579E0CE0109960E94018E1A
:10AB1000BE01675F7F4F8DE49CE00E9447908111EA
:10AB200016C069E579E0CE0101960E94018EBE0152
:10AB30006F5F7F4F8DE49CE00E94479001E08111A0
:10AB400001C000E0CE0101960E94968D01C001E097
:10AB5000CE0109960E94968D002309F43FC020E0A3
:10AB600030E040E650E4C701B6010E94D8949B0152
:10AB7000AC0160E070E080E890E40E94AD91AB0130
:10AB8000BC0140932A0250932B0260932C027093D5
:10AB90002D0222E0CE0101960E94238FBE016F5F3D
:10ABA0007F4F8BE39CE00E94888ECE0101960E942D
:10ABB000968D6DE579E0CE0101960E94018E6BE3E2
:10ABC0007CE0CE0101960E94FA8FBC018BE39CE0F1
:10ABD0000E946B8ECE0101960E94968D6CE679E004
:10ABE000CE0109960E94018EBE01675F7F4F8DE402
:10ABF0009CE00E944790811116C061E779E0CE0188
:10AC000001960E94018EBE016F5F7F4F8DE49CE034
:10AC10000E94479001E0811101C000E0CE01019641
:10AC20000E94968D01C001E0CE0109960E94968D8A
:10AC3000002309F43FC020E030E040E650E4C701C3
:10AC4000B6010E94D8949B01AC0160E070E080E204
:10AC500091E40E94AD91AB01BC0140932602509358
:10AC60002702609328027093290222E0CE01019608
:10AC70000E94238FBE016F5F7F4F8BE39CE00E9499
:10AC8000888ECE0101960E94968D66E779E0CE010E
:10AC900001960E94018E6BE37CE0CE0101960E943A
:10ACA000FA8FBC018BE39CE00E946B8ECE01019673
:10ACB0000E94968D6CE277E0CE0109960E94018E8B
:10ACC0006BE37CE0CE0109960E94FA8FBC01CE01B5
:10ACD00001960E94808ECE0101960E94A20FCE01A5
:10ACE00001960E94968DCE0109960E94968DD6C639
:10ACF00066E879E0CE0101960E94018EBE016F5F89
:10AD00007F4F8DE49CE00E944790082FCE01019672
:10AD10000E94968D002309F46EC08091510C909191
:10AD2000520C079708F4BAC646E050E06DE47CE0A8
:10AD3000CE0101960E944909BE016F5F7F4F85E3F6
:10AD40009CE00E94888ECE0101960E94968D85E33C
:10AD50009CE00E949191AB01BC0140930E02509384
:10AD60000F02609310027093110221E0CE01099648
:10AD70000E94238F6AE978E0CE0101960E94018E3D
:10AD8000BE01675F7F4FCE0101960E94FA8F64ED8E
:10AD900076E00E940B90BC018BE39CE00E946B8EDE
:10ADA000CE0101960E94968DCE0109960E94968D45
:10ADB0006BE37CE0CE0101960E94808ECE0101966D
:10ADC0000E94A20FCE0101960E94968D0E943C84A3
:10ADD00028EE33E040E050E00E941B96CA01B90122
:10ADE0000E9442936093930B7093940B8093950B06
:10ADF0009093960B53C66DE879E0CE0101960E94C0
:10AE0000018EBE016F5F7F4F8DE49CE00E944790F2
:10AE1000082FCE0101960E94968D0023E9F18091C2
:10AE2000510C9091520C079708F438C646E050E058
:10AE30006DE47CE0CE0101960E944909BE016F5F7E
:10AE40007F4F85E39CE00E94888ECE0101960E9490
:10AE5000968D85E39CE00E949191AB01BC014093EB
:10AE60000A0250930B0260930C0270930D0221E0D2
:10AE7000CE0109960E94238F6AEA78E0CE010196FE
:10AE80000E94018EBE01675F7F4FCE0101960E9436
:10AE9000FA8F64ED76E04DC364E979E0CE0109965E
:10AEA0000E94018EBE01675F7F4F8DE49CE00E948F
:10AEB0004790811116C068E979E0CE0101960E94A1
:10AEC000018EBE016F5F7F4F8DE49CE00E94479032
:10AED00001E0811101C000E0CE0101960E94968D33
:10AEE00001C001E0CE0109960E94968D002309F46D
:10AEF00056C08091C2049091C3040E941B246093A9
:10AF00001A0270931B0280931C0290931D0260939F
:10AF10002D0B70932E0B80932F0B9093300B80E0B2
:10AF200090E0A0E8BFE38093220290932302A093D5
:10AF30002402B09325028093250B9093260BA093B7
:10AF4000270BB093280B62E87BE08AEF9EE00E941B
:10AF50001B8A40911A0250911B0260911C02709151
:10AF60001D0222E030E08AEF9EE00E94708C109279
:10AF7000C00B1092BF0B80E090E00E947F094091CF
:10AF80001A0250911B0260911C0270911D0222E076
:10AF9000CE0109960E94238F6CE979E0A7C465EA87
:10AFA00079E0CE0109960E94018EBE01675F7F4F56
:10AFB0008DE49CE00E944790811116C06BEA79E015
:10AFC000CE0101960E94018EBE016F5F7F4F8DE41E
:10AFD0009CE00E94479001E0811101C000E0CE0199
:10AFE00001960E94968D01C001E0CE0109960E9453
:10AFF000968D002309F465C08091510C9091520CFC
:10B000000797F8F046E050E06DE47CE0CE01019651
:10B010000E944909BE016F5F7F4F85E39CE00E945B
:10B02000888ECE0101960E94968D85E39CE00E9459
:10B03000919160934D0270934E0280934F029093D2
:10B0400050028091BC040E94F52C80914D02909199
:10B050004E02A0914F02B091500280934D0B9093FD
:10B060004E0BA0934F0BB093500B61E77BE08AEF40
:10B070009EE00E941B8A40914D0250914E026091C9
:10B080004F027091500222E030E08AEF9EE00E9471
:10B09000708C1092C00B1092BF0B80E090E00E9469
:10B0A0007F0940914D0250914E0260914F02709184
:10B0B000500222E0CE0109960E94238F61EB79E0D5
:10B0C00015C46BEB79E0CE0109960E94018EBE019A
:10B0D000675F7F4F8DE49CE00E944790811116C00E
:10B0E00060EC79E0CE0101960E94018EBE016F5F97
:10B0F0007F4F8DE49CE00E94479001E0811101C0E8
:10B1000000E0CE0101960E94968D01C001E0CE01C3
:10B1100009960E94968D002309F49BC08091510CE2
:10B120009091520C069708F145E050E06DE47CE008
:10B13000CE0101960E944909BE016F5F7F4F85E3F2
:10B140009CE00E94888ECE0101960E94968D85E338
:10B150009CE00E9491910E945A94609349027093DE
:10B160004A0280934B0290934C028091BE049091CE
:10B17000BF040E94AE2720E030E048E051E40E9486
:10B1800078926093450270934602809347029093B1
:10B19000480260933D0B70933E0B80933F0B90935E
:10B1A000400B8091490290914A02A0914B02B091CC
:10B1B0004C028093450B9093460BA093470BB093A2
:10B1C000480B61E67BE08AEF9EE00E941B8A20919B
:10B1D000490230914A0240914B0250914C0260E08A
:10B1E00070E080E291E40E943B95AB01BC0121E05C
:10B1F00030E08AEF9EE00E946F8C65EC79E08AEF88
:10B200009EE00E944C8A4091450250914602609116
:10B2100047027091480222E030E08AEF9EE00E94EF
:10B22000708C1092C00B1092BF0B80E090E00E94D7
:10B230007F0940914502509146026091470270910A
:10B24000480223E0CE0109960E94238F6CEC79E03E
:10B25000C7C065ED79E0CE0109960E94018EBE015E
:10B26000675F7F4F8DE49CE00E944790811116C07C
:10B270006AED79E0CE0101960E94018EBE016F5FFA
:10B280007F4F8DE49CE00E94479001E0811101C056
:10B2900000E0CE0101960E94968D01C001E0CE0132
:10B2A00009960E94968D002309F4A8C08091510C44
:10B2B0009091520C069708F145E050E06DE47CE077
:10B2C000CE0101960E944909BE016F5F7F4F85E361
:10B2D0009CE00E94888ECE0101960E94968D85E3A7
:10B2E0009CE00E9491910E945A9460933D02709359
:10B2F0003E0280933F02909340028091BE04909161
:10B30000BF040E94AE2720E030E048E051E40E94F4
:10B31000789260934102709342028093430290932B
:10B3200044026093410B7093420B8093430B9093C4
:10B33000440B80913D0290913E02A0913F02B0915A
:10B3400040028093490B90934A0BA0934B0BB09310
:10B350004C0B62E57BE08AEF9EE00E941B8A209105
:10B360003D0230913E0240913F025091400260E028
:10B3700070E080E291E40E943B95AB01BC0121E0CA
:10B3800030E08AEF9EE00E946F8C65EC79E08AEFF6
:10B390009EE00E944C8A409141025091420260918D
:10B3A00043027091440222E030E08AEF9EE00E9466
:10B3B000708C1092C00B1092BF0B80E090E00E9446
:10B3C0007F09409141025091420260914302709185
:10B3D000440223E0CE0109960E94238F6FED79E0AD
:10B3E000CE0101960E94018EBE01675F7F4FCE01A4
:10B3F00001960E94FA8F69E076E09BC068EE79E0E2
:10B40000CE0109960E94018EBE01675F7F4F8DE4D9
:10B410009CE00E944790811116C06CEE79E0CE014D
:10B4200001960E94018EBE016F5F7F4F8DE49CE00C
:10B430000E94479001E0811101C000E0CE01019619
:10B440000E94968D01C001E0CE0109960E94968D62
:10B45000002309F471C060E08091C8040E947A85DD
:10B4600009E110E0C12CD12C76018091C8040E9422
:10B470000185BC01882777FD8095982F0E94449311
:10B480009B01AC01C701B6010E94AE916B017C012A
:10B490006AE070E080E090E00E946B840150110946
:10B4A00021F720E030E040EA50E4C701B6010E94F5
:10B4B000D89420E030E040E85AE30E94D89420E09D
:10B4C00030E048EC51E40E9478926093120270934D
:10B4D000130280931402909315026093630B709390
:10B4E000640B8093650B9093660B1092C00B1092C7
:10B4F000BF0B80E090E00E947F09409112025091C2
:10B500001302609114027091150222E0CE01099697
:10B510000E94238F69E778E0CE0101960E94018E98
:10B52000BE01675F7F4FCE0101960E94FA8F67E5EB
:10B5300076E00E940B90E5C160EF79E0CE010996BC
:10B540000E94018EBE01675F7F4F8DE49CE00E94E8
:10B550004790811116C064EF79E0CE0101960E94F8
:10B56000018EBE016F5F7F4F8DE49CE00E9447908B
:10B5700001E0811101C000E0CE0101960E94968D8C
:10B5800001C001E0CE0109960E94968D002309F4C6
:10B5900073C026E030E044E050E06DE47CE0CE0192
:10B5A00001960E94E890BE016F5F7F4F85E39CE0AB
:10B5B0000E94888ECE0101960E94968D85E39CE0C4
:10B5C0000E9487916B017C0160E778E0CE010996CB
:10B5D0000E94018EBE01675F7F4F8DE49CE00E9458
:10B5E000DF90AC014F5F5F4F6DE47CE0CE010196D0
:10B5F0000E944909BE016F5F7F4F85E39CE00E9476
:10B60000888ECE0101960E94968DCE0109960E94E9
:10B61000968D0091E2041091E30485E39CE00E9482
:10B620009191AB01BC019801C6010E946A31E7E922
:10B63000FBE027E63BE04191519161917191D90185
:10B640004D935D936D937D939D01BBE0EF3BFB07B5
:10B6500091F71092C00B1092BF0B80E090E00E9417
:10B660007F0944E050E06DE47CE0CE0109960E9441
:10B67000490968EF79E03AC169E17AE0CE010996BB
:10B680000E94018EBE01675F7F4F8DE49CE00E94A7
:10B690004790811116C06DE17AE0CE0101960E94BB
:10B6A000018EBE016F5F7F4F8DE49CE00E9447904A
:10B6B00001E0811101C000E0CE0101960E94968D4B
:10B6C00001C001E0CE0109960E94968D002309F485
:10B6D00056C08091C2049091C3040E941B246093C1
:10B6E00016027093170280931802909319026093C8
:10B6F000310B7093320B8093330B9093340B80E0BB
:10B7000090E5A3ECB7E480931E0290931F02A093F0
:10B710002002B09321028093290B90932A0BA093CF
:10B720002B0BB0932C0B65E37BE08AEF9EE00E942D
:10B730001B8A409116025091170260911802709175
:10B74000190222E030E08AEF9EE00E94708C109295
:10B75000C00B1092BF0B80E090E00E947F094091E7
:10B76000160250911702609118027091190222E09E
:10B77000CE0109960E94238F61E27AE0B7C06CE2A5
:10B780007AE0CE0109960E94018EBE01675F7F4F6D
:10B790008DE49CE00E944790811116C060E37AE03E
:10B7A000CE0101960E94018EBE016F5F7F4F8DE436
:10B7B0009CE00E94479001E0811101C000E0CE01B1
:10B7C00001960E94968D01C001E0CE0109960E946B
:10B7D000968D002309F4B1C08091510C9091520CC8
:10B7E0000497F8F044E050E06DE47CE0CE0101966F
:10B7F0000E944909BE016F5F7F4F85E39CE00E9474
:10B80000888ECE0101960E94968D85E39CE00E9471
:10B81000919160932202709323028093240290936B
:10B8200025028091220290912302A0912402B091DE
:10B8300025028093250B9093260BA093270BB093A2
:10B84000280B6DE17BE08AEF9EE00E941B8A40910D
:10B85000220250912302609124027091250222E07D
:10B8600030E08AEF9EE00E946F8C8091C20490913C
:10B87000C3040E941B2460931A0270931B028093DE
:10B880001C0290931D0260932D0B70932E0B8093DE
:10B890002F0B9093300B63E17BE08AEF9EE00E94D8
:10B8A0001B8A40911A0250911B0260911C027091F8
:10B8B0001D0222E030E08AEF9EE00E94708C109220
:10B8C000C00B1092BF0B80E090E00E947F09409176
:10B8D0001A0250911B0260911C0270911D0222E01D
:10B8E000CE0109960E94238F64E37AE0CE0101968F
:10B8F0000E94018EBE01675F7F4FCE0101960E94BC
:10B90000FA8FBC018BE39CE00E946B8ECE01019606
:10B910000E94968DCE0109960E94968D6BE37CE085
:10B92000CE0101960E94808ECE0101960E94A20F48
:10B93000CE0101960E94968DE4C06CE37AE0CE01C0
:10B9400009960E94018EBE01675F7F4F8DE49CE0E7
:10B950000E944790811116C060E47AE0CE01019602
:10B960000E94018EBE016F5F7F4F8DE49CE00E94BC
:10B97000479001E0811101C000E0CE0101960E94D4
:10B98000968D01C001E0CE0109960E94968D00239C
:10B9900009F484C08091510C9091520C0497F8F0F6
:10B9A00044E050E06DE47CE0CE0101960E9449093C
:10B9B000BE016F5F7F4F85E39CE00E94888ECE01C1
:10B9C00001960E94968D85E39CE00E949191609380
:10B9D0001E0270931F028093200290932102809197
:10B9E0001E0290911F02A0912002B091210280932B
:10B9F000290B90932A0BA0932B0BB0932C0B6BEF7E
:10BA00007AE08AEF9EE00E941B8A40911E025091CC
:10BA10001F02609120027091210222E030E08AEF43
:10BA20009EE00E946F8C8091C2049091C3040E949A
:10BA30001B24609316027093170280931802909350
:10BA400019026093310B7093320B8093330B9093F8
:10BA5000340B61EF7AE08AEF9EE00E941B8A4091EE
:10BA6000160250911702609118027091190222E09B
:10BA700030E08AEF9EE00E94708C1092C00B109212
:10BA8000BF0B80E090E00E947F0940911602509128
:10BA90001702609118027091190221CF112389F1C8
:10BAA0006CE277E0CE0101960E94018E6DE47CE0AD
:10BAB000CE0101960E94FA8FBC018AEF9EE00E949F
:10BAC000678ACE0101960E94968D1BC087EB9CE091
:10BAD0000E94D283182F8823F9F069EC7AE087E47A
:10BAE0009CE00E949E8E64E47AE08AEF9EE00E94D1
:10BAF0004C8A612F8AEF9EE00E94878A812F0E94E4
:10BB0000A6480E943C846093530C7093540C80931D
:10BB1000550C9093560C49C080912C0C882309F445
:10BB20004FC00E943C84F8EECF2EF3E0DF2EE12CD4
:10BB3000F12CA70196010E941B96CA01B9010E942F
:10BB400042932091930B3091940B4091950B50911F
:10BB5000960B0E94AD9120910E0230910F02409100
:10BB60001002509111020E94199418164CF50E946F
:10BB70003C84A70196010E941B96CA01B9010E944C
:10BB800042936093930B7093940B8093950B9093D7
:10BB9000960B8091290C90912A0C0E94A84664E192
:10BBA00070E080E090E00E946B8480912C0C8823F0
:10BBB000E9F064E670E080E090E00E946B8416C0DB
:10BBC0000E943C84C090530CD090540CE090550CD3
:10BBD000F090560C6C197D098E099F0968347E4ED1
:10BBE0008105910510F30E94742EDFCFA6960FB643
:10BBF000F894DEBF0FBECDBFDF91CF911F910F91A3
:10BC0000FF90EF90DF90CF90BF90AF909F908F907C
:10BC100008952DE43AE0FC013183208308952DE45A
:10BC20003AE0FC01318320830C94AB910F931F9376
:10BC3000CF93DF938C01EB0188E2FB0111928A958F
:10BC4000E9F74BE050E067E57AE0CE010E944799C2
:10BC50001B8641E050E060E070E04C875D876E87B6
:10BC60007F87F801458956896789708D488B598B84
:10BC70006A8B7B8B42E050E060E070E04C8B5D8B28
:10BC80006E8B7F8B1CA21DA21EA21FA240E050E063
:10BC900068E474E4488F598F6A8F7B8F40E050E0EE
:10BCA00068E474EC4C8F5D8F6E8F7F8F4DEC5CEC95
:10BCB0006CE47EE348A359A36AA37BA3DF91CF91F1
:10BCC0001F910F91089523E63AE0FC013183208310
:10BCD000458B568B678B708F0895CF93DF931F92A0
:10BCE0001F92CDB7DEB781E39EE02A8349830E948D
:10BCF0009C754981642F81E39EE00E9455752A81DD
:10BD0000622F81E39EE00E94557581E39EE00F90D3
:10BD10000F90DF91CF910C941A760F931F93CF93CE
:10BD2000DF938C01EB01262F41E06EE1D6DFF801B5
:10BD3000D483C383C038D10509F45BC0DCF4C034BC
:10BD4000D105A9F1C036D10509F442C0A09709F088
:10BD50008AC080E090E8A9E8B4E48093FD04909361
:10BD6000FE04A093FF04B093000580E090E0A5E7F7
:10BD7000B4E471C0C03CD10509F44CC0C03ED1054B
:10BD800009F459C0C03AD10509F06DC080E090E0D7
:10BD9000A8ECB3E48093FD049093FE04A093FF0409
:10BDA000B093000580E090E0AFE7B3E454C080E0DA
:10BDB00090ECA5E5B4E48093FD049093FE04A09379
:10BDC000FF04B093000580E090E0AEE3B4E443C02C
:10BDD00080E090E8A7E2B4E48093FD049093FE0431
:10BDE000A093FF04B093000580E090E0A6E1B4E4E6
:10BDF00032C080E090E0A1EEB3E48093FD04909324
:10BE0000FE04A093FF04B093000580E090E0A8EC4E
:10BE1000B3E421C080E090E0A5EAB3E48093FD04A0
:10BE20009093FE04A093FF04B093000580E090E897
:10BE3000A3E9B3E410C080E090E0A6E6B3E4809309
:10BE4000FD049093FE04A093FF04B093000580E0EE
:10BE500090E0ADE4B3E48093F9049093FA04A093E6
:10BE6000FB04B093FC04DF91CF911F910F910895D3
:10BE7000CF93DF93EC0181E39EE00E94937520E075
:10BE800042E06EE1CE0129DF60E270E0CE0145DFE5
:10BE900081E0DF91CF9108956F927F928F929F9270
:10BEA000AF92BF92CF92DF92EF92FF920F931F93C8
:10BEB000CF93DF93EC016EE181E39EE00E949C75DD
:10BEC000E091310EF091320E0190F081E02D63E0AF
:10BED00081E39EE0199581E39EE00E941A7646E098
:10BEE0006EE181E39EE00E94167681E39EE00E946F
:10BEF000FE740697D4F381E39EE00E940675682ED7
:10BF000081E39EE00E940675782E81E39EE00E9408
:10BF10000675C82E81E39EE00E940675D82E81E347
:10BF20009EE00E940675882E81E39EE00E940675C1
:10BF3000982EB62CA12CA728B501882777FD8095CF
:10BF4000982F0E9444936D837E838F839887F82C6B
:10BF5000E12CE928B701882777FD8095982F0E946A
:10BF6000449369877A878B879C871C2D00E00D2975
:10BF7000B801882777FD8095982F0E9444936D879C
:10BF80007E878F87988B198A1A8A1B8A1C8ADF9171
:10BF9000CF911F910F91FF90EF90DF90CF90BF90C6
:10BFA000AF909F908F907F906F900895CF92DF9287
:10BFB000EF92FF920F931F93CF93DF938C01EB01CE
:10BFC00084E2FB0111928A95E9F7C80165DF84E2FA
:10BFD00090E0A0E0B0E088839983AA83BB83F80156
:10BFE00085899689A789B08D8C839D83AE83BF8315
:10BFF00082E090E0A0E0B0E088879987AA87BB87BD
:10C00000188A198A1A8A1B8AC090FD04D090FE04EF
:10C01000E090FF04F0900005A7019601658176810C
:10C02000878190850E94789220E030E048EC52E4CD
:10C030000E94D8946C8B7D8B8E8B9F8BA701960171
:10C04000F80161857285838594850E94789220E04D
:10C0500030E048EC52E40E94D894688F798F8A8F40
:10C060009B8F2091F9043091FA044091FB04509188
:10C07000FC04F80165857685878590890E94789211
:10C0800020E030E048EC52E40E94D8946C8F7D8F21
:10C090008E8F9F8F81E0DF91CF911F910F91FF9045
:10C0A000EF90DF90CF900895FC0181E080831182B2
:10C0B00043EC5BEA66E77BE34283538364837583E7
:10C0C00048ED5BE666E77BE34683578360877187CD
:10C0D00042EF54EE64E67BE34287538764877587BB
:10C0E0000895FC01DB014D915D916D917C91139759
:10C0F000428353836483758314964D915D916D9152
:10C100007C911797468357836087718718964D9166
:10C110005D916D917C911B974287538764877587EA
:10C120000895CF93DF93FC01EB0142815381648139
:10C130007581488359836A837B83468157816085F3
:10C1400071854C835D836E837F8382859385A4850F
:10C15000B58588879987AA87BB87DF91CF91089596
:10C160000F931F93CF93DF93082F69E276E08AEF56
:10C170009EE00E944C8AC7E0D0E010E0B8010C2E8F
:10C1800002C0759567950A94E2F76170772742E0DF
:10C1900050E08AEF9EE00E94368B219778F7DF917E
:10C1A000CF911F910F9108951F93CF93DF931F920B
:10C1B000CDB7DEB7162F63E570E081E39EE04983DB
:10C1C0000E94A675612F81E39EE00E94557549810A
:10C1D000642F81E39EE00E94557581E39EE00F90FD
:10C1E000DF91CF911F910C941A76CF93DF93EC01DE
:10C1F00081E39EE00E94937540E06DE2CE01D4DFC2
:10C2000040E16DE2CE01D0DF48E06DE2CE01DF918A
:10C21000CF91CACF6F3F710534F4AB0177FF05C0F2
:10C2200040E050E002C04FEF50E06DE1BDCFEF9233
:10C23000FF921F93CF93DF931F92CDB7DEB77C01A0
:10C24000142F462F6EE12983AFDF412F6FE1C70125
:10C25000ABDF2981422F60E2C7010F90DF91CF91C0
:10C260001F91FF90EF90A0CF6F3F710534F4AB01A9
:10C2700077FF05C040E050E002C04FEF50E061E2C0
:10C2800093CF462F62E290CF6F3F710534F4AB013C
:10C2900077FF05C040E050E002C04FEF50E063E29E
:10C2A00083CF6F3F710534F4AB0177FF05C040E0E9
:10C2B00050E002C04FEF50E064E276CF6F3F71056F
:10C2C00034F4AB0177FF05C040E050E002C04FEF0F
:10C2D00050E065E269CF6F3F710534F4AB0177FF41
:10C2E00005C040E050E002C04FEF50E066E25CCF96
:10C2F0006F3F710534F4AB0177FF05C040E050E0BB
:10C3000002C04FEF50E068E24FCF6F3F710534F449
:10C31000AB0177FF05C040E050E002C04FEF50E0B6
:10C3200069E242CFAF92BF92CF92DF92EF92FF923B
:10C330000F931F93CF93DF938C01C62F7A0169016E
:10C3400063E570E081E39EE00E94A6756C2F81E3B7
:10C350009EE00E94557581E39EE00E941A7663E597
:10C3600070E081E39EE00E94A675A70163E570E09E
:10C3700081E39EE00E941876E6015E01AC18BD08DC
:10C3800081E39EE00E94FE74892B31F081E39EE000
:10C390000E9406758993F1CFAE14BF0421F0F80115
:10C3A000108281E0818381E39EE0DF91CF911F9134
:10C3B0000F91FF90EF90DF90CF90BF90AF900C94D3
:10C3C0001A76CF92DF92EF92FF920F931F93CF9343
:10C3D000DF93EC016B017A0189019C01225F3F4FE1
:10C3E00046E050E062E39EDF8F8590E0982F88273B
:10C3F0002E85822BF60191838083898990E0982F86
:10C4000088272889822BF701918380838B8990E08C
:10C41000982F88272A89822BF80191838083DF91C6
:10C42000CF911F910F91FF90EF90DF90CF900895E3
:10C430009B012C5F3F4FAB014E5F5F4FC2CFAF926E
:10C44000BF92CF92DF92EF92FF920F931F93CF9301
:10C45000DF9300D000D0CDB7DEB77C015B01BE0119
:10C460006F5F7F4FE5DFCE0101966C01870175019B
:10C470005E0197E0A90EB11CF601619171916F0107
:10C48000882777FD8095982F0E944493F801228198
:10C490003381448155810E94D894F701619371934F
:10C4A000819391937F010C5F1F4FCA14DB0421F726
:10C4B00026960FB6F894DEBF0FBECDBFDF91CF91A9
:10C4C0001F910F91FF90EF90DF90CF90BF90AF90B2
:10C4D0000895CF93DF931F92CDB7DEB79E012F5FF4
:10C4E0003F4F41E050E06DE11DDF898190E00F900A
:10C4F000DF91CF910895AF92BF92CF92DF92EF92EA
:10C50000FF920F931F93CF93DF931F92CDB7DEB7A8
:10C510008C015B016A0179019E012F5F3F4F41E071
:10C5200050E06EE1FFDE898190E0F5019183808328
:10C530009E012F5F3F4F41E050E06FE1C801F2DE06
:10C54000898190E0F601918380839E012F5F3F4FA8
:10C5500041E050E060E2C801E5DE898190E0F7014A
:10C56000918380830F90DF91CF911F910F91FF9066
:10C57000EF90DF90CF90BF90AF900895CF93DF936F
:10C580001F92CDB7DEB79E012F5F3F4F41E050E0D5
:10C5900061E2C8DE898190E00F90DF91CF9108952C
:10C5A000CF93DF931F92CDB7DEB79E012F5F3F4F32
:10C5B00041E050E062E2B6DE898190E00F90DF91C9
:10C5C000CF910895CF93DF931F92CDB7DEB79E0131
:10C5D0002F5F3F4F41E050E063E2A4DE898190E0AD
:10C5E0000F90DF91CF910895CF93DF931F92CDB736
:10C5F000DEB79E012F5F3F4F41E050E064E292DEE4
:10C60000898190E00F90DF91CF910895CF93DF93D0
:10C610001F92CDB7DEB79E012F5F3F4F41E050E044
:10C6200065E280DE898190E00F90DF91CF910895DF
:10C63000CF93DF931F92CDB7DEB79E012F5F3F4FA1
:10C6400041E050E066E26EDE898190E00F90DF917C
:10C65000CF910895CF93DF931F92CDB7DEB79E01A0
:10C660002F5F3F4F41E050E068E25CDE898190E05F
:10C670000F90DF91CF910895CF93DF931F92CDB7A5
:10C68000DEB79E012F5F3F4F41E050E069E24ADE96
:10C69000898190E00F90DF91CF910895CF93DF9340
:10C6A0001F92CDB7DEB79E012F5F3F4F41E050E0B4
:10C6B0006CE238DE69816F7070E06650710988271E
:10C6C00077FD8095982F0E9444939B01AC0160E018
:10C6D00070E080E090E40E943B9520E030E048EC80
:10C6E00050E40E94D8940F90DF91CF910895EF927B
:10C6F000FF920F931F93CF93DF931F92CDB7DEB7B7
:10C700008C01CB01BA0120E030E048EC50E40E94FB
:10C7100078920E941193E12CF12C75956795611523
:10C72000710521F08FEFE81AF80AF7CF8AE0E816D2
:10C73000F10484F49E012F5F3F4F41E050E06CE232
:10C74000C801F0DD46E04E0D8981807F482B6CE208
:10C75000C8012ADD0F90DF91CF911F910F91FF90BB
:10C76000EF900895CF93DF931F92CDB7DEB79E0170
:10C770002F5F3F4F41E050E060E3D4DD89810F90AF
:10C78000DF91CF910895DF92EF92FF920F931F9365
:10C79000CF93DF931F92CDB7DEB78C01F62EE42E38
:10C7A000D22E9E012F5F3F4F41E050E0BBDD8981DB
:10C7B00021E030E00E2C01C0220F0A94EAF7DD20C0
:10C7C00011F0282B02C020952823298349816F2D41
:10C7D000C801EADC0F90DF91CF911F910F91FF907C
:10C7E000EF90DF900895262F47E050E061E3CBCF34
:10C7F000262F46E050E067E2C6CF262F45E050E006
:10C8000067E2C1CF262F44E050E067E2BCCF262F7D
:10C8100042E050E067E2B7CF262F41E050E067E208
:10C82000B2CF262F40E050E067E2ADCF262F47E0A1
:10C8300050E067E2A8CF262F43E050E067E2A3CFA5
:10C84000262F43E050E06AE29ECF262F42E050E0E0
:10C850006AE299CF262F41E050E06AE294CF262F7A
:10C8600040E050E06AE28FCF262F44E050E06CE2D7
:10C870008ACF242F462F50E06FE285CF242F462FFA
:10C8800050E06EE280CF1F93CF93DF931F92CDB71E
:10C89000DEB7142F9E012F5F3F4F41E050E042DD95
:10C8A000898190E002C0959587951A95E2F781708D
:10C8B0000F90DF91CF911F91089547E050E061E321
:10C8C000E2CF46E050E067E2DECF45E050E067E2CD
:10C8D000DACF44E050E067E2D6CF42E050E067E2D2
:10C8E000D2CF41E050E067E2CECF40E050E067E2D7
:10C8F000CACF43E050E067E2C6CF43E050E06AE2CF
:10C90000C2CF42E050E06AE2BECF41E050E06AE2CE
:10C91000BACF40E050E06AE2B6CF46E050E06BE2CA
:10C92000B2CF45E050E06BE2AECF44E050E06BE2C6
:10C93000AACF42E050E06BE2A6CF41E050E06BE2CC
:10C94000A2CF40E050E06BE29ECF43E050E06BE2CC
:10C950009ACF44E050E06CE296CF462F50E060E37F
:10C9600092CF462F50E06FE28ECF462F50E06EE21E
:10C970008ACFEF92FF920F931F93CF93DF931F9273
:10C98000CDB7DEB77C016DE67AE08AEF9EE00E94CB
:10C990004C8A9E012F5F3F4F41E050E060E0C701AD
:10C9A000C1DC8981DDDB69EC7AE08AEF9EE00E94E0
:10C9B000778A0DE110E064E77AE08AEF9EE00E945A
:10C9C0004C8A40E150E0B8018AEF9EE00E94368B2D
:10C9D00069EC79E08AEF9EE00E944C8A9E012F5F0D
:10C9E0003F4F41E050E0602FC7019CDC8981B8DBFC
:10C9F00069EC7AE08AEF9EE00E94778A0F5F1F4F12
:10CA00000A331105C1F60F90DF91CF911F910F915D
:10CA1000FF90EF900895CF92DF92EF92FF92CF9325
:10CA2000DF93EC01882777FD8095982F0E9444932F
:10CA30006B017C0120E030E040E45FE30E94D89489
:10CA400020E030E048E452E40E9478920E94119382
:10CA5000C617D707ECF020E030E040EA5FE3C701FB
:10CA6000B6010E94D89420E030E048E452E40E94ED
:10CA7000789220E030E040E85FE30E94AE910E94AF
:10CA8000119321E06C177D070CF420E0822F01C088
:10CA900080E090E0DF91CF91FF90EF90DF90CF901A
:10CAA0000895CF92DF92EF92FF92CF93DF93EC0144
:10CAB0006C597F4F882777FD8095982F0E9444936B
:10CAC0006B017C0120E030E040E45FE30E94D894F9
:10CAD00020E030E048E452E40E9478920E941193F2
:10CAE000C617D707ECF020E030E040EA5FE3C7016B
:10CAF000B6010E94D89420E030E048E452E40E945D
:10CB0000789220E030E040E85FE30E94AE910E941E
:10CB1000119321E06C177D070CF420E0822F01C0F7
:10CB200080E090E0DF91CF91FF90EF90DF90CF9089
:10CB30000895CF92DF92EF92FF92CF93DF93EC01B3
:10CB400064567109882777FD8095982F0E94449339
:10CB50006B017C0120E030E040E45FE30E94D89468
:10CB600020E030E048E452E40E9478920E94119361
:10CB7000C617D707ECF020E030E040EA5FE3C701DA
:10CB8000B6010E94D89420E030E048E452E40E94CC
:10CB9000789220E030E040E85FE30E94AE910E948E
:10CBA000119321E06C177D070CF420E0822F01C067
:10CBB00080E090E0DF91CF91FF90EF90DF90CF90F9
:10CBC00008951F920F920FB60F9211240BB60F9279
:10CBD0002F933F934F935F936F937F938F939F9385
:10CBE000AF93BF93EF93FF938091610D0E94E8850F
:10CBF0002091640D3091650D2F5F3F4F3093650D8F
:10CC00002093640D9091630D953618F096E0909303
:10CC1000600D9091600D9430C9F128F4923069F064
:10CC20009330D1F05EC0953009F451C0963009F0D0
:10CC300058C091E09093300E51C0811152C02091A4
:10CC4000640D3091650D2436310508F442C0109210
:10CC5000300E1092630D1CC0813009F042C0E0918B
:10CC6000630D91E09E0F9093630DF0E02091640DB1
:10CC70003091650DEE0FFF1FEA59F24F318320838B
:10CC80001092650D1092640D94E029C0811117C0B7
:10CC9000E091630D91E09E0F9093630DF0E0209181
:10CCA000640D3091650DEE0FFF1FEA59F24F31838D
:10CCB00020831092650D1092640D93E010C02091B6
:10CCC000640D3091650D2536310558F007C081118E
:10CCD00008C01092650D1092640D03C095E090930A
:10CCE000600D9091620D992329F0811102C02F9A55
:10CCF00001C02F98FF91EF91BF91AF919F918F91BC
:10CD00007F916F915F914F913F912F910F900BBE4B
:10CD10000F900FBE0F901F9018956093610D1092A9
:10CD2000620D0895F89482E08093B0008093B10082
:10CD300094E69093B3001092B200809370007894C0
:10CD40008093600D1092630D8091610D60E00C94F2
:10CD50007A8582E08093600D1092630D08958F9222
:10CD60009F92AF92BF92CF92DF92EF92FF927B01A0
:10CD7000BA0180E090E00E9442934B015C01B70150
:10CD800080E090E00E9442936B017C012DEC3CEC32
:10CD90004CE45FE30E94D8949B01AC01C501B4014F
:10CDA0000E94749287FD17C02DEC3CEC4CE45FE3CD
:10CDB000C501B4010E94D8949B01AC01C701B60122
:10CDC0000E947492992787FD90958827990F881F54
:10CDD0009927019602C080E090E0FF90EF90DF90ED
:10CDE000CF90BF90AF909F908F9008958F929F9219
:10CDF000AF92BF92CF92DF92EF92FF920F931F9369
:10CE0000CF93DF936C01EB01EC84FD8486E0E816A0
:10CE1000F1040CF443C0EE0CFF1C06E010E045ECFE
:10CE2000842E4DE9942E4CE1A42E41E8B42E8A853F
:10CE30009B85FC01E00FF11F40815181F80134977F
:10CE4000E80FF91F60817181C60189DFFC01A5012E
:10CE5000940163E971E080E091E00E94E5954F0163
:10CE6000AA2497FCA094BA2C86269726A826B92631
:10CE70000E5F1F4F0E151F05D1F68C829D82AE826C
:10CE8000BF8280E290E0998788878FEF9FEF998338
:10CE9000888361E070E080E090E003C060E070E0D3
:10CEA000CB01DF91CF911F910F91FF90EF90DF9019
:10CEB000CF90BF90AF909F908F9008950F931F9346
:10CEC000CF93DF938C01EB0186E69DE09B878A87F9
:10CED0008091630D90E09D878C878091300E90E06B
:10CEE0009F878E878091600D853009F051C0C80101
:10CEF0001BD3882319F081E090E04CC0BE01C8012B
:10CF0000B0D78111F8CFBE01C80107D78111F3CF87
:10CF1000BE01C8017ED28111EECFBE01C801CCD4C2
:10CF20008111E9CFBE01C80169D58111E4CFBE01ED
:10CF3000C80192D38111DFCFBE01C801E3D18111B5
:10CF4000DACFBE01C8012DD18111D5CFBE01C801F4
:10CF500045D68111D0CFBE01C8010E94CC6F81118E
:10CF6000CACFBE01C8011BD08111C5CFBE01C80107
:10CF7000A2D08111C0CFBE01C80138DF672B682B5A
:10CF8000692B09F0B8CF82E08093600D1092630D99
:10CF900080E090E0DF91CF911F910F910895AF92C3
:10CFA000BF92CF92DF92EF92FF920F931F93CF9396
:10CFB000DF93EB018091630D883510F480E070C041
:10CFC000EA85FB858281938160E672E26ADD892BC6
:10CFD000A9F3EA85FB858481958164E971E1A9DD86
:10CFE000892B61F3BEE1CB2ED12C1DE1E12EF12C7A
:10CFF00000E010E08091630D90E00497E816F906D8
:10D00000ACF5EA85FB85C701880F991FE80FF91F6A
:10D010008081918164EF71E044DD892B79F25601C2
:10D02000AA0CBB1CEA85FB85EA0DFB1D8081918162
:10D0300068E572E07EDD892B21F0000F111F016091
:10D040000DC0EA85FB85EA0DFB1D8081918164EAB4
:10D0500076E06FDD892B49F0000F111F82E0E80EAA
:10D06000F11C82E0C80ED11CC5CF760181E0E81A20
:10D07000F108F594E794F986E8868AE2E816F10467
:10D080000CF49CCFC801AA2797FDA095BA2F8C83DA
:10D090009D83AE83BF8389E090E09983888381E09C
:10D0A000DF91CF911F910F91FF90EF90DF90CF9084
:10D0B000BF90AF900895AF92BF92CF92DF92EF9260
:10D0C000FF920F931F93CF93DF93EB018091630D3A
:10D0D000803211F080E05AC0EA85FB85828193811D
:10D0E0006CE271E0DEDC892BA9F3EA85FB858481A3
:10D0F00095816EEE72E01DDD892B61F306E010E094
:10D10000C12CD12C7601EA85FB85E00FF11F8081CF
:10D1100091816CE271E0C5DC892BE1F2580182E07B
:10D12000A80EB11CEA85FB85EA0DFB1D808191816B
:10D1300068E077E0FEDC892B39F0CC0CDD1CEE1CBE
:10D14000FF1C6894C0F810C0EA85FB85EA0DFB1D42
:10D15000808191816EEE72E0ECDC892B09F4BACF0C
:10D16000CC0CDD1CEE1CFF1C0C5F1F4F0E33110599
:10D1700051F68EE090E099878887CC82DD82EE823E
:10D18000FF828FE090E09983888381E0DF91CF91E7
:10D190001F910F91FF90EF90DF90CF90BF90AF90D5
:10D1A0000895AF92BF92CF92DF92EF92FF920F93CA
:10D1B0001F93CF93DF93EB018091630D823251F582
:10D1C000EA85FB858281938168E572E06ADC892BC0
:10D1D00009F18091630D90E081509048880F991F6C
:10D1E000EA85FB85E80FF91F8081918168E572E08F
:10D1F00058DC892B79F0198618868FEF9FEFDC01B8
:10D200008C839D83AE83BF8386E090E0998388837F
:10D2100081E06DC0EA85FB858281938160E47FE1D6
:10D2200040DC892B21F08091630D813210F480E085
:10D230005EC0EA85FB858481958160EA7FE079DCC8
:10D24000892BA9F358E0A52EB12C03E010E0C12CE6
:10D25000D12C7601EA85FB85C801880F991FE80F5C
:10D26000F91F8081918168E572E01BDC892BF9F25E
:10D27000EA85FB85EA0DFB1D8081918160E476E003
:10D2800058DC892B39F0CC0CDD1CEE1CFF1C68949B
:10D29000C0F810C0EA85FB85EA0DFB1D80819181F5
:10D2A00066E272E046DC892B09F4C1CFCC0CDD1CB0
:10D2B000EE1CFF1C0E5F1F4F84E0A80EB11C033252
:10D2C000110541F6EA85FB85EA5BFF4F808191817C
:10D2D00068E572E0E6DB892B09F4A9CF80E190E0F4
:10D2E00099878887CC82DD82EE82FF828DCFDF91A5
:10D2F000CF911F910F91FF90EF90DF90CF90BF9053
:10D30000AF900895AF92BF92CF92DF92EF92FF92CB
:10D310000F931F93CF93DF93EB018091630D8933BC
:10D3200010F480E06BC0EA85FB858281938160E424
:10D330007FE1B7DB892BA9F3EA85FB8584819581A1
:10D3400060EA7FE0F6DB892B61F338E0A32EB12C95
:10D3500003E010E0C12CD12C7601EA85FB85C801E1
:10D36000880F991FE80FF91F8081918168E572E0AD
:10D3700098DB892BB1F2EA85FB85EA0DFB1D8081E4
:10D38000918160E476E0D5DB892B39F0CC0CDD1C93
:10D39000EE1CFF1C6894C0F810C0EA85FB85EA0DFE
:10D3A000FB1D8081918166E272E0C3DB892B09F469
:10D3B000B8CFCC0CDD1CEE1CFF1C0E5F1F4F84E0B1
:10D3C000A80EB11C0B33110541F6EA85FB85EA581E
:10D3D000FF4F8081918168E572E063DB892B09F45E
:10D3E000A0CF8CE190E099878887CC82DD82EE82A5
:10D3F000FF828AE090E09983888381E0DF91CF917A
:10D400001F910F91FF90EF90DF90CF90BF90AF9062
:10D4100008956F927F928F929F92AF92BF92CF9218
:10D42000DF92EF92FF920F931F93CF93DF93EB0165
:10D430008091630D823208F45DC0EA85FB858281AC
:10D4400093816EE571E02DDB892B09F453C063E015
:10D45000A62EB12C02E010E0C12CD12C76013501B2
:10D460008091630D90E0A816B906CCF54801880CB0
:10D47000991CEA85FB85E80DF91D808191816EE993
:10D4800077E00FDB892B39F0CC0CDD1CEE1CFF1C88
:10D490006894C0F80FC0EA85FB85E80DF91D80810E
:10D4A00091816EEE72E0FDDA892B21F1CC0CDD1C4E
:10D4B000EE1CFF1CC501880F991FEA85FB85E80F4C
:10D4C000F91F808191816EE571E033DB22E0A20ECD
:10D4D000B11C892B19F00E5F1F4FC1CF8301015082
:10D4E000110915950795198708870031110524F44E
:10D4F0001986188680E009C0CC82DD82EE82FF8228
:10D500008CE090E09983888381E0DF91CF911F9137
:10D510000F91FF90EF90DF90CF90BF90AF909F90D2
:10D520008F907F906F900895AF92BF92CF92DF92CD
:10D53000EF92FF920F931F93CF93DF93EB01EA8556
:10D54000FB858281938168E273E2ABDA892B11F467
:10D5500080E077C08091630D843009F5EA85FB8512
:10D56000848195816AEC78E0E4DA892BC1F0EA8560
:10D57000FB858681978160E372E093DA892B79F0ED
:10D58000198618868FEF9FEFDC018C839D83AE8315
:10D59000BF8383E090E09983888381E052C08091CB
:10D5A000630D8434A8F2EA85FB858481958164E962
:10D5B00071E1BFDA892B61F206E010E0C12CD12CB9
:10D5C0007601EA85FB85E00FF11F8081918160E3A0
:10D5D00072E067DA892B09F4BBCF580182E0A80E0C
:10D5E000B11CEA85FB85EA0DFB1D808191816AE90A
:10D5F00076E09FDA892B39F0CC0CDD1CEE1CFF1C89
:10D600006894C0F810C0EA85FB85EA0DFB1D808197
:10D61000918160E372E08DDA892B09F499CFCC0C0B
:10D62000DD1CEE1CFF1C0C5F1F4F0638110549F670
:10D6300080E290E099878887CC82DD82EE82FF824B
:10D64000A8CFDF91CF911F910F91FF90EF90DF90C6
:10D65000CF90BF90AF9008958F929F92AF92BF925C
:10D66000CF92DF92EF92FF920F931F93CF93DF93AE
:10D6700000D01F92CDB7DEB74B01DB011A96ED91BA
:10D68000FC911B97828193816EEA7DE00ADA892BF7
:10D6900011F480E08FC0D4011A96ED91FC911B9794
:10D6A0008481958166ED76E0FCD9892B91F3E6E0E3
:10D6B000EE2EF12C20E030E040E050E0A12CB12C27
:10D6C000C12CD12CD4011A96ED91FC911B97EE0D33
:10D6D000FF1D8081918166EF71E029833A834B833E
:10D6E0005C83DFD9892BA9F287010E5F1F4FD4011C
:10D6F0001A96ED91FC911B97E00FF11F80819181AB
:10D700006CED74E016DA29813A814B815C81892BBA
:10D7100039F0B501C60101E00E94739621601CC07A
:10D72000D4011A96ED91FC911B97E00FF11F8081B7
:10D73000918160E971E029833A834B835C83F9D955
:10D7400029813A814B815C81892B09F4A2CFB501F3
:10D75000C60101E00E9473965B016C01B4E0EB0E20
:10D76000F11CE6ECEE16F10409F0ACCFD4011496EE
:10D770002C93149715963C93159716964C931697E1
:10D7800017965C931797B501C60100E20E948E962A
:10D7900012962C93129713963C93139785E090E082
:10D7A00011969C938E9380E390E019969C938E93B0
:10D7B000189781E00F900F900F900F90DF91CF910D
:10D7C0001F910F91FF90EF90DF90CF90BF90AF909F
:10D7D0009F908F9008958F929F92AF92BF92CF9219
:10D7E000DF92EF92FF920F931F93CF93DF937A0113
:10D7F0006901DA01CD91DC91FB0184859585C8171B
:10D80000D9070CF047C0CE01880F991F0284F38519
:10D81000E02DE80FF91FA080B180C170DD27F1E095
:10D82000CF27209719F484E690E002C08CE99FEF9F
:10D830004801880E991EB401C501EDD8892B89F4E1
:10D84000800E911EB401C501E6D8892B69F4B4019C
:10D85000600F711FC501DFD8892BF9F023E030E09C
:10D8600005C021E030E002C022E030E0D6018D9119
:10D870009C91119701968217930744F0F60111824B
:10D880001082D7018D919C91119701968D939C9355
:10D89000CE0105C081E090E002C08FEF9FEFDF91E5
:10D8A000CF911F910F91FF90EF90DF90CF90BF909D
:10D8B000AF909F908F9008954F925F926F927F925A
:10D8C0008F929F92AF92BF92CF92DF92EF92FF9290
:10D8D0000F931F93CF93DF9300D01F92CDB7DEB786
:10D8E0006C017B011C821B8281E090E09A8389831A
:10D8F0008091630D8D3010F480E06BC009E713E078
:10D900009E012D5F3F4FAE014F5F5F4FC60163DF4A
:10D91000892B91F79E012D5F3F4FAE014F5F5F4F07
:10D92000B701C60158DF019739F79E012D5F3F4FC0
:10D93000AE014F5F5F4FB701C6014DDF892BE1F6A6
:10D94000412C512C3201A12CB12C8091630D90E01F
:10D9500029813A81281739078CF509E713E09E01E0
:10D960002D5F3F4FAE014F5F5F4FB701C60133DF01
:10D970004C019E012D5F3F4FAE014F5F5F4FB701DE
:10D98000C60129DF21E08216910451F4892B09F0A8
:10D99000B3CF440C551C661C771C689440F80AC031
:10D9A000892809F0A9CF019709F0A6CF440C551C8E
:10D9B000661C771C8FEFA81AB80AC7CFF701B1868B
:10D9C000A086448255826682778281E090E09183CE
:10D9D00080830F900F900F900F90DF91CF911F9148
:10D9E0000F91FF90EF90DF90CF90BF90AF909F90FE
:10D9F0008F907F906F905F904F9008952F923F92FD
:10DA00004F925F926F927F928F929F92AF92BF924E
:10DA1000CF92DF92EF92FF920F931F93CF93DF93FA
:10DA200000D01F92CDB7DEB76C017B011C821B8238
:10DA3000DB011C968D919C911D971816190614F008
:10DA400080E0B5C0DB011A96ED91FC911B9782E056
:10DA500090E09A838983828193816AE67AE021D873
:10DA6000892B71F3D7011A96ED91FC911B9789814F
:10DA70009A819C012F5F3F4F3A832983880F991F1A
:10DA8000E80FF91F8081918169E773E052D8892BF3
:10DA9000B9F20CEB11E09E012D5F3F4FAE014F5FDD
:10DAA0005F4FB701C60197DE892B51F69E012D5FAE
:10DAB0003F4FAE014F5F5F4FB701C6018CDE01974C
:10DAC00009F0BECF212C312C2101A12CB12C2981B0
:10DAD0003A81F70184859585281739070CF05CC0D9
:10DAE0000CEB11E09E012D5F3F4FAE014F5F5F4F8A
:10DAF000B701C60170DE3C01B3E0AB16B10489F09A
:10DB00000CEB11E09E012D5F3F4FAE014F5F5F4F69
:10DB1000B701C60160DE4C01E3E0AE16B104F9F4D2
:10DB20000FC00CEB11E09E012D5F3F4FAE014F5F28
:10DB30005F4FB701C6014FDE6816790609F380CF43
:10DB40000CEB11E09E012D5F3F4FAE014F5F5F4F29
:10DB5000B701C60140DE8816990609F071CF61143D
:10DB6000710459F48A94892809F06ACF220C331C75
:10DB7000441C551C689420F80BC06A94672809F06F
:10DB80005FCF892809F05CCF220C331C441C551C44
:10DB9000AFEFAA1ABA0A9BCFB186A086248235823B
:10DBA0004682578282E090E09183808381E00F90EB
:10DBB0000F900F900F90DF91CF911F910F91FF90D9
:10DBC000EF90DF90CF90BF90AF909F908F907F901D
:10DBD0006F905F904F903F902F900895AF92BF92BB
:10DBE000CF92DF92EF92FF920F931F93CF93DF9329
:10DBF000EB01EA85FB858281938168E873E10E94ED
:10DC00005165892B11F480E07DC08091630D8430D3
:10DC100019F5EA85FB85848195816AEC78E00E949C
:10DC20009965892BC9F0EA85FB858681978160E338
:10DC300072E00E945165892B79F0198618868FEF62
:10DC40009FEFDC018C839D83AE83BF8387E090E0F0
:10DC50009983888381E056C08091630D843498F263
:10DC6000EA85FB858481958168E873E10E94996566
:10DC7000892B49F206E010E0C12CD12C7601EA850F
:10DC8000FB85E00FF11F8081918160E372E00E94CB
:10DC90005165892B09F4B7CF580182E0A80EB11C59
:10DCA000EA85FB85EA0DFB1D8081918160E476E0C9
:10DCB0000E949965892B39F0CC0CDD1CEE1CFF1CF1
:10DCC0006894C0F811C0EA85FB85EA0DFB1D8081D0
:10DCD000918160E372E00E949965892B09F493CFEA
:10DCE000CC0CDD1CEE1CFF1C0C5F1F4F0638110511
:10DCF00031F680E290E099878887CC82DD82EE82DF
:10DD0000FF82A4CFDF91CF911F910F91FF90EF90F1
:10DD1000DF90CF90BF90AF9008958F929F92AF9277
:10DD2000BF92CF92DF92EF92FF920F931F93CF9308
:10DD3000DF93EB018091630D8A3108F47AC0EA85A4
:10DD4000FB85808191818032934050F4198618863A
:10DD50008FEF9FEFDC018C839D83AE83BF836FC009
:10DD6000828193816CEA7DE00E945165892B09F4E0
:10DD700060C0EA85FB85848195816CEA7DE00E9424
:10DD80005165892B09F455C054E0A52EB12C03E050
:10DD900010E0C12CD12C76018091630D90E0A81683
:10DDA000B906E4F5EA85FB85C801880F991FE80FDD
:10DDB000F91F8081918166EB73E00E949965892B40
:10DDC00061F14501880C991CEA85FB85E80DF91D78
:10DDD0008081918160E679E00E945165892B39F05C
:10DDE000CC0CDD1CEE1CFF1C6894C0F810C0EA854A
:10DDF000FB85E80DF91D808191816CEB72E00E943A
:10DE00005165892BB1F0CC0CDD1CEE1CFF1C0E5FA4
:10DE10001F4F82E0A80EB11CBFCF85010150110930
:10DE200015950795198708870C30110524F4198674
:10DE3000188680E009C0CC82DD82EE82FF828BE012
:10DE400090E09983888381E0DF91CF911F910F91BA
:10DE5000FF90EF90DF90CF90BF90AF909F908F900A
:10DE600008958F929F92AF92BF92CF92DF92EF92DE
:10DE7000FF920F931F93CF93DF93EB018091630D7C
:10DE80008A3108F471C0EA85FB8580819181843FE5
:10DE9000914060F4198618868FEF9FEFDC018C8328
:10DEA0009D83AE83BF838BE090E066C082819381C7
:10DEB00060E679E00E945165892B09F455C073E052
:10DEC000A72EB12C02E010E0C12CD12C760180915C
:10DED000630D90E0A816B906E4F5EA85FB85C80154
:10DEE000880F991FE80FF91F8081918168E572E022
:10DEF0000E949965892B61F14501880C991CEA857E
:10DF0000FB85E80DF91D8081918160EB74E00E9432
:10DF10005165892B39F0CC0CDD1CEE1CFF1C68947C
:10DF2000C0F810C0EA85FB85E80DF91D808191815C
:10DF300068E572E00E945165892BB1F0CC0CDD1CC4
:10DF4000EE1CFF1C0E5F1F4F82E0A80EB11CBFCF5E
:10DF500085010150110915950795198708870C301F
:10DF6000110524F41986188680E009C0CC82DD8270
:10DF7000EE82FF8284E090E09983888381E0DF91E4
:10DF8000CF911F910F91FF90EF90DF90CF90BF90B6
:10DF9000AF909F908F900895AF92BF92CF92DF92F3
:10DFA000EF92FF920F931F93CF93DF93EB0180913A
:10DFB000630D863410F480E086C0EA85FB8582819B
:10DFC00093816EEE72E00E945165892BA1F3EA8580
:10DFD000FB85848195816EEE72E00E949965892BA4
:10DFE00051F3EA85FB858681978162E27BE00E949E
:10DFF0005165892B01F3EA85FB858085918562E275
:10E000007BE00E949965892BB1F25CE0A52EB12CD2
:10E0100005E010E0C12CD12C7601EA85FB85C80112
:10E02000880F991FE80FF91F808191816EEE72E0D1
:10E030000E945165892B09F4BECFEA85FB85EA0D64
:10E04000FB1D8081918166E678E00E949965892BAD
:10E0500039F0CC0CDD1CEE1CFF1C6894C0F811C01C
:10E06000EA85FB85EA0DFB1D808191816EEE72E0F1
:10E070000E949965892B09F49ECFCC0CDD1CEE1C07
:10E08000FF1C0E5F1F4F84E0A80EB11C0534110564
:10E0900021F6EA85FB85E657FF4F808191816EEE80
:10E0A00072E00E945165892B09F485CF80E290E0EF
:10E0B00099878887CC82DD82EE82FF8288E090E0BB
:10E0C0009983888381E0DF91CF911F910F91FF9019
:10E0D000EF90DF90CF90BF90AF9008953F924F9216
:10E0E0005F926F927F928F929F92AF92BF92CF92E8
:10E0F000DF92EF92FF920F931F93CF93DF9300D0A5
:10E100001F921F92CDB7DEB75C01562E19821A827C
:10E110001B821C821D8261E0852D0E947A8560E051
:10E12000852D0E94B38562E170E080E090E00E945E
:10E130006B8461E0852D0E94B38588E290E00E94A7
:10E14000918460E0852D0E947A8501E117E2852D9A
:10E150000E94E885892B31F401501109C1F78EEF37
:10E160009FEF6EC001E117E2852D0E94E8850197BF
:10E1700021F401501109C1F7F2CF08E210E0312C6F
:10E1800037E0432E88248394912C21E1E22E27E26C
:10E19000F22E852D0E94E885892B29F481E0E81A6A
:10E1A000F108B9F7DCCF0E9448846B017C0191E152
:10E1B000692E97E2792E852D0E94E885019729F432
:10E1C000E1E06E1A7108B9F7CACF0E9448846C1951
:10E1D0007D098E099F09693271058105910578F0E5
:10E1E000E1E0F0E0EC0FFD1FE30DF11D2081C40123
:10E1F000042C01C0880F0A94EAF7282B20834110D1
:10E2000004C0339487E0482E01C04A94015011099C
:10E2100009F0BBCF2981822F90E0F50191838083A3
:10E220003B81832F90E093838283230F81E090E0F2
:10E230003D81321302C080E090E091958195910973
:10E240000F900F900F900F900F90DF91CF911F9133
:10E250000F91FF90EF90DF90CF90BF90AF909F9085
:10E260008F907F906F905F904F903F900895FB014B
:10E270008081883251F028F4803139F0823239F4CB
:10E2800004C08B3311F0823411F481E0089580E0F2
:10E290000895FC017783668314821582108289E0D9
:10E2A000818381E0828383830895CF93DF93EC01A0
:10E2B000F0DF1B8A1A8ADF91CF910895FC018581D6
:10E2C0000895CF93DF93EB0167E0CE010E94D980E0
:10E2D00091E02F81821390E0892FDF91CF910895F3
:10E2E000EF92FF920F931F93CF93DF93EC018B017B
:10E2F000E42E8E819F810E940E80F12C41E0B801B6
:10E300008E819F810E944180882351F0FE1005C0BC
:10E31000B801CE01D6DF811104C0F394EF1470F779
:10E3200080E0DF91CF911F910F91FF90EF900895C2
:10E33000CF92DF92EF92FF920F931F93CF93DF93D1
:10E340001F921F92CDB7DEB76C01F42EE52EFC01B3
:10E350008681978169837A830E94F67E69817A81BA
:10E36000882311F1F601868197810E94E57F40E0C4
:10E370006EEBF601868197810E94897F0F2D1E2DFD
:10E3800089E0F82EF601868197810E94CA7FF80104
:10E3900081938F01FA94B1F7F601868197810E94EB
:10E3A000F67E91E0813009F090E0892F0F900F9078
:10E3B000DF91CF911F910F91FF90EF90DF90CF9061
:10E3C0000895CF93DF93EA01B3DF882351F068E02B
:10E3D000CE010E94D98091E02885821390E0892F98
:10E3E00001C080E0DF91CF910895EF92FF920F93EB
:10E3F0001F93CF93DF93EC018B017A018E819F8174
:10E400000E94F67EB8018E819F810E94E57F40E0E8
:10E410006EE48E819F810E94897F40E0F7016281D6
:10E420008E819F810E94897F40E0F70163818E8108
:10E430009F810E94897FF8018081803139F040E01E
:10E44000F70164818E819F810E94897F8E819F81E7
:10E450000E94F67EB8018E819F810E94E57F4881EF
:10E4600068E48E819F810E94897F64E170E080E092
:10E4700090E00E946B848881882331F06AE070E02C
:10E4800080E090E00E946B848E819F81DF91CF912C
:10E490001F910F91FF90EF900C94F67EEF92FF92F8
:10E4A0001F93CF93DF931F921F92CDB7DEB77C01EE
:10E4B000FC018681978169837A830E94F67E698157
:10E4C0007A81F701868197810E94E57F40E064EBC5
:10E4D000F701868197810E94897FF7018681978164
:10E4E0000E94617F182FF701868197810E94F67E36
:10E4F00081E0111180E00F900F90DF91CF911F917B
:10E50000FF90EF900895CF93DF93CDB7DEB72997B3
:10E510000FB6F894DEBF0FBECDBFFB0120812031C6
:10E52000C9F0AE014F5F5F4F4CDF882379F08D81DA
:10E530008F3351F020F48F3149F489E00CC08F35CE
:10E5400039F08F3739F002C08AE005C080E003C09F
:10E550008BE001C08CE029960FB6F894DEBF0FBEA9
:10E56000CDBFDF91CF910895FF920F931F93CF936B
:10E57000DF93CDB7DEB728970FB6F894DEBF0FBE96
:10E58000CDBF8C01FC01868197810E940E80F8012D
:10E590001482158241E0BE016F5F7F4FF8018681D2
:10E5A00097810E9441808823C1F1BE016F5F7F4F38
:10E5B000C80187DE882371F3F8018081811107C0CB
:10E5C000BE016F5F7F4FC80169DF811122C0F80172
:10E5D000F180BE016F5F7F4FC80195DF8F1518F482
:10E5E000F801818105C0BE016F5F7F4FC8018BDFDD
:10E5F000F801818384818F5F8483BE016F5F7F4FC9
:10E60000C80135DE882331F2F80185818F5F85836B
:10E61000C1CF81E0F8018083DACF28960FB6F89455
:10E62000DEBF0FBECDBFDF91CF911F910F91FF9045
:10E630000895DF92EF92FF920F931F93CF93DF9392
:10E64000CDB7DEB762970FB6F894DEBF0FBECDBF71
:10E650008C017B01D22E493028F0342F4D3018F038
:10E660003CE001C039E0B701C8013A8B4CDF3A8980
:10E67000831709F458C0AE014F5F5F4FB701C8015F
:10E680003A8B9FDE3A89882309F44FC0F7018081D5
:10E69000803109F448C03B3041F03C3021F03A3041
:10E6A00031F48FE305C08FE703C08FE501C08FE130
:10E6B0008D83AE014F5F5F4FB701C8013A8B95DE86
:10E6C000F80191813A89832F391708F4892FF801CD
:10E6D0008183D11028C0381730F53183E12CF12C1B
:10E6E000F801848190E0E816F906ECF44E2DBE01A5
:10E6F000665F7F4FC801F4DDF801D180BE01665F1F
:10E700007F4FC80100DF8D1518F4F801818105C025
:10E71000BE01665F7F4FC801F6DEF8018183FFEF1F
:10E72000EF1AFF0ADDCF81E001C080E062960FB6EC
:10E73000F894DEBF0FBECDBFDF91CF911F910F9137
:10E74000FF90EF90DF900895EF92FF920F931F9349
:10E75000CF93DF93CDB7DEB728970FB6F894DEBF1F
:10E760000FBECDBF8C01693020F06D3018F06CE029
:10E7700001C069E0F8016183E12CF12CF80184818A
:10E7800090E0E816F90694F44E2DBE016F5F7F4FBE
:10E79000C801A6DD21E0F8014181BE016F5F7F4F16
:10E7A000C80147DFFFEFEF1AFF0AE8CF28960FB640
:10E7B000F894DEBF0FBECDBFDF91CF911F910F91B7
:10E7C000FF90EF900895FC01868197810E94617F00
:10E7D00091E0813009F090E0892F08958F929F9207
:10E7E000AF92BF92CF92DF92EF92FF920F931F935F
:10E7F000CF93DF93EC016950633048F4E62FF0E0EB
:10E80000EE0FFF1FE958F54F0081118102C00EEE97
:10E8100012E08B818823E1F08881811119C00E9468
:10E820003C846B017C014801AA2497FCA094BA2C7B
:10E83000CE01C9DF81111FC00E943C84681979098B
:10E840008A099B096C157D058E059F05A0F4F0CF04
:10E85000B801882777FD8095982FDF91CF911F9180
:10E860000F91FF90EF90DF90CF90BF90AF909F906F
:10E870008F900C946B84DF91CF911F910F91FF903B
:10E88000EF90DF90CF90BF90AF909F908F900895C2
:10E89000CF93DF93EC018E819F810E94F67E8E8163
:10E8A0009F810E940B80488164E48E819F810E9439
:10E8B000897F8A81882329F06981CE01DF91CF91F8
:10E8C0008DCFDF91CF910895FA01208148E0249FF8
:10E8D00090011124818190E0982F8827990F990F3A
:10E8E000990F282B392BDB018C918031C1F4678182
:10E8F00070E08681AB01481B5109CA019695982F9B
:10E900008827979587950E94089660517109207F06
:10E9100053E0220F331F5A95E1F7260F371FC90125
:10E920000895EF92FF920F931F93CF93DF93CDB78C
:10E93000DEB729970FB6F894DEBF0FBECDBF8C01AE
:10E940007B01AE014F5F5F4F3CDD882339F0AE01A4
:10E950004F5F5F4FB701C801B7DF02C080E894EE98
:10E9600029960FB6F894DEBF0FBECDBFDF91CF91D1
:10E970001F910F91FF90EF900895813824EE920738
:10E980006CF0BC01882777FD8095982F0E944493F6
:10E9900020E030E040E05CE30C94D89460E070E06C
:10E9A0008EEF92EC0895BDDFE8CF0F931F93CF93C6
:10E9B000DF93CDB7DEB728970FB6F894DEBF0FBE52
:10E9C000CDBF8C01462FBE016F5F7F4F89DC88234E
:10E9D00031F0BE016F5F7F4FC801E5DF04C060E02A
:10E9E00070E08EEF92EC28960FB6F894DEBF0FBE63
:10E9F000CDBFDF91CF911F910F9108958091610E4E
:10EA000090E02091620E821B910908952091620E80
:10EA10008091610E281750F4E22FF0E0ED59F14F8C
:10EA2000808190E02F5F2093620E08958FEF9FEF1B
:10EA30000895E091620E8091610EE81730F4F0E0E5
:10EA4000ED59F14F808190E008958FEF9FEF089589
:10EA50000895CF92DF92EF92FF920F931F93CF937F
:10EA6000DF937C01CB018A0120913D0E222389F0A6
:10EA7000EB016B01C40ED51ECC15DD0561F069916B
:10EA8000D701ED91FC910190F081E02DC70119951E
:10EA9000F3CF642F91D1C801DF91CF911F910F91D6
:10EAA000FF90EF90DF90CF900895CF93DF931F9268
:10EAB000CDB7DEB7698320913D0E2223D1F020919E
:10EAC0003E0E203240F021E030E0FC01338322830F
:10EAD00080E090E014C080913F0EE82FF0E0E05C11
:10EAE000F14F998190838F5F80933F0E80933E0E0C
:10EAF00004C061E0CE0101965FD181E090E00F900B
:10EB0000DF91CF910895FC011382128248EE53E009
:10EB100060E070E0448355836683778381E89AE000
:10EB20009183808308951092620E1092610E10926C
:10EB30003F0E10923E0E83C081E080933D0E6093A5
:10EB4000600E10923F0E10923E0E0895F5CF0F9377
:10EB5000062F21E040913E0E60E47EE08091600E41
:10EB6000D4D010923F0E10923E0E10923D0E0F9197
:10EB700008958F929F92AF92BF92CF92DF92EF92C1
:10EB8000FF920F931F93CF93DF93EC01F62ED42EB9
:10EB900048015901EE2009F1CFDF1E2D143008F095
:10EBA00013E01150B8F0E881F98128E0129FB0011C
:10EBB0001124A501940104C05695479537952795D2
:10EBC0006A95D2F7CA01B9010190F081E02DCE011A
:10EBD0001995E7CF60E0CE01BADF4D2D413208F044
:10EBE00040E22C2D63E67EE08F2D47D01092620E1E
:10EBF0008093610EDF91CF911F910F91FF90EF9065
:10EC0000DF90CF90BF90AF909F908F900895CF925C
:10EC1000EF920F931F93C22EE12C00E010E09801B9
:10EC2000A8DF1F910F91EF90CF90089521E0EFCFD3
:10EC300021E0EDCF61E08BCF81E39EE064CF1092C5
:10EC4000F00E81E08093EE0E1092ED0E61E084E113
:10EC50000E94B38561E085E10E94B385E9EBF0E0B5
:10EC600080818E7F808380818D7F808388E4809304
:10EC7000B80085E48093BC000895413208F043C099
:10EC80009091F00E9111FCCF91E09093F00E2093B3
:10EC9000EE0E2FEF2093830E1092C80E240F2093B8
:10ECA000C70E9093EF0E9091EF0E880F892B8093F3
:10ECB000EF0E8091ED0E813061F41092ED0E809197
:10ECC000EF0E8093BB008091BC0083FDF8CF85ECF4
:10ECD00001C085EE8093BC008091F00E8130E1F39D
:10ECE0008091C80E841710F44091C80E29EC3EE0C4
:10ECF000FB01D9018A2F821B841718F48D9181930F
:10ED0000F9CF842F089580E008950F93413208F0E1
:10ED10004AC09091F00E9111FCCF92E09093F00ECA
:10ED20000093EE0E9FEF9093830E1092C80E4093C7
:10ED3000C70EFB0169EC7EE0DB019A2F961B94174E
:10ED400018F491919D93F9CF1092EF0E9091EF0EE0
:10ED5000880F892B8093EF0E8091ED0E813061F446
:10ED60001092ED0E8091EF0E8093BB008091BC005D
:10ED700083FDF8CF85EC01C085EE8093BC00222393
:10ED800021F08091F00E8230E1F38091830E8F3F6D
:10ED900061F08091830E803251F08091830E803338
:10EDA00041F483E007C081E005C080E003C082E059
:10EDB00001C084E00F910895613298F42091F00E23
:10EDC000243089F46093A50EFC0187EA9EE0DC0103
:10EDD0002A2F281B261718F421912D93F9CF80E0B4
:10EDE000089581E0089582E0089585ED8093BC0048
:10EDF0008091BC0084FDFCCF1092F00E089585EC4C
:10EE00008093BC001092F00E08951F920F920FB6DF
:10EE10000F9211240BB60F922F933F934F935F9352
:10EE20006F937F938F939F93AF93BF93EF93FF93D2
:10EE30008091B900887F803609F49DC070F58832D2
:10EE400009F45CC090F4803109F455C038F488238B
:10EE500009F4F3C0883009F44EC0F2C0883109F4D7
:10EE60004DC0803209F45EC0EBC0803409F469C043
:10EE700050F4803309F456C0883309F0E1C0809320
:10EE8000830EBDDFDDC0803509F44FC0883509F43D
:10EE90005DC0883409F0D4C0D2C0883909F4C3C039
:10EEA000A8F4883709F467C038F4883609F463C0D9
:10EEB000803709F460C0C4C0883809F4B4C0803910
:10EEC00009F45FC0803809F0BBC05BC0803B09F427
:10EED00082C038F4803A09F466C0883A09F47BC0ED
:10EEE000AFC0803C09F4A3C0883C09F4A0C0883BB3
:10EEF00009F486C0A5C08091EF0E10C09091C80E95
:10EF00008091C70E981770F5E091C80E81E08E0FC2
:10EF10008093C80EF0E0E753F14F80818093BB00EF
:10EF200085EC82C08093830E8AC0E091C80E81E098
:10EF30008E0F8093C80E8091BB00F0E0E753F14F35
:10EF400080839091C80E8091C70E6AC0E091C80E70
:10EF500081E08E0F8093C80E8091BB00F0E0E753F4
:10EF6000F14F80838091EE0E811169C081E0809322
:10EF7000ED0E84EA5DC083E08093F00E1092840E63
:10EF8000CFCF8091840E803208F04DC0E091840E86
:10EF900081E08E0F8093840E8091BB00F0E0EB57F0
:10EFA000F14F8083BDCF2BDF8091840E803230F40F
:10EFB000E091840EF0E0EB57F14F10826091840EE7
:10EFC00070E0E091E90EF091EA0E85E89EE0199577
:10EFD0001092840E35C084E08093F00E1092A60E3D
:10EFE0001092A50EE091EB0EF091EC0E1995809128
:10EFF000A50E811105C081E08093A50E1092A70E89
:10F00000E091A60E81E08E0F8093A60EF0E0E95508
:10F01000F14F80818093BB009091A60E8091A50E48
:10F02000981708F47DCF85E88093BC0009C085EC73
:10F030008093BC001092F00E03C01092830ED5DEB8
:10F04000FF91EF91BF91AF919F918F917F916F91C0
:10F050005F914F913F912F910F900BBE0F900FBE7C
:10F060000F901F90189508950895DC01ED91FC9183
:10F070000284F385E02D41E0199581E090E0089548
:10F08000FC011382128221E93AE031832083089542
:10F09000DC01ED91FC910084F185E02D6FEF199476
:10F0A000DC01ED91FC910284F385E02D40E01994A0
:10F0B00061E0F6DF80ED97E00C949184CF93DF93CD
:10F0C000CDB7DEB728970FB6F894DEBF0FBECDBF21
:10F0D0001D8220E42E8334E13F8334E53887198292
:10F0E0002A8320E12B8320E52C83FC012781421712
:10F0F00010F04FEF420FFC01308550E0FE01E40FAD
:10F10000F51F303121F4243011F4218101C0258113
:10F11000260F2068622F28960FB6F894DEBF0FBE28
:10F12000CDBFDF91CF91BCCFFC0165816B7F658343
:10F130006860B6CFFC016581262F246025836C6052
:10F14000AFCFCF93DF93EC01423018F08C81886011
:10F150008C834F836887222329F0413019F48C81F6
:10F1600084608C8364E670E080E090E00E946B84B1
:10F170006C8164FD31C0E881F9810284F385E02D62
:10F1800042E063E0CE01199584E991E10E94918407
:10F19000E881F9810284F385E02D42E063E0CE014D
:10F1A000199586E990E00E949184E881F9810284B2
:10F1B000F385E02D42E063E0CE01199586E990E009
:10F1C0000E949184E881F9810284F385E02D42E078
:10F1D00062E0CE01199513C06062CE0161DF84E95F
:10F1E00091E10E9491846C816062CE0159DF86E9D1
:10F1F00090E00E9491846C816062CE0151DF86E9CB
:10F2000090E00E9491846C816062CE0149DF8CE3C2
:10F2100090E00E94918484E08D83CE018BDFCE014B
:10F2200047DF82E08E8366E0CE013ADFCE01DF91D8
:10F23000CF912ECFCF92DF92FF920F931F93CF9358
:10F24000DF931F921F92CDB7DEB78C01677088E005
:10F25000689FB00111246064C80149835A8320DF8C
:10F260008EE190E00E9491844981C42E5A81D52E6E
:10F27000F12CD6016D916D01D801ED91FC910190B9
:10F28000F081E02DC801199588E290E00E949184F8
:10F29000F394B8E0FB12EDCF0F900F90DF91CF9178
:10F2A0001F910F91FF90DF90CF900895FC01868908
:10F2B0008F3F79F021853285662319F0232B31F4B5
:10F2C00003C02130310511F461E001C060E00C940D
:10F2D000B3850895FF920F931F93CF93DF93EC01B3
:10F2E000F62E8A0161E08F2D0E947A85FE8A1A87A8
:10F2F0000987E881F9810084F185E02D60E0CE0185
:10F30000DF91CF911F910F91FF9019946F927F928F
:10F310008F92AF92CF92EF92FF920F931F93CF9362
:10F32000DF93CDB7DEB73C01F62EFC01438724877F
:10F330000587E686C786A08A818A8F85828B888921
:10F34000838B8989848B8A89858B00E010E0F301A7
:10F35000E00FF11F61E086850E947A850F5F1F4FE5
:10F3600004301105A1F7FF2069F061E0F301838506
:10F370000E947A85F30184858F3F99F061E00E94B5
:10F380007A850FC000E010E0F301E00FF11F61E0AB
:10F3900082890E947A850F5F1F4F04301105A1F703
:10F3A000E4CF61E0F30185850E947A85FF2019F0A2
:10F3B000F301148203C080E1F301848360E0F30170
:10F3C00083850E94B38560E0F30185850E94B38543
:10F3D000F30184858F3F19F060E00E94B3858FEFC1
:10F3E000F301868B12861186DF91CF911F910F91C9
:10F3F000FF90EF90CF90AF908F907F906F90089597
:10F400006F927F928F92AF92CF92EF920F93CF93A2
:10F41000DF9300D0CDB7DEB73C012B834A836983ED
:10F420002FDE81EA9AE0F301918380831F921F927D
:10F430001F921F928C2CAE2CC02E2B81E22E4A8163
:10F44000042F2FEF6981462F61E0C3015FDF0F902A
:10F450000F900F900F900F900F900F90DF91CF9122
:10F460000F91EF90CF90AF908F907F906F90089515
:10F47000CF93DF93EC0161E08D850E94B38560E05E
:10F480008D85DF91CF910C94B385CF92DF92EF926F
:10F49000FF920F931F93CF93DF931F92CDB7DEB7E9
:10F4A0008C01C12CD12CE62EF12CC416A0F4B7018E
:10F4B0000C2C02C0759567950A94E2F76170F8010B
:10F4C000EC0DFD1D868549830E94B3858FEFC81A18
:10F4D000D80A4981EACFC8010F90DF91CF911F91DF
:10F4E0000F91FF90EF90DF90CF90C2CF0F931F93BB
:10F4F000CF93DF93EC01162F042F61E0413009F028
:10F5000060E08B850E94B3858C858F3F19F060E0A9
:10F510000E94B385023079F08C8184FF02C048E0FC
:10F520000BC0612F70E084E0759567958A95E1F7CF
:10F5300044E0CE01AADF44E0612FCE01DF91CF91FC
:10F540001F910F91A2CF0895CF92DF92EF92FF9279
:10F55000FC0185899689481B590B61097109A389AA
:10F56000B4899A01AB010E945F966B017C018FE028
:10F57000F594E794D794C7948A95D1F765857685F5
:10F58000882777FD8095982F2BE0660F771F881FBF
:10F59000991F2A95D1F727853089442737FD409553
:10F5A000542F2C0D3D1D4E1D5F1D0E943D962C0DB0
:10F5B0003D1D4E1D5F1DCA01B901FF90EF90DF9008
:10F5C000CF9008951F93CF93DF931F92CDB7DEB7EF
:10F5D000162F67E770E081E39EE04983B7DA612F79
:10F5E00081E39EE062DA4981642F81E39EE05DDA87
:10F5F00081E39EE00F90DF91CF911F911BCBCF93C2
:10F60000C62F67E770E081E39EE0A0DA6C2F81E30C
:10F610009EE04BDA81E39EE00DDB67E770E081E37B
:10F620009EE094DA41E050E067E770E081E39EE01D
:10F63000FFDA81E39EE0EAD9C82F81E39EE0FADA9F
:10F640008C2FCF910895CF93DF93C62F67E770E09B
:10F6500081E39EE07BDA6C2F81E39EE026DA81E392
:10F660009EE0E8DA67E770E081E39EE06FDA42E06F
:10F6700050E067E770E081E39EE0DADA81E39EE044
:10F68000C5D9D82F80E0C82F81E39EE0BFD9C82B11
:10F69000D92B81E39EE0CEDACE01DF91CF910895A0
:10F6A000CF93DF93EC01643008F063E0688381E37B
:10F6B0009EE039DA60EDCE01A2DF853509F039C070
:10F6C0006AEACE01C0DF9A8389836CEACE01BBDF90
:10F6D0009C838B836EEACE01B6DF9E838D8360EBC5
:10F6E000CE01B1DF9A8B898B62EBCE01ACDF9C8BB4
:10F6F0008B8B64EBCE01A7DF9E8B8D8B66EBCE01EF
:10F70000A2DF98878F8368EBCE019DDF9A87898778
:10F710006AEBCE0198DF9C878B876CEBCE0193DF81
:10F720009E878D876EEBCE018EDF988B8F8781E071
:10F7300001C080E0DF91CF910895CF93DF93EC017A
:10F740004EE264EF3FDF65E070E080E090E00E9411
:10F750006B8466EFCE01DF91CF9175CFCF93DF93AE
:10F76000EC01EBDFAC0160E070E0CE01EDDE685F44
:10F770007F4F8F4F9F4F34E095958795779567958D
:10F780003A95D1F70E94449320E030E040E251E402
:10F790000E947892DF91CF910895CF92DF92EF92FD
:10F7A000FF92CF93DF93EC0148814295440F440FC1
:10F7B000407C4C5C64EF06DF8881811105C065E008
:10F7C00070E080E090E012C0813029F468E070E0E1
:10F7D00080E090E00BC0823029F46EE070E080E0C1
:10F7E00090E004C06AE170E080E090E00E946B84E9
:10F7F00066EFCE0128DF6C01E12CF12CFE2CED2C04
:10F80000DC2CCC2468EFCE01FADEA7019601282B70
:10F81000CA01B901488128E030E0241B310904C045
:10F8200096958795779567952A95D2F7DF91CF9131
:10F83000FF90EF90DF90CF9008952F923F924F92DC
:10F840005F926F927F928F929F92AF92BF92CF9270
:10F85000DF92EF92FF920F931F93CF93DF93CDB779
:10F86000DEB72A970FB6F894DEBF0FBECDBF9A87DA
:10F87000898763DF8C0189859A858FDF6D837E831D
:10F880008F839887A80160E070E089859A855CDEA7
:10F890004B015C0180EA881A8FE0980AA108B10840
:10F8A000A5019401C501B4010E94E5952B013C011D
:10F8B0000CE075946794579447940A95D1F7A985FD
:10F8C000BA8511962D903C9012971C9115960D902B
:10F8D000BC91A02D0E9469966B017C018DE0F5948E
:10F8E000E794D794C7948A95D1F7E985FA85A781DB
:10F8F000B085A30192010E946996BB2797FDB09540
:10F90000AB2FC80ED91EEA1EFB1EF2E0CF0ED11C93
:10F91000E11CF11C32E0F594E794D794C7943A9532
:10F92000D1F780E8D80EE11CF11CE985FA85A189A0
:10F93000B289A70196010E945F96DC01CB014FE0DE
:10F94000B695A795979587954A95D1F789839A8318
:10F95000AB83BC836101EE24D7FCE094FE2C52E023
:10F96000CC0CDD1CEE1CFF1C5A95D1F7A185B2858D
:10F97000A30192010E9469962B013C016BE07594F2
:10F980006794579447946A95D1F7A381B481A501F0
:10F9900094010E946996EBE0959587957795679518
:10F9A000EA95D1F7460E571E681E791EC40CD51C69
:10F9B000E61CF71C012E04C0CC0CDD1CEE1CFF1C49
:10F9C0000A94D2F792E0C90ED11CE11CF11CC701C8
:10F9D000B60124E030E040E050E00E943D968D8189
:10F9E0009E81AF81B885821B930BA40BB50B9C0144
:10F9F000AD0160E573EC80E090E004C096958795DA
:10FA0000779567951A95D2F70E94E59597FD0DC0F9
:10FA1000660F771F881F991F29813A814B815C816E
:10FA20000E941B9649015A010CC029813A814B81E1
:10FA30005C810E941B9649015A01880C991CAA1CE2
:10FA4000BB1C9927B7FC9A958B2D7A2D692D9B01AC
:10FA5000AC010E94E5959B01AC01AEEDBBE00E94BC
:10FA60005F966C01FF24D7FCF094EF2CA3E4B3EE77
:10FA7000A50194010E946B96BB2797FDB095AB2F13
:10FA8000C80ED91EEA1EFB1E9FECC90E9EE0D91EB1
:10FA9000E11CF11CA4E0F594E794D794C794AA95CF
:10FAA000D1F7C80CD91CEA1CFB1CC701B6012A9669
:10FAB0000FB6F894DEBF0FBECDBFDF91CF911F917F
:10FAC0000F91FF90EF90DF90CF90BF90AF909F90FD
:10FAD0008F907F906F905F904F903F902F90089500
:10FAE0008F929F92AF92BF92CF92DF92EF92FF924E
:10FAF000CF93DF9300D01F92CDB7DEB74A015B01F1
:10FB00009CDE6B017C0120E03AE24DE257E4C50146
:10FB1000B4010E9478929B01AC0160E070E080E843
:10FB20009FE30E94AD9126EF38E248EA50E40E943C
:10FB30003B959B01AC01C701B60129833A834B83F6
:10FB40005C830E94449329813A814B815C810E94AD
:10FB500078920E9411930F900F900F900F90DF9169
:10FB6000CF91FF90EF90DF90CF90BF90AF909F909C
:10FB70008F900895CF93DF9300D01F92CDB7DEB75B
:10FB80009A01AB0129833A834B835C8356DE0E9442
:10FB9000449329813A814B815C810E94789221E0D3
:10FBA0003EED42E45EE30E943B959B01AC0160E0C8
:10FBB00070E080E89FE30E94AD9120E03AE24DE2E0
:10FBC00057E40E94D8940F900F900F900F90DF9100
:10FBD000CF910895FB016181828170E0762F6627C5
:10FBE000680F711D882777FD8095982F0E94449398
:10FBF00020E030E040E85DE30E94D89423E333E95D
:10FC000048E853E40C94AD91089521E06227FC018B
:10FC10008081A9C7CF93DF93EC01862F6883498346
:10FC20002A8361E067D761E088819DD760E08981A0
:10FC300061D760E08A815ED761E0898194D761E015
:10FC40008A8191D760E0CE01DF91CF91DECFFB01B9
:10FC500081819081890F9281890F9381981304C0CB
:10FC600081E094819D3009F080E008952F923F92C9
:10FC70004F925F926F927F928F929F92AF92BF92BC
:10FC8000CF92DF92EF92FF920F931F93CF93DF9368
:10FC900000D000D0CDB7DEB78C013B014E83ECD550
:10FCA0001B012C0180ED280E87E0381E411C511CE1
:10FCB00061E0C801AADFFE0131966F014E01F6E056
:10FCC0008F0E911CF60185E011928A95E9F7760175
:10FCD00027E0A22EB12CF80181817AD7019731F467
:10FCE000CBD56215730584059505A8F3F8018181CC
:10FCF0006FD7892B31F4C0D562157305840595053E
:10FD0000A8F3F801828164D7892B59F0F70120818B
:10FD100081E090E00A2C01C0880F0A94EAF7282BB2
:10FD20002083F1E0AF1AB108B0F69FEFE91AF90AA3
:10FD3000E814F90469F6A0D56215730584059505E4
:10FD400040F060E0C80161DF20E030E040EC5FE7B8
:10FD50002EC08981EE818E13B5CFB601C80177DF41
:10FD6000882309F4AFCF60E0C8014FDFB601C801B6
:10FD700031DFFB01DC016A946728B9F420E030E050
:10FD800040E151E4BF01CD010E94D89420E030E071
:10FD900040EA50E40E94789220E030E040E052E4F3
:10FDA0000E94AE919B01AC0102C09F01AD01B9015F
:10FDB000CA0126960FB6F894DEBF0FBECDBFDF9105
:10FDC000CF911F910F91FF90EF90DF90CF90BF9058
:10FDD000AF909F908F907F906F905F904F903F90EB
:10FDE0002F90089546E642CF4CE440CFFF920F9308
:10FDF0001F93CF93DF93FC010081C181D281F894DE
:10FE00008981F02EF0948F21898378941DE7115019
:10FE100009F182E090E085D588818023C1F3F894D0
:10FE20008A818F218A838981802B8983789480EECF
:10FE300091E077D5F89489818F21898386E490E0D9
:10FE400070D58881802311E009F010E078948AE968
:10FE500091E067D5812FDF91CF911F910F91FF9096
:10FE600008951F93CF93DF93FC011081C181D2814C
:10FE7000912F909560FF11C0F8948A8189238A831D
:10FE80008981812B89838AE090E04BD58A81812BFF
:10FE90008A83789487E390E010C0F8948A8189235C
:10FEA0008A838981812B898381E490E03AD58A8194
:10FEB000812B8A83789485E090E0DF91CF911F9128
:10FEC00030C50F931F93CF93DF93FC011081C18145
:10FED000D281F8948981812B89838A81012F0095B1
:10FEE00080238A8383E090E01CD5898180238983E5
:10FEF0008AE090E016D5C881789485E390E011D52A
:10FF00001C2381E009F480E0DF91CF911F910F91D4
:10FF10000895CF92DF92EF92FF920F931F93CF93AA
:10FF2000DF931F92CDB7DEB76C01E62E08E010E03C
:10FF3000FF24F39461E09F2D9E2109F460E0C60147
:10FF400049838FDFFF0C015011094981011511050B
:10FF500089F7411115C0F894D6011196ED91FC91E5
:10FF6000129791818C918095892381831196ED91CF
:10FF7000FC91129792818C91809589238283789449
:10FF80000F90DF91CF911F910F91FF90EF90DF9035
:10FF9000CF900895EF92FF920F931F93CF93DF932B
:10FFA0008C01C8E0D0E0F12CEE24E394C80189DF95
:10FFB0008111FE28EE0C2197C9F78F2DDF91CF918B
:10FFC0001F910F91FF90EF900895CF92DF92FF92D3
:10FFD0000F931F93CF93DF931F92CDB7DEB78C01A2
:10FFE000F62E40E065E5798394DFCF2C7981D72E1A
:10FFF00088E0F82EF60161916F0140E0C80189DFC9
:020000021000EC
:10000000FA94C1F70F90DF91CF911F910F91FF905C
:10001000DF90CF90089540E06CEC7BCFFC0113861D
:100020001586148627E030E0DF01A20FB31F139678
:100030001C922115310519F021503109F5CF089591
:100040001F93CF93DF93EC01162F60E0812F52D5E1
:10005000612F70E0FB01E254F34FE491E883FB0170
:10006000EC5FF24FE491F0E0EE0FFF1FE65BF24F22
:10007000859194919A838983CE01DF91CF911F91CD
:10008000CDCFAF92BF92CF92DF92EF92FF920F93BC
:100090001F93CF93DF931F92CDB7DEB75C01D62EAF
:1000A000E72EFC01158511115EC049839FDE498151
:1000B000811105C0F5011386158614866DC0442391
:1000C00019F040E060EF02C040E06CEEC50121DFB6
:1000D00001E0F12CC12C11E0C501F3DE682FC50150
:1000E0006983EFDE6981613019F48130B9F432C07F
:1000F0002F2D30E068131BC0F5018385181730F4ED
:10010000E20FF31F8381802349F402C0181731F0F6
:1001100060E0193058F4F501148708C0F501EF0DBF
:10012000F11D8381802B838361E009C0C12EF5011D
:10013000E20FF31F8381902F909589238383C5015C
:1001400090DE1F5F000F11F4F39401E0F7E0FF155C
:1001500008F0C2CF113438F0F501C386C11009C0D0
:1001600081E0858706C0F50113861586148610E0A8
:1001700013C0F50183818823B1F3ED2DFE2D80E0BE
:1001800090E0D501A80FB91F13962C9121930196E9
:1001900088309105B1F711E0812F0F90DF91CF9159
:1001A0001F910F91FF90EF90DF90CF90BF90AF9095
:1001B0000895DC0180E0615088F09D919827E92F37
:1001C000EF70F0E0E85AF34F249192959F70E92F79
:1001D000F0E0E859F34F84918227EDCF0895FC01B8
:1001E00010821482138215820895862F642F82C490
:1001F000862F642FB8C4862FEBC44F925F926F9204
:100200007F928F929F92AF92BF92CF92DF92EF92A6
:100210000F93CF93DF93EC014B013A015901029602
:10022000DEDF81EB9AE0998388836E018CE1C80E52
:10023000D11C26018CE3480E511CC601D0DF86E09C
:10024000C80ED11CC414D504C1F7FE01EE59FF4FEE
:10025000718260823296B182A0823296008331969A
:10026000E08237979182808238968AE090E091838D
:100270008083329684EF91E091838083339611825C
:10028000108271971082118212821382C459DF4F3B
:100290001882DF91CF910F91EF90DF90CF90BF90B8
:1002A000AF909F908F907F906F905F904F90089548
:1002B0002F923F924F925F926F927F928F929F9276
:1002C000AF92BF92CF92DF92EF92FF920F931F9364
:1002D000CF93DF93CDB7DEB728970FB6F894DEBF84
:1002E0000FBECDBF98878F83F12C4C0186E6880E18
:1002F000911C0F8118850E591F4FD4018C91F8164F
:10030000A0F4AF81B8858D919C91F801A081B18155
:10031000AF0DB11DFC012081318142E06C918F81D4
:100320009885F9011995F394E8CF512CEF81F88560
:10033000E959FF4FFA83E9830F8118850C591F4F44
:10034000C12CD12C7601C3948F8198858E599F4FF3
:100350009C838B83A981BA818C91581608F088C040
:10036000A52CB12CAF81B8858D919C91F801A0810D
:10037000B181AA0DBB1DFC012081318141E06C914E
:100380008F819885F9011995AF81B8858D919C91E0
:10039000F801A081B181AA0DBB1DFC01228133812E
:1003A00040E06C918F819885F9011995D701C601BC
:1003B000052C04C0880F991FAA1FBB1F0A94D2F7EF
:1003C0009C011C0120943094412CD4018C91EF812C
:1003D000F88540815181481648F5642C712CEB81D9
:1003E000FC81A081B181A60DB71DFA014481558120
:1003F0006C918F8198852D833E83FA011995660C47
:10040000771C2D813E81EF81F885E60DF71D892B44
:1004100029F480859185822B932B04C0808591855A
:1004200082219321918780874394CFCFF801A081C7
:10043000B181AA0DBB1DFA012281338141E06C918B
:100440008F819885F9011995AF81B8858D919C911F
:10045000F801A081B181AA0DBB1DFC012081318171
:1004600040E06C918F819885F9011995539472CF72
:1004700028960FB6F894DEBF0FBECDBFDF91CF91A7
:100480001F910F91FF90EF90DF90CF90BF90AF90B2
:100490009F908F907F906F905F904F903F902F90A4
:1004A0000895FC0180E090E0258D368D26173707F2
:1004B00039F0019636968A309105B1F78FEF9FEFAC
:1004C0000895DC0126E0629FA00DB11D11249096D5
:1004D0005C934E935F9721E091962C939197FC014A
:1004E000E459FF4F208131960190F081E02D2223C5
:1004F00031F0309749F0611107C0DC0102C030973C
:1005000019F05C968C9119940895CF92DF92FF9226
:100510000F931F93CF93DF931F92CDB7DEB76C017C
:10052000F62EFC0186E0689FE00DF11D112411A25A
:10053000878D90A181309105E1F01CF4892B51F059
:1005400042C08230910581F1039709F03CC040E040
:1005500050E02EC04423B9F141E050E0C601B1DFC4
:100560008BD1F601E85AFF4F6083718382839383B6
:100570002AC0498381D1F601E85AFF4F00811181D9
:1005800022813381601B710B820B930B7296008169
:10059000118120E030E04981061717072807390745
:1005A00018F442E050E004C041110DC043E050E0B7
:1005B0006F2DC6010F90DF91CF911F910F91FF908A
:1005C000DF90CF907ECF0F90DF91CF911F910F9151
:1005D000FF90DF90CF9008952F923F924F925F92BD
:1005E0006F927F928F929F92AF92BF92CF92DF9243
:1005F000EF92FF920F931F93CF93DF931F92CDB78C
:10060000DEB71C01FC014AE08FEF9FEF278D30A180
:10061000232B21F4148E968F858F11A2415036968C
:100620004111F4CF712C610126E6C20ED11C51019B
:1006300087E6A80EB11C4101A0E68A0E911C46E097
:10064000442ED6018C91781608F053C0612C81019C
:10065000070D111D070D111D085F1F4FF501E080EB
:100660006E1408F044C0F80140815181062C02C08C
:10067000569547950A94E2F741707E9C70011124CB
:10068000E60CF11CD401ED91FC91EE0DFF1D5080A4
:10069000B701C101498305DF498197FD02C0682F79
:1006A0001BC0019611F5442301F180E090E060E069
:1006B00070E0F101E80FF91F248D211110C0469E52
:1006C000F001479EF00D1124E20DF31D548EF68EBD
:1006D000E58E10A2178E41E0C10117DF06C06F5FE3
:1006E0007F4F06966A30710521F76394B7CF7394F4
:1006F000A8CF20E030E080E0F101E20FF31F91A1EC
:10070000911181E02A5F3F4F2C333105A9F70F90FB
:10071000DF91CF911F910F91FF90EF90DF90CF90DD
:10072000BF90AF909F908F907F906F905F904F9011
:100730003F902F900895CF92DF92EF92FF920F9308
:100740001F93CF93DF938C0197D0E801C45ADF4FFA
:10075000C880D980EA80FB806C197D098E099F09C9
:10076000F801E859FF4FC080D180E12CF12CC6166A
:10077000D706E806F90658F4C8019ADDC8012CDF4F
:10078000182F7AD0688379838A839B8301C010E015
:10079000812FDF91CF911F910F91FF90EF90DF900C
:1007A000CF9008950F931F93CF93DF93EC018C01AB
:1007B00004591F4F81E0F8018083CE01BCDF8823FC
:1007C00049F089A1882331F08F8D98A1019711F408
:1007D0008C8D03C0F801108280E0DF91CF911F91D2
:1007E0000F9108951F920F920FB60F9211242F931D
:1007F0003F938F939F93AF93BF938091F20E90910D
:10080000F30EA091F40EB091F50E3091F10E23E0AD
:10081000230F2D3720F40196A11DB11D05C026E838
:10082000230F0296A11DB11D2093F10E8093F20EAD
:100830009093F30EA093F40EB093F50E8091F60E04
:100840009091F70EA091F80EB091F90E0196A11DAE
:10085000B11D8093F60E9093F70EA093F80EB0930F
:10086000F90EBF91AF919F918F913F912F910F9072
:100870000FBE0F901F9018952FB7F8946091F20E4D
:100880007091F30E8091F40E9091F50E2FBF0895A4
:100890003FB7F8948091F60E9091F70EA091F80E64
:1008A000B091F90E26B5A89B05C02F3F19F001960F
:1008B000A11DB11D3FBF6627782F892F9A2F620F88
:1008C000711D811D911D42E0660F771F881F991FC2
:1008D0004A95D1F70895CF92DF92EF92FF92CF938E
:1008E000DF936B017C01D4DFEB01C114D104E1047F
:1008F000F10481F00E94AC91CBDF6C1B7D0B683E54
:10090000734098F381E0C81AD108E108F108C85192
:10091000DC4FEBCFDF91CF91FF90EF90DF90CF9046
:1009200008958230910538F0880F991F880F991F1C
:1009300005970197F1F70895789484B5826084BD96
:1009400084B5816084BD85B5826085BD85B58160D3
:1009500085BDEEE6F0E0808181608083E1E8F0E033
:100960001082808182608083808181608083E0E862
:10097000F0E0808181608083E1EBF0E08081846041
:100980008083E0EBF0E0808181608083E1E9F0E04A
:10099000808182608083808181608083E0E9F0E0F3
:1009A000808181608083E1EAF0E0808182608083E1
:1009B000808181608083E0EAF0E0808181608083D3
:1009C000E1E2F1E0808182608083808181608083C8
:1009D000E0E2F1E0808181608083EAE7F0E08081FD
:1009E0008460808380818260808380818160808355
:1009F0008081806880831092C100089580930105F2
:100A00000895863308F0865320917B00982F9870C4
:100A1000277F922B90937B0087702091010590E4B3
:100A2000299F90011124822B80937C0080917A0071
:100A3000806480937A0080917A0086FDFCCF80915B
:100A400078002091790090E0922B089590E0FC01CD
:100A50003197E231F10508F04CC0EB56FF4F0C9492
:100A60005996809180008F7703C0809180008F7DA0
:100A700080938000089580918000877FF9CF84B5AE
:100A80008F7702C084B58F7D84BD08958091B000BA
:100A90008F7703C08091B0008F7D8093B000089560
:100AA000809190008F7707C0809190008F7D03C068
:100AB00080919000877F8093900008958091A0009E
:100AC0008F7707C08091A0008F7D03C08091A00028
:100AD000877F8093A0000895809120018F7707C0C1
:100AE000809120018F7D03C080912001877F8093BA
:100AF00020010895CF93DF9390E0FC01E254F34F7F
:100B00002491FC01EC5FF24F8491882349F190E03D
:100B1000880F991FFC01E258F24FA591B4918C59AE
:100B2000924FFC01C591D4919FB7611108C0F89410
:100B30008C91209582238C93888182230AC0623015
:100B400051F4F8948C91322F309583238C938881C3
:100B5000822B888304C0F8948C91822B8C939FBF46
:100B6000DF91CF9108950F931F93CF93DF931F923F
:100B7000CDB7DEB7282F30E0F901E858F34F849164
:100B8000F901E254F34F1491F901EC5FF24F049133
:100B90000023C1F0882319F0698358DF6981E02FB1
:100BA000F0E0EE0FFF1FEC59F24FA591B4919FB703
:100BB000F8948C91611103C01095812301C0812BA1
:100BC0008C939FBF0F90DF91CF911F910F9108954C
:100BD000CF93DF93282F30E0F901E858F34F849149
:100BE000F901E254F34FD491F901EC5FF24FC49153
:100BF000CC2389F081112ADFEC2FF0E0EE0FFF1FEC
:100C0000E65BF24FA591B4912C912D2381E090E009
:100C100021F480E002C080E090E0DF91CF91089560
:100C20000F931F93762F90E0FC01E254F34F6491F1
:100C3000FC01EC5FF24FE4917111762FF0E0EE0FC2
:100C4000FF1FE65BF24F8591949189019A013F70F5
:100C5000472F0E949F07611571058105910531F0AD
:100C60006F5F7F4F8F4F9F4F9F7003C060E070E0BA
:100C7000CB011F910F910895FC01818D228D90E091
:100C8000805C9F4F821B91098F7399270895FC0107
:100C9000918D828D981731F0828DE80FF11D858D31
:100CA00090E008958FEF9FEF0895FC01918D828D64
:100CB000981761F0828DDF01A80FB11D5D968C91B0
:100CC000928D9F5F9F73928F90E008958FEF9FEFBB
:100CD00008958BE398E8892B39F080E090E0892B28
:100CE00019F0C9D1811123C080E090E0892B41F037
:100CF00080E090E0892B21F00E94000081111AC051
:100D000086EE98E8892B39F080E090E0892B19F085
:100D10005DD2811112C081E999E8892B99F080E0B8
:100D200090E0892B79F0FDD281110AC008950E94CC
:100D30000000DACF0E940000E3CF0E940000EBCF5A
:100D40000C9400000895FC01848DDF01A80FB11DF3
:100D5000A35ABF4F2C91848D90E001968F739927F1
:100D6000848FA689B7892C93A089B1898C918064DE
:100D70008C93938D848D981306C00288F389E02D9F
:100D800080818F7D80830895CF93DF93EC01888DE0
:100D90008823C1F0EA89FB89808185FD05C0A88987
:100DA000B9898C9186FD0EC00FB607FCF5CF808106
:100DB00085FFF2CFA889B9898C9185FFEDCFCE014F
:100DC000C2DFE8CFDF91CF910895CF92DF92FF92FB
:100DD0000F931F93CF93DF931F92CDB7DEB76C01B4
:100DE00081E0D60158968C9358975B969C915B97BF
:100DF0005C968C915C97981307C05096ED91FC918E
:100E00005197808185FD2DC0F601038D10E00F5FA5
:100E10001F4F0F731127F02EF601848DF81210C0AA
:100E20000FB607FCF9CFD6015096ED91FC91519782
:100E3000808185FFF1CFC601698385DF6981ECCFB1
:100E4000838DE80FF11DE35AFF4F6083D6015B9657
:100E50000C935B975296ED91FC9153978081806241
:100E60000CC0D6015696ED91FC9157976083509631
:100E7000ED91FC91519780818064808381E090E0C6
:100E80000F90DF91CF911F910F91FF90DF90CF9046
:100E90000895BF92CF92DF92EF92FF92CF93DF93AC
:100EA000EC016A017B01B22EE889F98982E0808336
:100EB000411581EE580761057105A1F060E079E008
:100EC0008DE390E0A70196010E941B962150310905
:100ED000410951095695479537952795211580E188
:100EE000380798F0E889F989108260E874E88EE1A3
:100EF00090E0A70196010E941B96215031094109FB
:100F000051095695479537952795EC85FD85308392
:100F1000EE85FF852083188EEC89FD89B082EA89F1
:100F2000FB89808180618083EA89FB898081886078
:100F30008083EA89FB89808180688083EA89FB89D4
:100F400080818F7D8083DF91CF91FF90EF90DF9044
:100F5000CF90BF900895CF93DF93EC01E881F981A2
:100F60000284F385E02D1995EA89FB8980818F7EC3
:100F70008083EA89FB898081877F8083EA89FB8976
:100F800080818F778083EA89FB8980818F7D808350
:100F90008A8D898FDF91CF910895FC01538D448D07
:100FA000252F30E0842F90E0821B930B541710F014
:100FB000CF960895019708951F920F920FB60F9242
:100FC00011240BB60F922F938F939F93EF93FF9360
:100FD000E0910A0FF0910B0F8081E091100FF091DA
:100FE000110F82FD12C090818091130F8F5F8F735C
:100FF0002091140F821751F0E091130FF0E0E650AA
:10100000F14F958F8093130F01C08081FF91EF9175
:101010009F918F912F910F900BBE0F900FBE0F904D
:101020001F9018951F920F920FB60F9211240BB6B6
:101030000F922F933F934F935F936F937F938F9371
:101040009F93AF93BF93EF93FF938AEF9EE07BDE76
:10105000FF91EF91BF91AF919F918F917F916F9190
:101060005F914F913F912F910F900BBE0F900FBE4C
:101070000F901F9018958AEF9EE0FEDD21E0892BEE
:1010800009F420E0822F08951092FD0E1092FC0EBC
:1010900088EE93E0A0E0B0E08093FE0E9093FF0E08
:1010A000A093000FB093010F8BEB9AE09093FB0E8F
:1010B0008093FA0E85EC90E09093070F8093060FD3
:1010C00084EC90E09093090F8093080F80EC90E0FF
:1010D00090930B0F80930A0F81EC90E090930D0F8B
:1010E00080930C0F82EC90E090930F0F80930E0F83
:1010F00086EC90E09093110F8093100F1092130FD5
:101100001092140F1092150F1092160F08951F923F
:101110000F920FB60F9211240BB60F922F938F934D
:101120009F93EF93FF93E091A70FF091A80F808119
:10113000E091AD0FF091AE0F82FD12C090818091D1
:10114000B00F8F5F8F732091B10F821751F0E09134
:10115000B00FF0E0E956F04F958F8093B00F01C0CB
:101160008081FF91EF919F918F912F910F900BBEF6
:101170000F900FBE0F901F9018951F920F920FB6F1
:101180000F9211240BB60F922F933F934F935F93BF
:101190006F937F938F939F93AF93BF93EF93FF933F
:1011A00087E99FE0D0DDFF91EF91BF91AF919F91D3
:1011B0008F917F916F915F914F913F912F910F9000
:1011C0000BBE0F900FBE0F901F90189587E99FE000
:1011D00053DD21E0892B09F420E0822F089510923D
:1011E0009A0F1092990F88EE93E0A0E0B0E0809300
:1011F0009B0F90939C0FA0939D0FB0939E0F8BEB32
:101200009AE09093980F8093970F85ED90E09093DC
:10121000A40F8093A30F84ED90E09093A60F80938A
:10122000A50F80ED90E09093A80F8093A70F81ED1C
:1012300090E09093AA0F8093A90F82ED90E0909395
:10124000AC0F8093AB0F86ED90E09093AE0F809340
:10125000AD0F1092B00F1092B10F1092B20F10920A
:10126000B30F08951F920F920FB60F9211240BB671
:101270000F922F938F939F93EF93FF93E0914410DE
:10128000F09145108081E0914A10F0914B1082FD61
:1012900012C0908180914D108F5F8F7320914E10FE
:1012A000821751F0E0914D10F0E0EC5CFF4E958F0D
:1012B00080934D1001C08081FF91EF919F918F919C
:1012C0002F910F900BBE0F900FBE0F901F9018958F
:1012D0001F920F920FB60F9211240BB60F922F93FD
:1012E0003F934F935F936F937F938F939F93AF93AE
:1012F000BF93EF93FF9384E390E125DDFF91EF919E
:10130000BF91AF919F918F917F916F915F914F911D
:101310003F912F910F900BBE0F900FBE0F901F901B
:10132000189584E390E1A8DC21E0892B09F420E002
:10133000822F0895109237101092361088EE93E0A5
:10134000A0E0B0E08093381090933910A0933A1049
:10135000B0933B108BEB9AE0909335108093341050
:1013600085E391E0909341108093401084E391E0F5
:10137000909343108093421080E391E09093451046
:101380008093441081E391E090934710809346103E
:1013900082E391E0909349108093481086E391E0B6
:1013A00090934B1080934A1010924D1010924E1053
:1013B00010924F10109250100895CF92DF92EF923A
:1013C000FF920F931F93CF93DF937C016A01EB0190
:1013D00000E010E00C151D0571F06991D701ED9149
:1013E000FC910190F081E02DC7011995892B19F02E
:1013F0000F5F1F4FEFCFC801DF91CF911F910F916A
:10140000FF90EF90DF90CF9008956115710581F006
:10141000DB010D900020E9F7AD0141505109461B59
:10142000570BDC01ED91FC910280F381E02D1994C2
:1014300080E090E00895EF92FF920F931F93CF9377
:10144000DF938C017B01C0E0D0E0F701EC0FFD1FC2
:101450006491662359F0F801A081B181ED91FC916E
:10146000C8011995892B11F02196EFCFCE01DF919C
:10147000CF911F910F91FF90EF900895DC01ED91B6
:10148000FC91DB0114964D915C9115976D917C91C7
:101490000280F381E02D1994B8CFDC01ED91FC912D
:1014A0000190F081E02D199467EC7AE0AECF0F93B4
:1014B0001F93CF93DF93EC01BEDF8C01CE01F4DFED
:1014C000800F911FDF91CF911F910F9108950F937E
:1014D0001F93CF93DF93EC01D1DF8C01CE01E4DFCA
:1014E000800F911FDF91CF911F910F9108950F935E
:1014F0001F93CF93DF93EC0188DF8C01CE01D4DF03
:10150000800F911FDF91CF911F910F9108950F933D
:101510001F93CF93DF93EC01C0DF8C01CE01C4DFBA
:10152000800F911FDF91CF911F910F9108958F929E
:101530009F92AF92BF92CF92DF92EF92FF920F9362
:101540001F93CF93DF93CDB7DEB7A1970FB6F89473
:10155000DEBF0FBECDBF7C01C42EE52FCB01D22E46
:1015600019A221E02D1510F02AE0D22E8E010F5D78
:101570001F4F8D2C912CA12CB12C6C2D7E2FA501F1
:1015800094010E941B968C2DD29E8019112401502B
:1015900011098A3014F4805D01C0895CF8018083F0
:1015A000211531054105510521F0C22EE32FCA0155
:1015B000E4CFB801C70129DFA1960FB6F894DEBFCA
:1015C0000FBECDBFDF91CF911F910F91FF90EF9094
:1015D000DF90CF90BF90AF909F908F900895CF9263
:1015E000DF92EF92FF920F931F93CF93DF93EC0163
:1015F0006A017B012115310579F4E881F9810190B7
:10160000F081E02D642FDF91CF911F910F91FF901A
:10161000EF90DF90CF9019942A303105D9F477FFFD
:1016200018C06DE23ADF8C0144275527BA014C19E6
:101630005D096E097F092AE0CE0179DF800F911FD5
:10164000DF91CF911F910F91FF90EF90DF90CF909E
:1016500008952AE0B701A601CE01DF91CF911F9135
:101660000F91FF90EF90DF90CF9061CF9A01AB0187
:10167000662757FD6095762FB2CF0F931F93CF93B8
:10168000DF93EC019A01AB01662757FD6095762F39
:10169000A6DF8C01CE0108DF800F911FDF91CF9173
:1016A0001F910F9108950F931F93CF93DF93EC0138
:1016B00096DF8C01CE01F8DE800F911FDF91CF9174
:1016C0001F910F9108952115310541F4DC01ED9131
:1016D000FC910190F081E02D642F199428CF0F9395
:1016E0001F93CF93DF93EC019A01462F50E060E007
:1016F00070E0E9DF8C01CE01D7DE800F911FDF9112
:10170000CF911F910F9108950F931F93CF93DF9364
:10171000EC01D9DF8C01CE01C7DE800F911FDF9174
:10172000CF911F910F9108954F925F926F927F9288
:101730008F929F92AF92BF92CF92DF92EF92FF92E1
:101740000F931F93CF93DF93EC016A017B01B22EBD
:101750009A01AB01C701B6010E94CC95882319F00C
:101760006AEC7AE026C026013701E89477F82FEF7B
:101770003FEF4FE75FE7C301B2010E94CC958111B3
:101780000CC02FEF3FEF4FE75FE7C301B201ACD6CC
:1017900018161CF46EEC7AE00CC02FEF3FEF4FE709
:1017A0005FE4C701B6010E9419941816A4F462ED13
:1017B0007AE0CE01DF91CF911F910F91FF90EF90D2
:1017C000DF90CF90BF90AF909F908F907F906F9061
:1017D0005F904F901ACE2FEF3FEF4FE75FECC701BE
:1017E000B60182D687FDE3CF20E030E0A901C70132
:1017F000B6017AD687FF09C06DE2CE014EDE8C01BC
:10180000F7FAF094F7F8F09402C000E010E0A12C91
:1018100060E070E080E09FE3AB1439F020E030E05E
:1018200040E251E465D6A394F7CF9B01AC01C70118
:10183000B60194D56B017C01F9D62B013C0122D76E
:101840009B01AC01C701B60188D56B017C012AE080
:10185000B301A201CE016BDE080F191FBB2031F0CE
:101860006AE677E0CE01D1DD080F191F7B2C7720C7
:1018700021F120E030E040E251E4C701B6010E94CE
:10188000D8946B017C01CDD64B01AA2497FCA0947F
:10189000BA2C2AE030E0B501A401CE01A0DE080F89
:1018A000191FC501B401F0D69B01AC01C701B601F7
:1018B00054D56B017C017A94DACFC801DF91CF91C6
:1018C0001F910F91FF90EF90DF90CF90BF90AF905E
:1018D0009F908F907F906F905F904F90089524CF4E
:1018E0000F931F93CF93DF93EC011EDF8C01CE018A
:1018F000DBDD800F911FDF91CF911F910F91089534
:101900000F931F93CF93DF93EC010E943C84688771
:1019100079878A879B87E881F9810680F781E02DA6
:10192000CE01199597FF15C00E943C840885198542
:101930002A853B85601B710B820B930B0C811D81EB
:101940002E813F81601771078207930720F38FEF85
:101950009FEFDF91CF911F910F910895FC01448378
:101960005583668377830895CF92DF92EF92FF923B
:101970000F931F93CF93DF937C016A01EB0100E08B
:1019800010E00C151D0541F0C701BADF97FD04C03A
:1019900089930F5F1F4FF5CFC801DF91CF911F9142
:1019A0000F91FF90EF90DF90CF9008954F925F924C
:1019B0006F927F928F929F92AF92BF92CF92DF925F
:1019C000EF92FF920F931F93CF93DF934C01EB01A4
:1019D00086E0849F8001859F100D1124060F171F3C
:1019E000FB01E017F10708F582819381892B19F13A
:1019F0003696F7CF4081518164817581DA01A60F57
:101A0000B71F2C91332727FD30958217930709F5CF
:101A10006F5F7F4F75836483228133816217730701
:101A200051F03696E017F10728F3C40169DF97FDFE
:101A300046C0FE01F7CFEC1BFD0BF595E7952BEAB1
:101A40003AEAE29FC001E39F900DF29F900D1124AE
:101A500038C06115710529F3A480B5809501215026
:101A6000310935832483DA01A20FB31FAC91BB2760
:101A7000A7FDB0958A179B07F9F421153105C9F028
:101A80006A017B01E21AF30AE40EF51E412C512C87
:101A9000D6016D906D01D7017D907D01671006C064
:101AA000BFEF4B1A5B0A4216530690F342165306D9
:101AB00099F6B582A482B5CF232B71F6B2CF8FEF02
:101AC0009FEFDF91CF911F910F91FF90EF90DF90EB
:101AD000CF90BF90AF909F908F907F906F905F90CE
:101AE0004F900895CF93DF9300D000D0CDB7DEB7ED
:101AF000FE01319626E0DF011D922A95E9F77A83EF
:101B000069835C834B8341E050E0BF014FDF21E0FC
:101B1000892B09F020E0822F26960FB6F894DEBFBD
:101B20000FBECDBFDF91CF910895DCCFFC01808146
:101B300091810C947197CF93DF93EC018881998107
:101B4000009711F00E947197198218821D821C82E1
:101B50001B821A82DF91CF9108950F931F93CF9329
:101B6000DF93EC018B016F5F7F4F888199810E9429
:101B70000098009731F0998388831B830A8381E062
:101B800001C080E0DF91CF911F910F910895CF9315
:101B9000DF93EC0188819981892B29F08A819B81CF
:101BA0008617970758F4CE01D8DF882341F08C813F
:101BB0009D81892B19F4E881F981108281E0DF9100
:101BC000CF910895EF92FF920F931F93CF93DF93DE
:101BD000EC017B018A01BA01DADF811103C0CE0179
:101BE000AADF07C01D830C83B701888199810E94F9
:101BF0003299CE01DF91CF911F910F91FF90EF901D
:101C00000895FC01118210821382128215821482BF
